:020000040000FA
:04000000DEEF12F02D
:0221A800120023
:1021AB00286E756C6C290001C0FEF202C0FFF212A2
:1021BB0000D30E066E030E076EB3EC17F01200027F
:1021CB0050030BAA6E01C0A9FFA69CA69EA6800079
:1021DB00F000F0A8501200C6500F0B080AD8B40438
:1021EB00D0C6500F0B0B0AD8B4C586C7A0FED7C9F3
:1021FB00501200D30E016E030E026E000E046E0021
:10220B000E036E040E066E000E056E58EC1BF012DC
:10221B0000FF0E056EFF0E066EFF0E076E7F0E089B
:10222B006E05C001F006C002F007C003F008C00441
:10223B00F0120001C0F6FF02C0F7FFF86A0201209E
:10224B00EE21F0FE51D926FF51DA220C0E0900F5D2
:10225B00CFDEFFE806FBE2120001500302F3CF05CD
:10226B00F0F4CF06F001500402F35006260250039F
:10227B0002F350062605C001F006C002F012000161
:10228B0050021003100410D8B408D0000E011A002D
:10229B000E021A000E031A800E041A01C001F0027E
:1022AB00C002F003C003F004C004F01200D00E0310
:1022BB006EFF0E046E01C005F002C006F003500560
:1022CB002604500622065006E10A0E055CD8B00221
:1022DB00D0010E01D0000E016E026A1200BF0E0378
:1022EB006EFF0E046E01C005F002C006F003500530
:1022FB002604500622065006E11A0E055CD8B002E1
:10230B00D0010E01D0000E016E026A120014BE0540
:10231B00D0145010E11304D8B00DD013C015F01425
:10232B00C016F0151E161E154A162A15C013F016E8
:10233B00C014F0120013C013F014C014F0120000FC
:10234B000E056E000E046E000E056E000E046E0A76
:10235B00D0150E036EC60EE82EFED7032EFCD7004B
:10236B00D0044A052A0150045C02500558D8B0121B
:10237B0000EFD708C305F009C306F00AC307F00B3B
:10238B00C308F001C005F002C006F003C007F0045B
:10239B00C008F0089E05C001F006C002F007C0039C
:1023AB00F008C004F01200456E3DC00CF03EC00DAD
:1023BB00F03FC00EF040C00FF041C010F042C01112
:1023CB00F043C012F044C013F0210E0201FE25149D
:1023DB006E000EFF21156E4550B8EC36F012000062
:1023EB000E106E000E0F6E0BD00EC001F0026A0CB9
:1023FB00C003F00DC004F003EC16F00F4A102A0FC7
:10240B00500A24D96E10500B20DA6EDF500E6E0E70
:10241B0050D8B41200E9D7056EC580C5B0FED7C73A
:10242B00A403D0046A042A01D0046AC5501F0B040C
:10243B00100009D8A4F4D7780EEBEC13F0000EEBD8
:10244B00EC13F00550EBEC13F0C584C5A41200FDA2
:10245B00D7010E076E200E01180210D8B414D0F756
:10246B000E036EFF0E046E01C005F002C006F003F2
:10247B0050052604500622065004E1050E055CD8D3
:10248B00A002D0000E076E07C001F0026A12000115
:10249B00C003F002C004F002D0014A022A01C0F6C8
:1024AB00FF02C0F7FF000EF86E0F0EF76403D008A3
:1024BB0000F55005D0F6CFE9FFF7CFEAFFEF50005C
:1024CB0009D8A4EAD70350015C016E0450025802EC
:1024DB006E1200000E0001641B000E651B000E66E1
:1024EB001B800E671B60C034F061C035F062C036D4
:1024FB00F063C037F064C038F065C039F066C03A9D
:10250B00F067C03BF0A6EC28F034C060F035C0613A
:10251B00F036C062F037C063F01200C580C5B0FE64
:10252B00D7EE0EEBEC13F0C7A403D0046A042A0118
:10253B00D0046AC5501F0B04100009D8A4F4D71E91
:10254B000EEBEC13F0C7A403D0046A042A01D004E9
:10255B006AC5501F0B04100009D8A4F4D7C584C555
:10256B00A41200FDD7BF0E096EFF0E0A6E07C00B3B
:10257B00F008C00CF009500B260A500C220C500628
:10258B00E11A0E0B5CD8B002D0010E01D0000E0D7B
:10259B006E0E6A0D500E10D8B406D0200E07100721
:1025AB006E0850086E120007C007F008C008F01242
:1025BB0000AB0EF66E210EF76E000EF86E03EECC2E
:1025CB00F010EE07F00900F5CFEEFFE550E150FA01
:1025DB00E103EED3F014EE00F0EE6AE550E150FCAF
:1025EB00E1E250FAE103EE00F0B40EEE6AE806FD0C
:1025FB00E10201FF6BFE6B000107EF56F0F00E00DE
:10260B0001F86F000EF96FECC0FAF0EDC0FBF000B3
:10261B000EFD6F000EFC6F000EFF6F000EFE6FFACB
:10262B000EE46F000EE56FEEC0E6F0EFC0E7F0F8DA
:10263B000EE86F000EE96F87EC13F00001FC51EC14
:10264B0025D96EFD51ED21DA6E000EDF6E120003FF
:10265B00C007F004C008F001C009F002C00AF0077F
:10266B0050056E0850066E074A082A05C0F6FF068D
:10267B00C0F7FF000EF86E09C0D9FF0AC0DAFF09D8
:10268B004A0A2A0F0EF76403D00800F55005D0F65E
:10269B00CFE9FFF7CFEAFFEF50DF6EDF50D8B41270
:1026AB0000DED7000E0D6E000E0C6E000E0F6E00CE
:1026BB000E0E6E020120EE02F0FE51D926FF51DA0A
:1026CB0022DECF1EF0DDCF1FF0FF0E1E24106EFF9B
:1026DB000E1F20116E20EE04F0FE51D926FF51DAA9
:1026EB0022DECF20F0DDCF21F0FF0E2024126EFF73
:1026FB000E2120136E1CC014F01DC015F049EC19EF
:10270B00F01200E6C0EAF0E7C0EBF0000E03011791
:10271B006F000E166F17D0E4C0C0F0E5C0C1F0EA31
:10272B000E0001C26F000EC36FE8C0C4F0E9C0C554
:10273B00F0BEEC2FF00001C051030116270001C1C0
:10274B005103011723EAC0F6FFEBC0F7FFF86A0845
:10275B0000F5500009D8A4DFD716C3E4F017C3E582
:10276B00F01200C580C5B0FED70450EBEC13F0C7D8
:10277B00A403D0096A092A01D0096AC5501F0B09A5
:10278B00100009D8A4F4D70650EBEC13F0C7A40340
:10279B00D0096A092A01D0096AC5501F0B0910001C
:1027AB0009D8A4F4D70850EBEC13F0C7A403D00955
:1027BB006A092A01D0096AC5501F0B09100009D8F4
:1027CB00A4F4D7C584C5A41200FDD7036EC69EC959
:1027DB00CF02F0C9CF02F003C0C9FFC6BE1200C6BC
:1027EB00500F0B080AD8B40CD0C6500F0B0B0AD8DD
:1027FB00B407D0C6889EA6FED7C7B41200C7501226
:10280B0000C6500F0B080AD8B405D0C6500F0B0BDF
:10281B000AD8A41200C7B0FED7C7A403D0016A011F
:10282B002A01D0016AC5501F0B01100009D8A4F46E
:10283B00D7C5501200000E066E02AE06D0016C0218
:10284B001ED8B0022A010E066E04AE04D0036C042F
:10285B001ED8B0042A03500410D8B418D0010E05AA
:10286B006E04D0D89003360436052A04AEFAD7038B
:10287B0050015C04500258D8A004D00350015E04F0
:10288B0050025AD89004320332052EF1D70650D895
:10289B00B404D0016C021ED8B0022A01C001F002B0
:1028AB00C002F01200000E066E04AE06D0036C04DC
:1028BB001ED8B0042A010E066E02AE06D0016C02C1
:1028CB001ED8B0022A010E061A000E086E000E0763
:1028DB006E03500410D8B41CD0010E056E04D0D872
:1028EB009003360436052A04AEFAD7D8900736087B
:1028FB00360350015C04500258D8A005D003500198
:10290B005E0450025A0780D89004320332052EED34
:10291B00D70650D8B404D0076C081ED8B0082A07C5
:10292B00C001F008C002F01200C580C5B0FED7048C
:10293B0050EBEC13F0C7A403D0066A062A01D006AD
:10294B006AC5501F0B06100009D8A4F4D7000EEB74
:10295B00EC13F0C7A403D0066A062A01D0066AC599
:10296B00501F0B06100009D8A4F4D7000EEBEC1384
:10297B00F0C7A403D0066A062A01D0066AC5501F09
:10298B000B06100009D8A4F4D7000EEBEC13F0C71C
:10299B00A403D0066A062A01D0066AC5501F0B068F
:1029AB00100009D8A4F4D7C584C5A41200FDD72004
:1029BB00EE11F0070EDE6AE806FDE201A010D00969
:1029CB005011260A5012220B5013220C5014220DB8
:1029DB005015220E5016220F50172210501822D8C5
:1029EB009009360A360B360C360D360E360F36106E
:1029FB0036D89008320732063205320432033202DF
:102A0B00320132015002100310041005100610079A
:102A1B00100810D8A4D2D711C001F012C002F013C5
:102A2B00C003F014C004F015C005F016C006F01773
:102A3B00C007F018C008F01200000E0114096E0058
:102A4B000E02140A6E800E03140B6E7F0E04140C10
:102A5B006E09500A100B100C10D8A408D0000E01F0
:102A6B006E000E026E000E036E000E046E000E055D
:102A7B0014096E000E06140A6E800E07140B6E7F7F
:102A8B000E08140C6E09500A100B100C10D8A40869
:102A9B00D0000E056E000E066E000E076E000E08BF
:102AAB006E055001180AE10650021807E1075003A2
:102ABB001804E108500418D8B402D0D8901200D8EA
:102ACB0080120003011CA10AD013C00AF014C00B22
:102ADB00F011C00CF012C00DF0F5EC11F016BE05A4
:102AEB00D015C01AF016C01BF004D0000E1B6E00E0
:102AFB000E1A6E000E196E000E186E0CD0000E0220
:102B0B006E200E016E11C003F012C004F003EC1620
:102B1B00F0184A192A1A50185C1950800A176E1BA4
:102B2B0050800A1758D8A0EAD703011CB10AD0135A
:102B3B00C00AF014C00BF011C00CF012C00DF0F570
:102B4B00EC11F013C001F014C002F04DEC12F01AAE
:102B5B00500124116E1B500220126E1200AE0E118A
:102B6B00EC12F0D50E11EC12F0800E11EC12F0A855
:102B7B000E11EC12F03F0E11EC12F0D30E11EC1201
:102B8B00F0000E11EC12F0400E11EC12F0200E11B1
:102B9B00EC12F0000E11EC12F0A10E11EC12F0C8B9
:102BAB000E11EC12F0DA0E11EC12F0120E11EC12F7
:102BBB00F0810E11EC12F0CF0E11EC12F0D90E11B8
:102BCB00EC12F0F10E11EC12F0DB0E11EC12F040E6
:102BDB000E11EC12F0A40E11EC12F0A60E11EC1269
:102BEB00F0AF0E11EC12F0000E11EC12F0100E11F2
:102BFB00EC12F0400E11EC12F0120003500410D83E
:102C0B00B404D003500410D8A404D00150D4EC1059
:102C1B00F0120020EE04F00350D9260450DA22DE25
:102C2B0050DE10D8B416D020EE04F00350D9260491
:102C3B0050DA2210EE02F00350E1260450E222DEBD
:102C4B0050E65CE650800A096EDE50800A0958D8BF
:102C5B00B0120020EE02F00350D9260450DA22DE27
:102C6B00CF05F0DDCF06F003C0D9FF04C0DAFFDEDD
:102C7B00CF07F0DDCF08F005500724D96E065008BA
:102C8B0020DA6E01C0DFFF20EE02F00350D92604DC
:102C9B0050DA22DE2A000EDD221200C580C5B0FEFE
:102CAB00D73C0EEBEC13F0C7A403D0046A042A0143
:102CBB00D0046AC5501F0B04100009D8A4F4D70028
:102CCB000EEBEC13F0C7A403D0046A042A01D00462
:102CDB006AC5501F0B04100009D8A4F4D7180EEBCB
:102CEB00EC13F0C7A403D0046A042A01D0046AC50C
:102CFB00501F0B04100009D8A4F4D7200EEBEC13D3
:102D0B00F0C7A403D0046A042A01D0046AC5501F7B
:102D1B000B04100009D8A4F4D7000EEBEC13F0C78A
:102D2B00A403D0046A042A01D0046AC5501F0B0403
:102D3B00100009D8A4F4D7C584C5A41200FDD7018F
:102D4B00C008F002C009F003C00AF004C00BF00584
:102D5B0006D8A0060605280FE10628D8A40CD0003B
:102D6B000E026E000E016E1200084A092A0A4A0B67
:102D7B002A0506D8A0060608C0D9FF09C0DAFFDF6E
:102D8B0050D8B41ED00AC0F6FF0BC0F7FFF86A0884
:102D9B0000F5500009D8B414D005500610D8B41063
:102DAB00D008C0D9FF09C0DAFFDF50076E0AC0F6A2
:102DBB00FF0BC0F7FFF86A0800F5500718D8B4D41A
:102DCB00D708C0D9FF09C0DAFFDF50076E0AC0F67B
:102DDB00FF0BC0F7FFF86A0800F550075C016E02A5
:102DEB006AD8A00206120002BE06D0025057E1803C
:102DFB000E015CD8B0120003C007F004C008F00845
:102E0B0034083207320834083207320834083207E4
:102E1B003207C00AF008C00BF00AC007F00BC0085D
:102E2B00F0070ED89007360836E82EFBD707C00AF6
:102E3B00F008C00BF001500A2602500B2205500679
:102E4B0010D8B415D003C007F0070E0716010E08F3
:102E5B006E072A02D0D8900836072EFCD7D30E0A5D
:102E6B0024D96E030E0B20DA6E0850DF121200030A
:102E7B00C007F0070E0716010E086E072A02D0D8FE
:102E8B00900836072EFCD70850FF0A096ED30E0A9E
:102E9B0024D96E030E0B20DA6E0950DF16120000D8
:102EAB0001763577355E6E5E50D8A409D0000E746E
:102EBB006F000E756F000E766F000E776F12007439
:102ECB00C078F075C079F076C07AF077C07BF020CF
:102EDB000E05D0D8907B337A3379337833E82EF9DB
:102EEB00D778515D6E768FFF0E7417FF0E7517FF37
:102EFB000E7617000E7717960E5E5E5EAE0DD05EE9
:102F0B0050800A970FD8A0D2D7D8907733763375E5
:102F1B003374335E3EF9D70DD01F0E5E6407D0C6F7
:102F2B00D7D89074377537763777375E065E50D8BB
:102F3B00A4F7D75D50D8B408D0771F761F751F74D0
:102F4B006D000E75237623772374C074F075C075EE
:102F5B00F076C076F077C077F01200400E0C6E80E2
:102F6B000E0D6E000E0B6E020E0F6E000E0A6E0033
:102F7B000E096ED8900C32D8900C32D8900C32D8F7
:102F8B00900D32D8900D32D8900D32000E116E404C
:102F9B00D011500B24B00F11EC12F00F500F0B117E
:102FAB00EC12F00F380F0B100911EC12F0000E1091
:102FBB006EC580C5B0FED7C7A403D0086A082A0126
:102FCB00D0086AC5501F0B08100009D8A4F4D77895
:102FDB000EEBEC13F0400EEBEC13F0000E0E6E0C40
:102FEB00D009500624D96E0A500720DA6EDF50EB59
:102FFB00EC13F00E2A094A0A2A0D500E5CD8A0F0E9
:10300B00D7C584C5B4FED7102A070E1064D1D711CB
:10301B002A0C50115CD8B01200BBD70CC30BF00DAF
:10302B00C30CF00EC30DF00FC30EF001C00BF0027A
:10303B00C00CF003C00DF004C00EF00BC005F00C7B
:10304B00C006F00DC007F00EC008F0180E05D0D862
:10305B00900832073206320532E82EF9D7055009AF
:10306B006E0A6A09500A10D8A419D0D8900B3405EF
:10307B006E0C34066E0D34076E0E34086E0550065A
:10308B001007100810D8A405D0000E026E020E0116
:10309B006E1200000E026E030E016E120009280A5A
:1030AB0010D8A41CD00BC005F00CC006F00DC00747
:1030BB00F00EC008F0090ED8900536063607360814
:1030CB0036E82EF9D70550061007100810D8A402C1
:1030DB00D0010E01D0000E016E026A1200000E022A
:1030EB006E040E016E1200C580C5B0FED73C0EEB10
:1030FB00EC13F0C7A403D0086A082A01D0086AC5EC
:10310B00501F0B08100009D8A4F4D7030EEBEC13D7
:10311B00F0C7A403D0086A082A01D0086AC5501F5B
:10312B000B08100009D8A4F4D7C584C5B4FED7C5C5
:10313B0080C5B0FED73D0EEBEC13F0C7A403D0084F
:10314B006A082A01D0086AC5501F0B08100009D85D
:10315B00A4F4D7000E0F6E090E0F24D96EDA6A0095
:10316B000EDA22F1EC10F0DF6E050E0F18D8A40565
:10317B00D0C58AC588C5A811D0FDD7C59AC588C545
:10318B00B8FED7C7A403D0086A082A01D0086AC5BD
:10319B00501F0B08100009D8A4F4D70F2A050E0FE7
:1031AB0064DAD7090E046E000E056E000E066E0073
:1031BB000E076E1200000E00016815706F000E698D
:1031CB0015716F800E6A15726F7F0E6B15736F70B2
:1031DB0051711172117311D8A408D0000E686F00D1
:1031EB000E696F000E6A6F000E6B6F000E6C157020
:1031FB006F000E6D15716F800E6E15726F7F0E6FF7
:10320B0015736F7051711172117311D8A408D0001E
:10321B000E6C6F000E6D6F000E6E6F000E6F6F6B8E
:10322B00AF09D0686D691FD8B0692B6A1FD8B06A17
:10323B002B800E6B576FAF09D06C6D6D1FD8B06DB7
:10324B002B6E1FD8B06E2B800E6F57000E681B00B5
:10325B000E691B000E6A1B800E6B1B000E6C1B0095
:10326B000E6D1B000E6E1B800E6F1B6C51685D6D1F
:10327B005169596E516A596F516B59D8B002D0D8F8
:10328B00901200D88012000C50105C1150800A165E
:10329B006E0D50800A1658D8B00CD010C01AF01111
:1032AB00C01BF00CC010F00DC011F01AC00CF01BBD
:1032BB00C00DF00E50125C1350800A166E0F50802A
:1032CB000A1658D8B00CD012C01AF013C01BF00E4F
:1032DB00C012F00FC013F01AC00EF01BC00FF0029B
:1032EB000120EE3CF0FE51D926FF51DA22DFB2125B
:1032FB00000EC018F00FC019F032D00CC01AF00D30
:10330B00C01BF021D01AC001F01BC002F018C00383
:10331B00F019C004F014C005F015C006F0FEC2D9B8
:10332B00FFFFC2DAFFDECF16F0DDCF17F001D809B1
:10333B00D00500FA6E1650FD6E1750FE6EFF6AFA3E
:10334B005012001A4A1B2A1A50105C1150800A1690
:10335B006E1B50800A1658D8B0D5D7184A192A18A0
:10336B0050125C1350800A166E1950800A1658D8EA
:10337B00A01200C3D70B6EC580C5B0FED7EE0EEB07
:10338B00EC13F01E0EEBEC13F0C7A403D0086A0885
:10339B002A01D0086AC5501F0B08100009D8A4F4E5
:1033AB00D7C584C5B4FED7000E026E0A0E016EA5FA
:1033BB00EC11F0C580C5B0FED7EE0EEBEC13F00BA5
:1033CB0050EBEC13F0C7A403D0086A082A01D0080D
:1033DB006AC5501F0B08100009D8A4F4D7C584C5C3
:1033EB00B4FED7000E026E0A0E016EA5EC11F0C5ED
:1033FB0080C5B0FED7EF0EEBEC13F0C7A403D008DB
:10340B006A082A01D0086AC5501F0B08100009D89A
:10341B00A4F4D7000E0D6E000E0C6EF1EC10F0083C
:10342B006E08500A6E096A0C5009240C6E0D500A76
:10343B00200D6EC59AC588C5B8FED7F1EC10F00803
:10344B006E08500C240C6E000E0D200D6EC59AC527
:10345B0088C5B8FED7C584C5B4FED70CC006F00D21
:10346B00C007F0120000C370F001C371F002C37209
:10347B00F003C373F060C070F061C071F062C07292
:10348B00F063C073F08A0E0001646FFF0E656F70FE
:10349B00C066F071C067F072C068F073C069F01855
:1034AB000E05D0D8906933683367336633E82EF94D
:1034BB00D7665164256E6F000E65216F6F6FBF0F5E
:1034CB00D06F5104E1200E6E5DD8A009D060C060B2
:1034DB00F061C061F062C062F063C063F012006F14
:1034EB00BF06D06F5108E1090E6E5DD8B004D00055
:1034FB000E6F6F010E6E6FFF0E646FFF0E656FFF29
:10350B000E666FFF0E676F6E51E82A05D0D8906775
:10351B0033663365336433E82EF9D764C06AF065DC
:10352B00C06BF066C06CF067C06DF06A51701564CB
:10353B006F6B517115656F6C517215666F6D5173B1
:10354B0015676F6451651166116711D8B4BFD76ADF
:10355B001D646F6B1D656F6C1D666F6D1D676F64F2
:10356B005170176551711766517217675173177048
:10357B00C060F071C061F072C062F073C063F01292
:10358B0000000E126E08AE12D0081E071E061E0596
:10359B001E041E031E021E016C000E0222032204D7
:1035AB00220522062207220822010E126E10AE10EF
:1035BB00D0101E0F1E0E1E0D1E0C1E0B1E0A1E09FA
:1035CB006C000E0A220B220C220D220E220F22104F
:1035DB002209500A100B100C100D100E100F1010AA
:1035EB0010D8B43CD0010E116E0AD0D89009360A0F
:1035FB00360B360C360D360E360F361036112A10AA
:10360B00AEF4D70950015C0A5002580B5003580C0A
:10361B005004580D5005580E5006580F50075810AF
:10362B00500858D8A010D00950015E0A50025A0B0E
:10363B0050035A0C50045A0D50055A0E50065A0F8F
:10364B0050075A1050085AD89010320F320E320DC4
:10365B00320C320B320A320932112ED3D71250D818
:10366B00B410D0081E071E061E051E041E031E02E4
:10367B001E016C000E0222032204220522062207E1
:10368B0022082201C001F002C002F003C003F004C3
:10369B00C004F005C005F006C006F007C007F0082F
:1036AB00C008F0120001C00BF002C00CF005500670
:1036BB0010D8B412000BC0D9FF0CC0DAFF03C0DF67
:1036CB00FF05500B24076E06500C20086EFF0E07EB
:1036DB0024D96EFF0E0820DA6E03C0DFFF065004FC
:1036EB00E1030E055CD8A0120020EE01F00B50D9BF
:1036FB00260C50DA2203C0DFFF20EE02F00B50D96C
:10370B00260C50DA2203C0DFFF05500B24076E0690
:10371B00500C20086EFE0E0724D96EFF0E0820DA1F
:10372B006E03C0DFFF05500B24076E06500C2008FC
:10373B006EFD0E0724D96EFF0E0820DA6E03C0DF74
:10374B00FF065004E1070E055CD8A0120020EE0323
:10375B00F00B50D9260C50DA2203C0DFFF05500BBB
:10376B0024076E06500C20086EFC0E0724D96EFF42
:10377B000E0820DA6E03C0DFFF065004E1090E05C8
:10378B005CD8A012000BC007F00CC008F0071E0895
:10379B001E074A082A030E0714096E0A6A09500B02
:1037AB00260A500C220950055E0A50065AFC0E05DB
:1037BB0016FF0E06160BD00BC0D9FF0CC0DAFF0399
:1037CB00C0DFFF0506D8A006060B4A0C2A055006DB
:1037DB0010D8B41200F0D7C580C5B0FED7D00EEB11
:1037EB00EC13F0C7A403D0046A042A01D0046AC501
:1037FB00501F0B04100009D8A4F4D76A0EEBEC137E
:10380B00F0C7A403D0046A042A01D0046AC5501F70
:10381B000B04100009D8A4F4D7000EEBEC13F0C77F
:10382B00A403D0046A042A01D0046AC5501F0B04F8
:10383B00100009D8A4F4D7C584C5B4FED7C580C57C
:10384B00B0FED7D00EEBEC13F0C7A403D0046A0480
:10385B002A01D0046AC5501F0B04100009D8A4F428
:10386B00D7370EEBEC13F0C7A403D0046A042A017C
:10387B00D0046AC5501F0B04100009D8A4F4D7025A
:10388B000EEBEC13F0C7A403D0046A042A01D00496
:10389B006AC5501F0B04100009D8A4F4D7C584C502
:1038AB00B4FED7C580C5B0FED7D00EEBEC13F0C776
:1038BB00A403D0046A042A01D0046AC5501F0B0468
:1038CB00100009D8A4F4D76B0EEBEC13F0C7A403CC
:1038DB00D0046A042A01D0046AC5501F0B041000DF
:1038EB0009D8A4F4D7000EEBEC13F0C7A403D00453
:1038FB006A042A01D0046AC5501F0B04100009D8B2
:10390B00A4F4D7C584C5A41200FDD7096E0950D8FD
:10391B00A404AE1AD001C005F002C006F003C00724
:10392B00F004C008F0051E061E071E081E052A001F
:10393B000E06220722082205C00BF006C00CF0076A
:10394B00C00DF008C00EF008D001C00BF002C00C87
:10395B00F003C00DF004C00EF00150021003100470
:10396B0010D8A409D0000E016E000E026E000E03DB
:10397B006E000E046E1200960E0A6E06D00A2AD83E
:10398B00900E320D320C320B32000E0B14056E0002
:10399B000E0C14066E000E0D14076EFE0E0E1408A0
:1039AB006E0550061007100810D8B40DD0E7D70AD3
:1039BB002A010E0B26000E0C220D220E22D8900E81
:1039CB00320D320C320B32000E0B14056E000E0C46
:1039DB0014066E000E0D14076EFF0E0E14086E0506
:1039EB0050061007100810D8B407D0E1D70A06D834
:1039FB00900B360C360D360E360DBE03D0020E0A6A
:103A0B0060F5D70AA00D9ED8900A320AC005F006C1
:103A1B006A076A086A05C008F0076A066A056A053C
:103A2B00500B1206500C1207500D1208500E1209B3
:103A3B0050D8A404AE01D00E8E0BC001F00CC00206
:103A4B00F00DC003F00EC004F0120023EECCF0100A
:103A5B00EE0FF0060EDBCFE3FFE806FCE20CC01A1C
:103A6B00F00DC01BF01A501B10D8A404D00F0E1A67
:103A7B006E000E1B6E1AC001F01BC002F04DEC1253
:103A8B00F001C01EF002C01FF01AC31CF01BC31DB7
:103A9B00F01DBE0ED01E501C5C1D50800A0E6E1FFA
:103AAB0050800A0E58D8B004D01CC01EF01DC01F89
:103ABB00F01EC01CF01FC01DF018C318F019C3195D
:103ACB00F003011CA10DD016D0000E026E200E01CA
:103ADB006E0AC003F00BC004F003EC16F01E4A1F75
:103AEB002A18501E5C1F50800A0E6E1950800A0E49
:103AFB0058D8A0EAD7000E176E000E166E1FD01AFC
:103B0B00C0F6FF1BC0F7FF000EF86E0F0EF7640335
:103B1B00D00800F55005D0F6CFE9FFF7CFEAFFEF5D
:103B2B00500E6E0E50016E026A0AC003F00BC004F9
:103B3B00F003EC16F01A4A1B2A164A172A1C5016C9
:103B4B005C1750800A0E6E1D50800A0E58D8A0D7F5
:103B5B00D703011CB10DD016D0000E026E200E0142
:103B6B006E0AC003F00BC004F003EC16F01E4A1FE4
:103B7B002A18501E5C1F50800A0E6E1950800A0EB8
:103B8B0058D8A0EAD71EC00AF01FC00BF0120000D5
:103B9B000E2A6E28AE12D0281E271E261E251E2486
:103BAB001E231E221E216C000E22222322242225DC
:103BBB0022262227222822010E2A6E20AE12D02086
:103BCB001E1F1E1E1E1D1E1C1E1B1E1A1E196C00E8
:103BDB000E1A221B221C221D221E221F2220220112
:103BEB000E2A1A20EE2BF0070EDE6AE806FDE22104
:103BFB00502210231024102510261027102810D81F
:103C0B00B446D0010E296E0AD0D890213622362325
:103C1B003624362536263627362836292A28AEF47A
:103C2B00D7D8902B362C362D362E362F36303631C4
:103C3B003632362150195C22501A5823501B582407
:103C4B00501C5825501D5826501E5827501F5828B9
:103C5B00502058D8A011D02150195E22501A5A2347
:103C6B00501B5A24501C5A25501D5A26501E5A2799
:103C7B00501F5A2850205A2B80D890283227322692
:103C8B003225322432233222322132292EC9D72A2D
:103C9B0050D8B410D0321E311E301E2F1E2E1E2DAA
:103CAB001E2C1E2B6C000E2C222D222E222F22308E
:103CBB0022312232222BC019F02CC01AF02DC01B3E
:103CCB00F02EC01CF02FC01DF030C01EF031C01FF5
:103CDB00F032C020F01200000E166E000E156E00B2
:103CEB000E0F6E000E0E6E02D0084A092A010E143A
:103CFB006E08C0F6FF09C0F7FFF86A0800F5502000
:103D0B000AD8B419D0F70E0A6EFF0E0B6E08C0F668
:103D1B00FF09C0F7FFF86A0800F5500C6E0D6A0A30
:103D2B00500C260B500D220D5004E1050E0C5CD8E7
:103D3B00A002D0000E146E14C010F0116A105011B6
:103D4B0010D8B408D0D1D7000E0F6E010E0E6E082E
:103D5B004A092A30D008C0F6FF09C0F7FFF86A08F5
:103D6B0000F5500A6E0B6A0B50000AD8A423D00A38
:103D7B00502B0AD8B4ECD7060AD8B4E5D71BD0150C
:103D8B00C001F016C002F0000E046E0A0E036E3274
:103D9B00EC11F008C0F6FF09C0F7FFF86A0800F550
:103DAB0050015E000E025A300E0124156E000E02F9
:103DBB0020166ECDD7D00E0A6EFF0E0B6E08C0F616
:103DCB00FF09C0F7FFF86A0800F5500C6E0D6A0A80
:103DDB00500C260B500D220D5006E10A0E0C5CD830
:103DEB00B002D0010E01D0000E126E136A125013E6
:103DFB0010D8A4C5D70E500F10D8A40DD015C00ADB
:103E0B00F016C00BF00A1E0B1E0A4A0B2A0AC0083A
:103E1B00F00BC009F0120015C008F016C009F01223
:103E2B000004C344F005C345F006C346F007C3477F
:103E3B00F034C044F035C045F036C046F037C047CB
:103E4B00F0810E386EFF0E396E44C03AF045C03B20
:103E5B00F046C03CF047C03DF0180E05D0D8903D61
:103E6B00323C323B323A32E82EF9D73A50382442C0
:103E7B006E000E3920436E43BE0FD0435004E11742
:103E8B000E425CD8A009D034C034F035C035F036C2
:103E9B00C036F037C037F0120043BE5ED042C03898
:103EAB00F0FF0E396EFF0E3A6E7F0E3B6E000E3C2E
:103EBB006E386601D007D03C343C323B323A323953
:103ECB0032382EF6D739C03EF03AC03FF03BC040F7
:103EDB00F03CC041F03E504414386E3F504514390D
:103EEB006E405046143A6E415047143B6E38503971
:103EFB00103A103B10D8B4C7D744C038F045C0397E
:103F0B00F046C03AF047C03BF0200E05D0D8903BAE
:103F1B00323A3239323832E82EF9D7385039103A32
:103F2B00103B10D8B408D03E5044263F5045224099
:103F3B00504622415047223E1C386E3F1C396E4082
:103F4B001C3A6E411C3B6E38504416395045163A9C
:103F5B005046163B50471636D044C038F045C03952
:103F6B00F046C03AF047C03BF0200E05D0D8903B4E
:103F7B00323A3239323832E82EF9D7385039103AD2
:103F8B00103B10D8A408D0000E446E000E456E00F6
:103F9B000E466E000E16D0D8904434386E45343928
:103FAB006E46343A6E47343B6E385039103A103BFC
:103FBB0010D8B408D0000E446E000E456E800E462D
:103FCB006EBF0E476E44C034F045C035F046C03668
:103FDB00F047C037F01200C580C5B0FED7EE0EEB30
:103FEB00EC13F0C7A404D00101946B942B02D00105
:103FFB0001946BC5501F0B94110009D8A4F2D7582C
:10400B000EEBEC13F0C7A404D00101946B942B02BC
:10401B00D00101946BC5501F0B94110009D8A4F269
:10402B00D7C584C5B4FED78CC100F18DC101F18E0B
:10403B00C102F18FC103F190C104F191C105F1925D
:10404B00C106F193C107F192EC44F0C580C5B0FEF7
:10405B00D7EE0EEBEC13F0C7A404D00101946B94D4
:10406B002B02D00101946BC5501F0B94110009D882
:10407B00A4F2D7000EEBEC13F0C7A404D00101940B
:10408B006B942B02D00101946BC5501F0B94110044
:10409B0009D8A4F2D7C584C5B4FED7C580C5B0FE78
:1040AB00D7EF0EEBEC13F0C7A404D00101946B9483
:1040BB002B02D00101946BC5501F0B94110009D832
:1040CB00A4F2D7000E996F000E9A6F000E9B6F0033
:1040DB000E9C6FF1EC10F00101946F9451992595A2
:1040EB006F000E9A21966F000E9B21976F000E9C0E
:1040FB0021986F97C198F196C197F195C196F1955B
:10410B006B95C199F196C19AF197C19BF198C19C9E
:10411B00F1C59AC588C5B8FED7F1EC10F001019432
:10412B006F94519925956F000E9A21966F000E9BF7
:10413B0021976F000E9C21986F97C198F196C197AC
:10414B00F195C196F1956B95C199F196C19AF1973D
:10415B00C19BF198C19CF1C59AC588C5B8FED7F132
:10416B00EC10F00101946F94519925996F000E9A00
:10417B00219A6F000E9B219B6F000E9C219C6FC59B
:10418B008AC588C5B8FED7C584C5B4FED799C18C7E
:10419B00F19AC18DF19BC18EF19CC18FF11200C5BB
:1041AB0080C5B0FED7EE0EEBEC13F0C7A404D00124
:1041BB0001946B942B02D00101946BC5501F0B948F
:1041CB00110009D8A4F2D7480EEBEC13F0C7A404E6
:1041DB00D00101946B942B02D00101946BC5501F3D
:1041EB000B94110009D8A4F2D7C584C5B4FED78CA3
:1041FB00C100F18DC101F18EC102F18FC103F190AC
:10420B00C104F191C105F192C106F193C107F1927D
:10421B00EC44F0C580C5B0FED7EE0EEBEC13F0C747
:10422B00A404D00101946B942B02D00101946BC5B3
:10423B00501F0B94110009D8A4F2D700F0000EEB1D
:10424B00EC13F0C7A404D00101946B942B02D001A2
:10425B0001946BC5501F0B94110009D8A4F2D7C55C
:10426B0084C5B4FED7C580C5B0FED7EF0EEBEC13FB
:10427B00F0C7A404D00101946B942B02D0010194DC
:10428B006BC5501F0B94110009D8A4F2D7000E99DF
:10429B006F000E9A6F000E9B6F000E9C6FF1EC106F
:1042AB00F00101946F94519925956F000E9A219608
:1042BB006F000E9B21976F000E9C21986F97C198F2
:1042CB00F196C197F195C196F1956B95C199F196C0
:1042DB00C19AF197C19BF198C19CF1C59AC588C54C
:1042EB00B8FED7F1EC10F00101946F94519925951C
:1042FB006F000E9A21966F000E9B21976F000E9CFC
:10430B0021986F97C198F196C197F195C196F19548
:10431B006B95C199F196C19AF197C19BF198C19C8C
:10432B00F1C59AC588C5B8FED7F1EC10F001019420
:10433B006F94519925996F000E9A219A6F000E9BDD
:10434B00219B6F000E9C219C6FC58AC588C5B8FE4A
:10435B00D7C584C5B4FED799C18CF19AC18DF19B99
:10436B00C18EF19CC18FF1120060C06EF061C06F05
:10437B00F062C070F063C071F0000165BF58D0658A
:10438B005104E1800E645DD8A052D06EC044F06F32
:10439B00C045F070C046F071C047F0000E486E008B
:1043AB000E496E000E4A6E7F0E4B6E2CEC2AF044BB
:1043BB00C06EF045C06FF046C070F047C071F000A2
:1043CB0001810E6427FF0E652365BF8BD0655104F9
:1043DB00E1800E645DD8A085D06EC044F06FC045FF
:1043EB00F070C046F071C047F0000E486E000E49E9
:1043FB006E000E4A6E7F0E4B6E2CEC2AF044C06E94
:10440B00F045C06FF046C070F047C071F0000181FD
:10441B000E6427FF0E652365BF64D0655104E180F0
:10442B000E645DD8A05ED0000E656F7F0E59D0650F
:10443B00AF58D0820E645DFF0E6559D8B052D06E66
:10444B00C044F06FC045F070C046F071C047F0003B
:10445B000E486E000E496E800E4A6E0C0E4B6E2C83
:10446B00EC2AF044C06EF045C06FF046C070F047C8
:10447B00C071F0660E00016427000E652365AF3135
:10448B00D0820E645DFF0E6559D8B02BD06EC04440
:10449B00F06FC045F070C046F071C047F0000E4899
:1044AB006E000E496E800E4A6E0C0E4B6E2CEC2A73
:1044BB00F044C06EF045C06FF046C070F047C0715D
:1044CB00F0660E00016427000E652365AF0AD082EB
:1044DB000E645DFF0E6559D8B004D0FF0E656F8278
:1044EB000E646F7F0E6425666F000E6521676F6823
:1044FB006B696B170ED8906637673768376937E883
:10450B002EF9D766C06AF067C06BF068C06CF069B3
:10451B00C06DF06AC044F06BC045F06CC046F06DE6
:10452B00C047F06EC048F06FC049F070C04AF071E0
:10453B00C04BF02CEC2AF044C060F045C061F04653
:10454B00C062F047C063F060C060F061C061F062B0
:10455B00C062F063C063F0120046C058F047C05908
:10456B00F048C053F049C054F0F6D04AC0F6FF4BA8
:10457B00C0F7FF000EF86E0F0EF76403D00800F5BE
:10458B005005D0F6CFE9FFF7CFEAFFEF505A6E4A4E
:10459B004A4B2A020120EE28F0FE51D926FF51DAB0
:1045AB00225A504E6E4F6ADE504E5CDE504F58D83A
:1045BB00A0D2D020EE2AF0FE51D926FF51DA22DE0E
:1045CB00CF4CF0DDCF4DF05A504C5C000E4D58D80F
:1045DB00A0C2D00A0E5A18D8A40BD020EE02F0FEBF
:1045EB0051D926FF51DA22DECF58F0DDCF59F0B387
:1045FB00D020EE2CF0FE51D926FF51DA22DE50DE10
:10460B0010D8A40BD020EE24F0FE51D926FF51DA9E
:10461B0022DECF55F0DDCF56F023D020EE28F0FE72
:10462B0051D926FF51DA22DECF4CF0DDCF4DF020F1
:10463B00EE2CF0FE51D926FF51DA22DECF4EF0DD03
:10464B00CF4FF05A504E26000E4F224C504E5CD995
:10465B006E4D504F58DA6EDF50506E5050556E56AF
:10466B006A55C057F0575058244C6E000E59204DC8
:10467B006EFF0E4E6EFF0E4F6E20EE02F0FE51D906
:10468B0026FF51DA22DECF50F0DDCF51F04E5050E5
:10469B00264F5051224C50505C5150800A526E4D57
:1046AB0050800A5258D8B021D046C058F047C05954
:1046BB00F020EE26F0FE51D926FF51DA22DECF4C48
:1046CB00F0DDCF4DF020EE2FF0FE51D926FF51DA61
:1046DB0022DF504E6E4F6A4EBE4F064C504E264D4B
:1046EB00504F224E5053264F50542258C03DF05934
:1046FB00C03EF053C03FF054C040F020EE30F0FE0F
:10470B0051D926FF51DA22DECF41F0DDCF42F02026
:10471B00EE32F0FE51D926FF51DA22DECF43F0DD27
:10472B00CF44F05A50D9EC11F0020120EE2EF0FEDE
:10473B0051D926FF51DA22DF504C6E4D6A4CBE4DDB
:10474B000657504E6E4F6A4C504E264D504F224ED0
:10475B005058264F5059224AC0F6FF4BC0F7FF0066
:10476B000EF86E0F0EF76403D00800F55005D0F667
:10477B00CFE9FFF7CFEAFFEF500009D8B41200F5ED
:10478B00D6116E1150D8A408AE32D001C009F00278
:10479B00C00AF003C00BF004C00CF005C00DF0060E
:1047AB00C00EF007C00FF008C010F0091E0A1E0B58
:1047BB001E0C1E0D1E0E1E0F1E101E092A000E0AA9
:1047CB00220B220C220D220E220F22102209C013C3
:1047DB00F00AC014F00BC015F00CC016F00DC0178A
:1047EB00F00EC018F00FC019F010C01AF010D00165
:1047FB00C013F002C014F003C015F004C016F0058E
:10480B00C017F006C018F007C019F008C01AF00165
:10481B00500210031004100510061007100810D8D2
:10482B00A409D0000E016E000E026E000E036E0086
:10483B000E046E1200960E126E0AD0122AD8901A1F
:10484B003219321832173216321532143213322013
:10485B00EE13F0000EDE14096E000EDE140A6E006D
:10486B000EDE140B6EFE0EDE140C6EFF0EDE140D40
:10487B006EFF0EDE140E6EFF0EDE140F6EFF0EDEDD
:10488B0014106E09500A100B100C100D100E100F97
:10489B00101010D8B415D0D1D7122A010E13260040
:1048AB000E1422152216221722182219221A22D888
:1048BB00901A32193218321732163215321432134B
:1048CB003220EE13F0000EDE14096E000EDE140A19
:1048DB006E000EDE140B6EFF0EDE140C6EFF0EDE82
:1048EB00140D6EFF0EDE140E6EFF0EDE140F6EFF38
:1048FB000EDE14106E09500A100B100C100D100E5A
:10490B00100F101010D8B40BD0C7D71206D89013B5
:10491B00361436153616361736183619361A361526
:10492B00BE03D0020E1260F1D712B010D0FF0E13DF
:10493B0016FF0E14167F0E1516FF0E1616FF0E170A
:10494B0016FF0E1816FF0E1916FF0E1A16D8901218
:10495B003212C009F00A6A0B6A0C6A0D6A0E6A0FF2
:10496B006A106A0DC010F00CC00FF00BC00EF00AED
:10497B00C00DF009C00CF00B6A0A6A096A095013E2
:10498B00120A5014120B5015120C5016120D501710
:10499B00120E5018120F50191210501A121150D823
:1049AB00A408AE01D0168E13C001F014C002F0158E
:1049BB00C003F016C004F0120035C04DF036C04EE7
:1049CB00F037C04FF038C050F039C051F03AC052F8
:1049DB00F03BC053F03CC054F054AE02D0010E017A
:1049EB00D0000E4B6E4C6A4B504C10D8B410D054B8
:1049FB001E531E521E511E501E4F1E4E1E4D6C003E
:104A0B000E4E224F22502251225222532254220365
:104A1B00011BAF1C931BBF05D01B5108E11A05D816
:104A2B00B005D0000E486E010E476E04D01AC34776
:104A3B00F01BC348F018C349F019C34AF04B504C54
:104A4B0010D8A402D01CA503D04906D8A04A060052
:104A5B000E566E4F0E556E000E6D6F7CD05506D8F0
:104A6B00A056061E0E5524D96E030E5620DA6E4D37
:104A7B00C001F04EC002F04FC003F050C004F05123
:104A8B00C005F052C006F053C007F054C008F00A3E
:104A9B000E096E000E0A6E000E0B6E000E0C6E00F1
:104AAB000E0D6E000E0E6E000E0F6E000E106EC60B
:104ABB00EC1AF001C03DF002C03EF003C03FF00421
:104ACB00C040F005C041F006C042F007C043F008FB
:104ADB00C044F03DC013F03FC014F08CEC11F01348
:104AEB0050300FDF6E4706D8A048064906D8A04ABB
:104AFB00064DC019F04EC01AF04FC01BF050C01C31
:104B0B00F051C01DF052C01EF053C01FF054C02016
:104B1B00F00A0E216E000E226E000E236E000E2484
:104B2B006E000E256E000E266E000E276E000E28F0
:104B3B006ECDEC1DF019C04DF01AC04EF01BC04FDE
:104B4B00F01CC050F01DC051F01EC052F01FC053DE
:104B5B00F020C054F056BE20D0565003E15504D877
:104B6B00A01BD04D504E104F1050105110521053DF
:104B7B00105410D8A473D748BE05D0485002E14753
:104B8B0004D8B06CD74ABE08D04A5003E14904D8C8
:104B9B00A003D003011CB362D74B504C10D8A40315
:104BAB00D003011CA517D05506D8A056064B504C68
:104BBB0010D8A404D0000E466E2B0E03D0000E4668
:104BCB006E2D0E456E1E0E5524D96E030E5620DA31
:104BDB006E45C0DFFF33C011F034C012F01E0E550E
:104BEB0024136E030E5620146E49C015F04AC016DE
:104BFB00F067EC15F011C033F012C034F012001E48
:104C0B0050800B2B6E1E501E24326E1DBE32803216
:104C1B0050D8B40DD03228D8A408D0000E1B6E008B
:104C2B000E1C6E000E1D6E000E1E6E1D8E06D0002D
:104C3B000E1B6E000E1C6E000E1D6E000E1E6E22E5
:104C4B0050800B2B1A22502224336E21BE3380331B
:104C5B0050D8B40DD03328D8A408D0000E1F6E0046
:104C6B000E206E000E216E000E226E218E06D000DD
:104C7B000E1F6E000E206E000E216E000E226E1F98
:104C8B0050201021102210D8A417D0000E1B6E003C
:104C9B000E1C6E000E1D6E000E1E6E800E1D127F02
:104CAB000E1E122B501E121BC01BF01CC01CF01D25
:104CBB00C01DF01EC01EF012003250D8A409D00047
:104CCB000E1B6E000E1C6E000E1D6E000E1E6E1265
:104CDB0000335032C023F0246A235E000E245A7F27
:104CEB000E23242C6E000E24202D6E1BC027F01CCF
:104CFB00C028F01DC029F01EC02AF0000E1B6E004C
:104D0B000E1C6E000E1D6E000E1E6E000E2E6E0023
:104D1B000E2F6E000E306E000E316E000E336E28AD
:104D2B00D03350D8B411D0D8902736283629362A0C
:104D3B0036D8901B361C361D361E3631BE1B80D81E
:104D4B00902E362F36303631361F50275C205028A8
:104D5B00582150295822502A58D8A009D0318C1FDD
:104D6B0050275E2050285A2150295A22502A5A3354
:104D7B002A190E3364D5D72750281029102A10D89A
:104D8B00B411D02E800FD0D8901B361C361D361E7A
:104D9B003631BE1B80D8902E362F36303631362C1E
:104DAB0006D8A02D061DAEEFD7000E336E31AE1711
:104DBB00D0FF0E2E14236EFF0E2F14246EFF0E3019
:104DCB0014256E7F0E3114266E23502410251026C9
:104DDB0010D8B403D0010E336E02D01BB0FBD73307
:104DEB0050D8B41FD0010E1B26000E1C221D221EF4
:104DFB00221EA017D01BC023F01CC024F01DC02501
:104E0B00F01EC026F02634263225322432233223DC
:104E1B00C01BF024C01CF025C01DF026C01EF02CBA
:104E2B004A2D2A2DBE10D02D5003E12C28D8A00BD3
:104E3B00D0000E2D6E2C68000E1B6E000E1C6E002B
:104E4B000E1D6E000E1E6E2DBE05D02D5011E12CC9
:104E5B0004D8B00ED0000E2D6E000E2C6E000E1B63
:104E6B006E000E1C6E000E1D6E000E1E6E000E2BC5
:104E7B006E2CC032F032A002D01D8E01D01D9ED8F8
:104E8B009032301E6E0ED701C0D9FF02C0DAFF037D
:104E9B00C0DEFF04C0DDFF20EE02F00150D9260278
:104EAB0050DA2205C0DEFF06C0DDFF20EE04F00164
:104EBB0050D9260250DA2207C0DEFF08C0DDFF20E2
:104ECB00EE15F00150D9260250DA22040EDE6E00E8
:104EDB000EDD6E20EE17F00150D9260250DA2204B7
:104EEB000EDE6E000EDD6EFF0E096EFF0E0A6E20DB
:104EFB00EE15F00150D9260250DA22DECF0BF0DD91
:104F0B00CF0CF020EE02F00150D9260250DA22DE4F
:104F1B00CF0DF0DDCF0EF00B500D5E0C500E5A097D
:104F2B00500D260A500E2220EE19F00150D9260200
:104F3B0050DA220DC0DEFF0EC0DDFFFF0E096EFF43
:104F4B000E0A6E20EE15F00150D9260250DA22DE41
:104F5B00CF0BF0DDCF0CF020EE04F00150D9260280
:104F6B0050DA22DECF0DF0DDCF0EF00B500D5E0CC4
:104F7B00500E5A09500D260A500E2220EE1BF0013E
:104F8B0050D9260250DA220DC0DEFF0EC0DDFF2005
:104F9B00EE19F00150D9260250DA2210EE11F00171
:104FAB0050E1260250E222DECFE6FFDDCFE5FF2007
:104FBB00EE1BF00150D9260250DA2210EE13F0014D
:104FCB0050E1260250E222DECFE6FFDDCFE5FF20E7
:104FDB00EE2EF00150D9260250DA22010EDF6E20A0
:104FEB00EE2FF00150D9260250DA22010EDF6E208F
:104FFB00EE21F00150D9260250DA22000EDE6E00AF
:10500B000EDD6E20EE26F00150D9260250DA22007A
:10501B000EDE6E000EDD6E20EE24F00150D926025E
:10502B0050DA22000EDE6E000EDD6E20EE28F0014F
:10503B0050D9260250DA22000EDE6E000EDD6E20F5
:10504B00EE2AF00150D9260250DA22000EDE6E0055
:10505B000EDD6E20EE2CF00150D9260250DA220024
:10506B000EDE6E000EDD6E20EE34F00150D92602FE
:10507B0050DA225D0EDE6E5C0EDD6E20EE30F0013E
:10508B0050D9260250DA22FF0EDE6EFF0EDD6E20A7
:10509B00EE32F00150D9260250DA22000EDE6E00FD
:1050AB000EDD6E20EE0BF00150D9260250DA2200F5
:1050BB000EDE6E000EDD6E20EE0DF00150D92602D5
:1050CB0050DA22000EDE6E000EDD6E20EE0FF001C8
:1050DB0050D9260250DA22000EDE6E000EDD6E0075
:1050EB000E0F6E0F50030D01C009F002C00AF0F352
:1050FB00500926F4500A22370E0924D96E000E0AE5
:10510B0020DA6E000EDE6E000EDD6E0F50030D0109
:10511B00C009F002C00AF0F3500926F4500A2239F4
:10512B000E0924D96E000E0A20DA6E000EDF6E0F08
:10513B002A020E0F64D6D701C0FEF202C0FFF21294
:10514B00003750800B406E37503724426E36BE42CC
:10515B00804250D8B40DD04228D8A408D0000E34C9
:10516B006E000E356E000E366E000E376E368E06E6
:10517B00D0000E346E000E356E000E366E000E37FC
:10518B006E3B50800B416E40504118D8A4408C3B75
:10519B00503B24416E3ABE41804150D8B40DD041B2
:1051AB0028D8A408D0000E386E000E396E000E3AC7
:1051BB006E000E3B6E3A8E06D0000E386E000E3926
:1051CB006E000E3A6E000E3B6E4250415CD8B02220
:1051DB00D040AC02D0800E401A42C043F041C042D6
:1051EB00F043C041F034C043F038C034F043C03812
:1051FB00F035C043F039C035F043C039F036C04309
:10520B00F03AC036F043C03AF037C043F03BC037FA
:10521B00F043C03BF0000E436E425041C03CF03DAA
:10522B006A3C5E000E3D5A3DBE2CD03D5004E11A47
:10523B000E3C5CD8A026D03450351036103710D821
:10524B00B402D0010E01D0000E436E000E346E007E
:10525B000E356E000E366E000E376E41C042F015E5
:10526B00D043A005D0D89043300109436E02D0D86B
:10527B0090433234B0438E37343732363235323492
:10528B0032422A4150425CD8A0EBD740BC28D042D6
:10529B0050D8A409D0000E346E000E356E000E36B9
:1052AB006E000E376E120038503426395035223AC4
:1052BB005036223B50372237A071D043A005D0D8AF
:1052CB009043300109436E02D0D890433234B0433F
:1052DB008E37343732363235323432422A5FD03859
:1052EB0050345C395035583A5036583750800A3C58
:1052FB006E3B50800A3C58D8B025D03450385C3CBB
:10530B006E355039583D6E36503A583E6E37503BDD
:10531B00583F6EFF0E3C24346EFF0E3D20356EFF62
:10532B000E3E20366EFF0E3F20376E800E401A4326
:10533B006C4350D8A40FD0010E3426000E35223604
:10534B0022372208D03850345E3950355A3A50360D
:10535B005A3B50375A3450351036103710D8A41CDE
:10536B00D04350D8A419D0000E346E000E356E0009
:10537B000E366E000E376E1200D890343635363638
:10538B0036373643BE348043A002D0D88001D0D804
:10539B009043364250D8A4420636AEEED7000E41AB
:1053AB006E43AE0BD043C03CF07F0E3C16D8B4031B
:1053BB00D0010E416E02D034B0FBD74150D8B4208F
:1053CB00D0010E3426000E35223622372237A01894
:1053DB00D034C03CF035C03DF036C03EF037C03F56
:1053EB00F03F343F323E323D323C323CC034F03D34
:1053FB00C035F03EC036F03FC037F04228D8A4424B
:10540B002A4228D8B403D04250D8A40DD0000E3471
:10541B006E000E356E000E366E000E376E4250D893
:10542B00A402D0000E406E42A002D0368E01D036C0
:10543B009ED8904230376E40BE378E34C034F03534
:10544B00C035F036C036F037C037F0120047508009
:10545B000B506E47504724566E46BE56805650D85A
:10546B00B40DD05628D8A408D0000E446E000E45BB
:10547B006E000E466E000E476E468E08D0000E4430
:10548B006E000E456E000E466E000E476E4B508042
:10549B000B501A4B504B24556E4ABE55805550D865
:1054AB00B40DD05528D8A408D0000E486E000E4974
:1054BB006E000E4A6E000E4B6E4A8E08D0000E48E0
:1054CB006E000E496E000E4A6E000E4B6E5550D894
:1054DB00B403D05650D8A409D0000E446E000E452C
:1054EB006E000E466E000E476E12004A504402F3D9
:1054FB00CF5BF0F4CF5CF05B50516E526A536A5441
:10550B006A5C50576E586A596A5A6A49504502F399
:10551B00CF5BF0F4CF5CF05B505126000E52225360
:10552B002254225C505726000E582259225A2248E8
:10553B00504602F3CF5BF0F4CF5CF05B505126008A
:10554B000E5222532254225C505726000E582259D9
:10555B00225A2253C054F052C053F051C052F05152
:10556B006A48504502F3CF5BF0F4CF5CF05B5051CF
:10557B00265C505222000E5322000E5422495044F6
:10558B0002F3CF5BF0F4CF5CF05B5051265C5052D2
:10559B0022000E5322000E542253C054F052C0531B
:1055AB00F051C052F0516A48504402F3CF5BF0F413
:1055BB00CF5CF05B5051265C505222000E53220000
:1055CB000E54224A504502F3CF5BF0F4CF5CF05BF4
:1055DB005057265C505822000E5922000E5A224971
:1055EB00504602F3CF5BF0F4CF5CF05B5057265C78
:1055FB00505822000E5922000E5A224A504602F3EE
:10560B00CF5BF0F4CF5CF05B504C6E5C504D6E4E4C
:10561B006A4F6A4EC04FF04DC04EF04CC04DF04C2F
:10562B006A4C5057264D5058224E5059224F505AC3
:10563B002251C04CF052C04DF053C04EF054C04FED
:10564B00F0190E05D0D8904F324E324D324C32E815
:10565B002EF9D74C5057264D5058224E5059224FA9
:10566B00505A2253C054F052C053F051C052F05113
:10567B006A555056C04CF04D6A4C26000E4D228296
:10568B000E4C245B6EFF0E4D205C6E0FD0D89057E6
:10569B0036583659365A3654BE5780D890513652F2
:1056AB0036533654365B06D8A05C0659AEEFD7009E
:1056BB000E556E54AE17D0FF0E51144C6EFF0E529A
:1056CB00144D6EFF0E53144E6E7F0E54144F6E4CD2
:1056DB00504D104E104F10D8B403D0010E556E0222
:1056EB00D057B0FBD75550D8B41FD0010E5726005A
:1056FB000E582259225A225AA017D057C04CF05894
:10570B00C04DF059C04EF05AC04FF04F344F324E8F
:10571B00324D324C324CC057F04DC058F04EC05940
:10572B00F04FC05AF05B4A5C2A5CBE0DD05C500354
:10573B00E15B28D8A008D0000E576E000E586E8083
:10574B000E596E7F0E20D05CBE05D05C500EE15B17
:10575B0004D8B00BD0000E576E000E586E000E59C9
:10576B006E000E5A6E000E506E0FD05BC056F0FFDF
:10577B000E5716FF0E58167F0E5916000E5A165658
:10578B00B0598ED89056305A6E50505A1257C0445A
:10579B00F058C045F059C046F05AC047F0120040CF
:1057AB000E0A180B10D8A496D0120E0C180D10D888
:1057BB00A449D0000E056E400E046E000E076E124B
:1057CB000E066E0EC008F0B7EC13F0000E056E401F
:1057DB000E046E000E076E130E066E000E086EB7EB
:1057EB00EC13F0000E056E420E046E000E076E12E7
:1057FB000E066E000E086EB7EC13F0000E056E422F
:10580B000E046E000E076E130E066E000E086EB7BA
:10581B00EC13F0000E056E440E046E000E076E12B4
:10582B000E066E000E086EB7EC13F0000E056E44FC
:10583B000E046E000E076E130E066E000E086EB78A
:10584B00EC13F048D0000E056E400E046E000E07F0
:10585B006E130E066E0EC008F0B7EC13F0000E05BB
:10586B006E400E046E000E076E120E066E000E08D2
:10587B006EB7EC13F0000E056E420E046E000E07B1
:10588B006E120E066E000E086EB7EC13F0000E05CE
:10589B006E420E046E000E076E130E066E000E089F
:1058AB006EB7EC13F0000E056E440E046E000E077F
:1058BB006E120E066E000E086EB7EC13F0000E059E
:1058CB006E440E046E000E076E130E066E000E086D
:1058DB006EB7EC13F0420E0A180B10D8A496D01228
:1058EB000E0C180D10D8A449D0000E056E420E04F4
:1058FB006E000E076E120E066E0EC008F0B7EC139C
:10590B00F0000E056E400E046E000E076E120E06B2
:10591B006E000E086EB7EC13F0000E056E400E0411
:10592B006E000E076E130E066E000E086EB7EC13AC
:10593B00F0000E056E420E046E000E076E130E067F
:10594B006E000E086EB7EC13F0000E056E440E04DD
:10595B006E000E076E120E066E000E086EB7EC137D
:10596B00F0000E056E440E046E000E076E130E064D
:10597B006E000E086EB7EC13F048D0000E056E42A9
:10598B000E046E000E076E130E066E0EC008F0B7F7
:10599B00EC13F0000E056E400E046E000E076E1237
:1059AB000E066E000E086EB7EC13F0000E056E407F
:1059BB000E046E000E076E130E066E000E086EB709
:1059CB00EC13F0000E056E420E046E000E076E1205
:1059DB000E066E000E086EB7EC13F0000E056E444B
:1059EB000E046E000E076E120E066E000E086EB7DA
:1059FB00EC13F0000E056E440E046E000E076E13D2
:105A0B000E066E000E086EB7EC13F0440E0A180B60
:105A1B0010D8A41200120E0C180D10D8A449D000E7
:105A2B000E056E440E046E000E076E120E066E0E01
:105A3B00C008F0B7EC13F0000E056E400E046E00BC
:105A4B000E076E120E066E000E086EB7EC13F0000A
:105A5B000E056E400E046E000E076E130E066E00E2
:105A6B000E086EB7EC13F0000E056E420E046E00BE
:105A7B000E076E120E066E000E086EB7EC13F000DA
:105A8B000E056E420E046E000E076E130E066E00B0
:105A9B000E086EB7EC13F0000E056E440E046E008C
:105AAB000E076E130E066E000E086EB7EC13F01297
:105ABB0000000E056E440E046E000E076E130E06EC
:105ACB006E0EC008F0B7EC13F0000E056E400E041E
:105ADB006E000E076E120E066E000E086EB7EC13FC
:105AEB00F0000E056E400E046E000E076E130E06D0
:105AFB006E000E086EB7EC13F0000E056E420E042E
:105B0B006E000E076E120E066E000E086EB7EC13CB
:105B1B00F0000E056E420E046E000E076E130E069D
:105B2B006E000E086EB7EC13F0000E056E440E04FB
:105B3B006E000E076E120E066E000E086EB7EC139B
:105B4B00F0120074C089F075C08AF076C08BF077C4
:105B5B00C08CF089C0A1F08AC0A2F08BC0A3F08CDE
:105B6B00C0A4F0000E0001A115786F000EA21579EC
:105B7B006F800EA3157A6F7F0EA4157B6F800E7A44
:105B8B001933E17F0E7B1978117911D8A42DD074BC
:105B9B00C048F075C049F076C04AF077C04BF0743E
:105BAB00C044F075C045F076C046F077C047F02C86
:105BBB00EC2AF044C034F045C035F046C036F0470F
:105BCB00C037F074C038F075C039F076C03AF07752
:105BDB00C03BF0A6EC28F034C074F035C075F0363D
:105BEB00C076F037C077F01200A4BF07D0A451A342
:105BFB0011A21134E1A105D8B031D0FF0EA1157857
:105C0B006FFF0EA215796FFF0EA3157A6F7F0EA48F
:105C1B00157B6F785179117A117B11D8A409D07447
:105C2B00C074F075C075F076C076F077C077F0125F
:105C3B0000A4AF14D0000E0301156F210E146FB921
:105C4B000E016EFF0E026E0EEC11F001C074F0022D
:105C5B00C075F003C076F004C077F01200170E7811
:105C6B006FA1C079F0A2C07AF0A3C07BF0A4C07C76
:105C7B00F0786701D007D07C357C337B337A33796E
:105C8B0033782FF6D779C099F07AC09AF07BC09B06
:105C9B00F07CC09CF0000199519A119B119C11D87A
:105CAB00A42AD0000E856F000E866F000E876F0042
:105CBB000E886F0BD0D890A137A237A337A437012A
:105CCB000E8527000E862387238823A3AFF3D7FFE8
:105CDB000E8525786FFF0E8621796FFF0E87217A4F
:105CEB006FFF0E88217B6F7851995F79519A5B7AA0
:105CFB00519B5B7B519C5B810E9927FF0E9A23FF77
:105D0B000E9B23FF0E9C23FF0EA115786FFF0EA297
:105D1B0015796F7F0EA3157A6F000EA4157B6F009C
:105D2B000E7811A16F000E7911A26F800E7A11A35C
:105D3B006F000E7B11A46F99A108D0A151A127A2CE
:105D4B0051A223A351A323A451A4239C359C339B81
:105D5B00339A339933A151A127A251A223A351A363
:105D6B0023A451A423000E816F000E826F000E83BB
:105D7B006F000E846F81C08DF082C08EF083C08F58
:105D8B00F084C090F0000E9D6F000E9E6F000E9F72
:105D9B006F010EA06F43D09D518125916F9E518253
:105DAB0021926F9F518321936FA0518421946F9106
:105DBB0051A15D9251A2599351A359A451800A78D4
:105DCB006F9451800A7859D8A01CD09D5191258190
:105DDB006F9E519221826F9F519321836FA051949B
:105DEB0021846F9151A15F9251A25B9351A35B945C
:105DFB0051A45B9D518D279E518E239F518F23A0C4
:105E0B00519023A151A127A251A223A351A323A4B3
:105E1B0051A423D890A0339F339E339D339D519E25
:105E2B00119F11A011D8A4B7D7A151A211A311A4EE
:105E3B0011D8B454D0000E956F000E966F800E974C
:105E4B006F3F0E986F95C068F096C069F097C06A67
:105E5B00F098C06BF0000E6C6F000E6D6F800E6EC5
:105E6B006F3F0E6F6FE0EC18F00001D8A037D00039
:105E7B000E956F000E966F800E976F3F0E986F000A
:105E8B000E686F000E696F800E6A6F3F0E6B6F9519
:105E9B00C06CF096C06DF097C06EF098C06FF0E0DC
:105EAB00EC18F00001D8B006D0020E8D27000E8E34
:105EBB00238F2313D0010E8D15786F000E8E15795D
:105ECB006F000E8F157A6F000E90157B6F78518DCA
:105EDB002779518E237A518F237B5190238DC07854
:105EEB00F08EC079F08FC07AF090C07BF07B357B61
:105EFB00337A3379337833000E7825A16F000E791E
:105F0B0021A26F000E7A21A36F3F0E7B21A46F9904
:105F1B00C078F09AC079F09BC07AF09CC07BF017E8
:105F2B000ED890783779377A377B37E82EF9D778D0
:105F3B0051A1277951A2237A51A3237B51A423A1E9
:105F4B00C089F0A2C08AF0A3C08BF0A4C08CF089EA
:105F5B00C095F08AC096F08BC097F08CC098F095E6
:105F6B00C074F096C075F097C076F098C077F012B9
:105F7B0000C2C0D9FFC3C0DAFFDECFF6FFDDCFF71B
:105F8B00FFF86A0800F550250AD8A406D3C2C0D979
:105F9B00FFC3C0DAFFDE2A000EDD22000E0301195B
:105FAB006F000E186F18C31CF319C31DF31A691B6E
:105FBB0069000E0001D56F000E19D003011C81C2C0
:105FCB00C0D9FFC3C0DAFFDE2A000EDD2233D003B7
:105FDB00011C83F5D703011C85F2D703011C87EF46
:105FEB00D703011C89ECD7000ED56F010ED46F229D
:105FFB00D0C2C0D9FFC3C0DAFFDECFF6FFDDCFF7CB
:10600B00FFF86A0800F550C66FC76BC751000AD876
:10601B00A4EAD7C651200AD8B4E0D7030AD8B4E013
:10602B00D7080AD8B4D7D7060AD8B4C7D71D0AD809
:10603B00B4CED7D9D70001D451D511D8B4D9D70301
:10604B00011CB11C93C2C0D9FFC3C0DAFFDECFF66F
:10605B00FFDDCFF7FFF86A0800F5502A0AD8A42312
:10606B00D0C2C0D9FFC3C0DAFFDE2A000EDD22C4C6
:10607B00C0D9FFC5C0DAFFDFCFC6F0020EDE26DFC8
:10608B00CFC7F0000EDD22C6C0D9FFC7C0DAFFDED6
:10609B00CF18F3DDCF19F319AF41D01C81186D194F
:1060AB001FD8B0192B3BD0C2C0D9FFC3C0DAFFDE5B
:1060BB00CF08F0DDCF09F071EC1EF008C018F30922
:1060CB00C019F307D0C2C0D9FFC3C0DAFFDE2A0064
:1060DB000EDD22D00E0001C66FFF0EC76FC2C0D9F6
:1060EB00FFC3C0DAFFDECFF6FFDDCFF7FFF86A089C
:1060FB0000F550C86FC96BC651C827C751C923C912
:10610B005106E10A0EC85DD8B002D0010E01D000D5
:10611B000ED66FD76BD651D711D8A4D4D7C2C0D94E
:10612B00FFC3C0DAFFDECFF6FFDDCFF7FFF86A085B
:10613B0000F5502E0AD8A471D0000E03011B6F007E
:10614B000E1A6FC2C0D9FFC3C0DAFFDE2A000EDD04
:10615B0022C2C0D9FFC3C0DAFFDECFF6FFDDCFF717
:10616B00FFF86A0800F5502A0AD8A41CD0C2C0D97F
:10617B00FFC3C0DAFFDE2A000EDD22C4C0D9FFC583
:10618B00C0DAFFDFCFC6F0020EDE26DFCFC7F0008E
:10619B000EDD22C6C0D9FFC7C0DAFFDECF1AF3DD92
:1061AB00CF1BF33BD0C2C0D9FFC3C0DAFFDECF0891
:1061BB00F0DDCF09F071EC1EF008C01AF309C01B1B
:1061CB00F307D0C2C0D9FFC3C0DAFFDE2A000EDD51
:1061DB0022D00E0001C66FFF0EC76FC2C0D9FFC31E
:1061EB00C0DAFFDECFF6FFDDCFF7FFF86A0800F568
:1061FB0050C86FC96BC651C827C751C923C95106AF
:10620B00E10A0EC85DD8B002D0010E01D0000ED845
:10621B006FD96BD851D911D8A4D4D7C2C0D9FFC369
:10622B00C0DAFFDECFF6FFDDCFF7FFF86A0800F527
:10623B0050076E086AB8EC12F007500001E06FE0EF
:10624B0051D8B437D0C2C0D9FFC3C0DAFFDECFC636
:10625B00F0DDCFC7F0010EC627000EC723C6C0F670
:10626B00FFC7C0F7FFF86A0800F550076E086AB859
:10627B00EC12F007500001E16FE151D8B41AD0C213
:10628B00C0D9FFC3C0DAFFDECFC6F0DDCFC7F00247
:10629B000EC627000EC723C6C0F6FFC7C0F7FFF810
:1062AB006A0800F550076E086AB8EC12F007500048
:1062BB0001E26FC2C0D9FFC3C0DAFFDECFF6FFDD4C
:1062CB00CFF7FFF86A0800F550640AD8B40ED0C2B5
:1062DB00C0D9FFC3C0DAFFDECFF6FFDDCFF7FFF883
:1062EB006A0800F550690AD8A43FD0C2C0D9FFC3D1
:1062FB00C0DAFFDE2A000EDD22C4C0D9FFC5C0DA2A
:10630B00FFDFCFC6F0020EDE26DFCFC7F0000EDDBB
:10631B0022C6C0D9FFC7C0DAFFDECFCAF0DDCFCBB4
:10632B00F0000ECBBFFF0ECC6FCD6FCE6FCF6FD00B
:10633B006FD16FC0C033F0C1C034F0CAC035F0CBE1
:10634B00C036F0CCC037F0CDC038F0CEC039F0CF6E
:10635B00C03AF0D0C03BF0D1C03CF0E2EC24F033BB
:10636B00C0C0F034C0C1F01200660EE019D8A440D2
:10637B00D0C2C0D9FFC3C0DAFFDECFF6FFDDCFF747
:10638B00FFF86A0800F5CFE3F0C2C0D9FFC3C0DA4B
:10639B00FFDE2A000EDD22C4C0D9FFC5C0DAFFDF45
:1063AB00CFC6F0040EDE26DFCFC7F0000EDD22C60F
:1063BB00C0D9FFC7C0DAFFDECFDCF0DECFDDF0DE09
:1063CB00CFDEF0DECFDFF0C0C07CF0C1C07DF0DCF3
:1063DB00C07EF0DDC07FF0DEC080F0DFC081F0E377
:1063EB00C082F0DCEC3AF07CC0C0F07DC0C1F01292
:1063FB0000E00E016E000E026EF60E036EFF0E0431
:10640B006E000E066E020E056EA5EC16F001500224
:10641B0010D8A458D0C2C0D9FFC3C0DAFFDECFC694
:10642B00F0DDCFC7F0010E0001C627000EC723C653
:10643B00C0F6FFC7C0F7FFF86A0800F5CFE3F0BF5F
:10644B000EC66FFF0EC76FC2C0D9FFC3C0DAFFDE27
:10645B00CFF6FFDDCFF7FFF86A0800F550C86FC91C
:10646B006BC651C827C751C923C95106E11A0EC8BB
:10647B005DD8B002D0010E01D0000EDA6FDB6BDA03
:10648B0051DB11C4C0D9FFC5C0DAFFDFCFC6F004A2
:10649B000EDE26DFCFC7F0000EDD22C6C0D9FFC748
:1064AB00C0DAFFDECFDCF0DECFDDF0DECFDEF0DEFC
:1064BB00CFDFF0020EC2C0D9FFC3C0DAFFDE260069
:1064CB000EDD2281D7C2C0D9FFC3C0DAFFDECFF603
:1064DB00FFDDCFF7FFF86A0800F550730AD8A42A3E
:1064EB00D0C2C0D9FFC3C0DAFFDE2A000EDD22C442
:1064FB00C0D9FFC5C0DAFFDFCFC6F0020EDE26DF44
:10650B00CFC7F0000EDD22C6C0D9FFC7C0DAFFDE51
:10651B00CFD2F0DDCFD3F0C0C00AF0C1C00BF0D2A8
:10652B00C00CF0D3C00DF02BEC1DF00AC0C0F00B6B
:10653B00C0C1F01200C2C0D9FFC3C0DAFFDECFF674
:10654B00FFDDCFF7FFF86A0800F550250AD8A4172E
:10655B00D0C2C0D9FFC3C0DAFFDE2A000EDD220095
:10656B000E026E250E016EC0C003F0C1C004F00315
:10657B00EC16F0000E0001C16F010EC06F1200C2CD
:10658B00C0D9FFC3C0DAFFDE2A000EDD22000E00E9
:10659B0001C16F000EC06F1200C2C0D9FFC3C0DAB9
:1065AB00FFDECFF6FFDDCFF7FFF86A0800F55001ED
:1065BB006E026AC0C003F0C1C004F003EC16F0C257
:1065CB00C0D9FFC3C0DAFFDE2A000EDD22D2D768A6
:1065DB00C070F069C071F06AC072F06BC073F0707C
:1065EB00C09EF071C09FF072C0A0F073C0A1F09E6E
:1065FB00C06CF09FC06DF0A0C06EF0A1C06FF0201A
:10660B000E06D00001D8906F336E336D336C33E8C8
:10661B002EF8D76CC088F06DC089F06EC08AF06F11
:10662B00C08BF0A19F800EA05D4C0EA159D8A05D30
:10663B00D068C001F069C002F06AC003F06BC004FF
:10664B00F013EC18F001500210D8A409D068C06800
:10665B00F069C069F06AC06AF06BC06BF01200970A
:10666B000EF66EEE0EF76EF86A0900F5CF34F009F0
:10667B0000F5CF35F00900F5CF36F00A00F5CF372E
:10668B00F0000E386E000E396E800E3A6E030E3B24
:10669B006EA6EC28F034C09AF035C09BF036C09C47
:1066AB00F037C09DF00001885189118A118B11D8E8
:1066BB00A409D09AC068F09BC069F09CC06AF09D99
:1066CB00C06BF012009AC001F09BC002F09CC0039B
:1066DB00F09DC004F045EC11F001C068F002C069F8
:1066EB00F003C06AF004C06BF01200E00EA05D3E38
:1066FB000EA159D8B009D0800EA05D390EA159D882
:10670B00A0A5D79869996918D168C001F069C00232
:10671B00F06AC003F06BC004F0BFEC11F001C0686D
:10672B00F002C069F003C06AF004C06BF0980E0071
:10673B0001A05D3F0EA159D8B08ED0300EA05D3FA9
:10674B000EA159D8B04DD0000E996F000E986F0066
:10675B000E386E000E396E800E3A6EBF0E3B6E0019
:10676B000E486E000E496E000E4A6E400E4B6E6860
:10677B00C044F069C045F06AC046F06BC047F02CCE
:10678B00EC2AF044C034F045C035F046C036F04733
:10679B00C037F0A6EC28F034C01BF035C01CF03627
:1067AB00C01DF037C01EF0000E386E000E396E00A3
:1067BB000E3A6E400E3B6E68C034F069C035F06A1D
:1067CB00C036F06BC037F0A6EC28F034C01FF035A4
:1067DB00C020F036C021F037C022F005EC26F0A423
:1067EB00D0000E996F010E986F000E386E000E39A7
:1067FB006E800E3A6EBF0E3B6E68C034F069C035CA
:10680B00F06AC036F06BC037F0A6EC28F034C01B32
:10681B00F035C01CF036C01DF037C01EF0000E382E
:10682B006E000E396E800E3A6E3F0E3B6E68C034B2
:10683B00F069C035F06AC036F06BC037F0A6EC28B3
:10684B00F034C01FF035C020F036C021F037C02225
:10685B00F005EC26F069D01C0EA05D400EA159D8B6
:10686B00B04DD0000E996F020E986F000E386E006F
:10687B000E396EC00E3A6EBF0E3B6E68C034F069B7
:10688B00C035F06AC036F06BC037F0A6EC28F03498
:10689B00C01BF035C01CF036C01DF037C01EF00019
:1068AB000E386E000E396E800E3A6E3F0E3B6E0048
:1068BB000E486E000E496EC00E4A6E3F0E4B6E6850
:1068CB00C044F069C045F06AC046F06BC047F02C7D
:1068DB00EC2AF044C034F045C035F046C036F047E2
:1068EB00C037F0A6EC28F034C01FF035C020F036CE
:1068FB00C021F037C022F005EC26F016D0000E991F
:10690B006F030E986F000E1B6E000E1C6E800E1D1B
:10691B006EBF0E1E6E68C01FF069C020F06AC021EA
:10692B00F06BC022F005EC26F01BC068F01CC069B0
:10693B00F01DC06AF01EC06BF068C044F069C04522
:10694B00F06AC046F06BC047F068C048F069C049B8
:10695B00F06AC04AF06BC04BF02CEC2AF044C09AA2
:10696B00F045C09BF046C09CF047C09DF09AC044D8
:10697B00F09BC045F09CC046F09DC047F09AC048C4
:10698B00F09BC049F09CC04AF09DC04BF02CEC2A08
:10699B00F044C094F045C095F046C096F047C097C0
:1069AB00F06F0EF66EEE0EF76EF86A0900F5CF3843
:1069BB00F00900F5CF39F00900F5CF3AF00A00F5F0
:1069CB00CF3BF094C048F095C049F096C04AF09781
:1069DB00C04BF0770EF66EEE0EF76EF86A0900F507
:1069EB00CF44F00900F5CF45F00900F5CF46F00A8A
:1069FB0000F5CF47F02CEC2AF044C034F045C035FD
:106A0B00F046C036F047C037F0A6EC28F034C08C07
:106A1B00F035C08DF036C08EF037C08FF0670EF6B4
:106A2B006EEE0EF76E000EF86E0900F5CF38F0091A
:106A3B0000F5CF39F00900F5CF3AF00A00F5CF3B5E
:106A4B00F094C048F095C049F096C04AF097C04BFF
:106A5B00F08CC044F08DC045F08EC046F08FC0471F
:106A6B00F02CEC2AF044C034F045C035F046C0366B
:106A7B00F047C037F0A6EC28F034C074F035C07581
:106A8B00F036C076F037C077F074C044F075C0456F
:106A9B00F076C046F077C047F09AC048F09BC049EB
:106AAB00F09CC04AF09DC04BF02CEC2AF044C08007
:106ABB00F045C081F046C082F047C083F06B0EF604
:106ACB006EEE0EF76EF86A0900F5CF38F00900F597
:106ADB00CF39F00900F5CF3AF00A00F5CF3BF0942F
:106AEB00C048F095C049F096C04AF097C04BF07380
:106AFB000EF66EEE0EF76EF86A0900F5CF44F0094C
:106B0B0000F5CF45F00900F5CF46F00A00F5CF4769
:106B1B00F02CEC2AF044C034F045C035F046C036BA
:106B2B00F047C037F0A6EC28F034C08CF035C08DA0
:106B3B00F036C08EF037C08FF08CC044F08DC0455E
:106B4B00F08EC046F08FC047F094C048F095C04916
:106B5B00F096C04AF097C04BF02CEC2AF044C0845E
:106B6B00F045C085F046C086F047C087F00001991C
:106B7B00AF47D068C048F069C049F06AC04AF06BB3
:106B8B00C04BF084C038F085C039F086C03AF0872E
:106B9B00C03BF080C034F081C035F082C036F0834A
:106BAB00C037F0A6EC28F034C044F035C045F036C1
:106BBB00C046F037C047F02CEC2AF044C090F045AB
:106BCB00C091F046C092F047C093F068C060F06986
:106BDB00C061F06AC062F06BC063F090C064F0916A
:106BEB00C065F092C066F093C067F06FEC12F06076
:106BFB00C068F061C069F062C06AF063C06BF012EC
:106C0B000068C048F069C049F06AC04AF06BC04BDD
:106C1B00F084C038F085C039F086C03AF087C03BAD
:106C2B00F080C034F081C035F082C036F083C037BD
:106C3B00F0A6EC28F034C044F035C045F036C04621
:106C4B00F037C047F02CEC2AF044C090F045C091CF
:106C5B00F046C092F047C093F098C06CF099C06DAD
:106C6B00F00001D8906C376D37D8906C376D377B4F
:106C7B000E6C25F66EEE0E6D21F76EF86A000EF8AF
:106C8B00220900F5CF64F00900F5CF65F00900F596
:106C9B00CF66F00A00F5CF67F090C060F091C0614D
:106CAB00F092C062F093C063F06FEC12F060C078AA
:106CBB00F061C079F062C07AF063C07BF068C064A9
:106CCB00F069C065F06AC066F06BC067F078C060B1
:106CDB00F079C061F07AC062F07BC063F06FEC12A8
:106CEB00F060C07CF061C07DF062C07EF063C07F5D
:106CFB00F098C06CF099C06DF00001D8906C376DB6
:106D0B0037D8906C376D378B0E6C25F66EEE0E6D9B
:106D1B0021F76EF86A000EF8220900F5CF60F00932
:106D2B0000F5CF61F00900F5CF62F00A00F5CF63F3
:106D3B00F07CC064F07DC065F07EC066F07FC067FC
:106D4B00F06FEC12F060C09AF061C09BF062C09CD7
:106D5B00F063C09DF00001885189118A118B11D805
:106D6B00B4A8D4B0D4226E22C03BF011D0940E0D37
:106D7B00D0990E0BD0810E09D09A0E07D0840E0538
:106D8B00D08E0E03D0E60E01D0F80E3B6E20D03B1A
:106D9B0050166E176A1750000AD8A419D01650B0A7
:106DAB000AD8B4F2D7050AD8B4EDD7710AD8B4E82B
:106DBB00D7120AD8B4DDD70A0AD8B4DED7380AD826
:106DCB00B4DDD7120AD8B4D2D70A0AD8B4D3D72095
:106DDB00EE07F01450D9261550DA223B50186E19D5
:106DEB006ADE50185CDE501958D8A0120020EE094C
:106DFB00F01450D9261550DA22DECF16F0DDCF175E
:106E0B00F03B50165C000E1758D8A012000EC0298C
:106E1B00F00FC02AF020EE03F01450D9261550DAEB
:106E2B0022DECF2FF0DDCF30F02F503010D8B41240
:106E3B0000D89030322F32D89030322F32D8903059
:106E4B00322F3220EE03F01450D9261550DA22DE01
:106E5B00CF16F0DDCF17F0070E1616000E1716160D
:106E6B00501710D8B402D02F4A302A20EE0BF01452
:106E7B0050D9261550DA22DE50DE10D8A40BD020C4
:106E8B00EE03F01450D9261550DA22DECF39F0DD9F
:106E9B00CF3AF023D020EE07F01450D9261550DA54
:106EAB0022DECF16F0DDCF17F020EE0BF01450D909
:106EBB00261550DA22DECF18F0DDCF19F03B501833
:106ECB0026000E19221650185CD96E17501958DA75
:106EDB006EDF501A6E1A50396E3A6A020120EE3F7D
:106EEB00F0FE51D926FF51DA22DFA274D120EE0237
:106EFB00F01450D9261550DA22DF50D8A487D020B1
:106F0B00EE07F01450D9261550DA22DECF16F0DD3D
:106F1B00CF17F016503B5C016E1750D8A017280204
:106F2B006A025E20EE05F01450D9261550DA22DEE7
:106F3B00CF03F0DDCF04F032EC11F001C02DF002E5
:106F4B00C02EF02DC001F02EC002F02FC003F03088
:106F5B00C004F032EC11F001C035F002C036F0374E
:106F6B006A386A000E346E000E336E43D039C02778
:106F7B00F03AC028F0000E326E000E316E32D01493
:106F8B00C0D9FF15C0DAFFDECF16F0DDCF17F03515
:106F9B005016263650172216C0F6FF17C0F7FFF80B
:106FAB006A0800F5CF3CF0010E3526000E3622376D
:106FBB00223822000E266E000E256E07D0D8903C8C
:106FCB00322706D8A02806254A262A265008E1088B
:106FDB000E255CD8B004D027502810D8A4EFD73199
:106FEB004A322A2F50315C30503258D8A0C8D73390
:106FFB004A342A20EE05F01450D9261550DA22DE39
:10700B0050335CDE503458D8B01200B0D720EE02AB
:10701B00F01450D9261550DA22DE04D8A412002021
:10702B00EE07F01450D9261550DA22DECF16F0DD1C
:10703B00CF17F016503B5C016E1750D8A0172802E3
:10704B006A025E20EE05F01450D9261550DA22DEC6
:10705B00CF03F0DDCF04F032EC11F001C02DF002C4
:10706B00C02EF02DC001F02EC002F020EE03F01464
:10707B0050D9261550DA22DECF03F0DDCF04F032E3
:10708B00EC11F001C035F002C036F0376A386A00F7
:10709B000E346E000E336E91D0000E326E000E3138
:1070AB006E6ED014C0D9FF15C0DAFFDECF16F0DD3F
:1070BB00CF17F0355016263650172216C0F6FF178D
:1070CB00C0F7FFF86A0800F5CF3CF0010E3526003B
:1070DB000E362237223822000E166EFF0E176E0068
:1070EB000E1014016EFF0E1114026E3CC003F0045F
:1070FB006A32EC11F001C018F002C019F0000E1248
:10710B0014016EFF0E1314026E3C500008036E0048
:10711B000ED8A0E82A0108046E32EC11F0015018C9
:10712B00260250192219C018F0196A165018161792
:10713B005019161250016E026A3C500008036E0083
:10714B000ED8A0E82A0108046E32EC11F010503C66
:10715B0002F3CF1AF0F4CF1BF001501A2602501B8A
:10716B00221BC01AF01B6AFF0E1A16000E1B1618F4
:10717B00501A10236E19501B10246E314A322A39C3
:10718B0050315C3A503258D8A08CD720EE03F01413
:10719B0050D9261550DA22DECF16F0DDCF17F03995
:1071AB0050165E3A50175A16503526175036220095
:1071BB000E3722000E3822334A342A20EE05F01403
:1071CB0050D9261550DA22DE50335CDE503458D8B5
:1071DB00B0120062D720EE02F01450D9261550DA07
:1071EB0022DF50D8A4D8D020EE07F01450D92615A2
:1071FB0050DA22DECF16F0DDCF17F016503B5C01D4
:10720B006E1750D8A01728026A025E20EE05F01404
:10721B0050D9261550DA22DECF03F0DDCF04F03241
:10722B00EC11F001C02DF002C02EF02DC001F02E9C
:10723B00C002F02FC003F030C004F032EC11F001AB
:10724B00C035F002C036F0376A386A000E346E0073
:10725B000E336E94D00CC02BF00DC02CF039C02720
:10726B00F03AC028F0000E326E000E316E7DD01455
:10727B00C0D9FF15C0DAFFDECF16F0DDCF17F03522
:10728B005016263650172216C0F6FF17C0F7FFF818
:10729B006A0800F5CF3CF0010E3526000E3622377A
:1072AB00223822000E266E000E256E52D03CA024F2
:1072BB00D02BC001F02CC002F029C003F02AC0046F
:1072CB00F010C005F011C006F0FEC2D9FFFFC2DA04
:1072DB00FFDECF16F0DDCF17F001D809D00500FA8D
:1072EB006E1650FD6E1750FE6EFF6AFA50120000BC
:1072FB000E1F6E000E1E6E23D02BC001F02CC00291
:10730B00F029C003F02AC004F012C005F013C00628
:10731B00F0FEC2D9FFFFC2DAFFDECF16F0DDCF17CA
:10732B00F001D809D00500FA6E1650FD6E1750FE0D
:10733B006EFF6AFA501200000E216E000E206ED8FE
:10734B00903C322B4A2C2A2706D8A02806254A2601
:10735B002A265008E1080E255CD8B004D027502807
:10736B0010D8A4A4D7314A322A2F50315C30503276
:10737B0058D8A07DD7294A2A2A334A342A20EE0529
:10738B00F01450D9261550DA22DE50335CDE50341F
:10739B0058D8B012005FD720EE02F01450D9261542
:1073AB0050DA22DE04D8A4120020EE07F01450D9D4
:1073BB00261550DA22DECF16F0DDCF17F016503B34
:1073CB005C016E1750D8A01728026A025E20EE05EA
:1073DB00F01450D9261550DA22DECF03F0DDCF049E
:1073EB00F032EC11F001C02DF002C02EF02DC001D7
:1073FB00F02EC002F020EE03F01450D9261550DA0F
:10740B0022DECF03F0DDCF04F032EC11F001C035FA
:10741B00F002C036F0376A386A000E346E000E3355
:10742B006EB8D00CC02BF00DC02CF0000E326E00DD
:10743B000E316E8FD014C0D9FF15C0DAFFDECF1618
:10744B00F0DDCF17F0355016263650172216C0F642
:10745B00FF17C0F7FFF86A0800F5CF3CF0010E35B7
:10746B0026000E362237223822000E166EFF0E171C
:10747B006E000E1014016EFF0E1114026E3CC00351
:10748B00F0046A32EC11F001C018F002C019F000E0
:10749B000E1214016EFF0E1314026E3C5000080303
:1074AB006E000ED8A0E82A0108046E32EC11F00130
:1074BB005018260250192219C018F0196A165018C4
:1074CB0016175019161250016E026A3C5000080331
:1074DB006E000ED8A0E82A0108046E32EC11F010F1
:1074EB00503C02F3CF1AF0F4CF1BF001501A2602D6
:1074FB00501B221BC01AF01B6AFF0E1A16000E1B24
:10750B001618501A10236E19501B10246E2BC00125
:10751B00F02CC002F029C003F02AC004F023C005F0
:10752B00F024C006F0FEC2D9FFFFC2DAFFDECF1691
:10753B00F0DDCF17F001D809D00500FA6E1650FD1B
:10754B006E1750FE6EFF6AFA5012002B4A2C2A312E
:10755B004A322A3950315C3A503258D8A06BD72076
:10756B00EE03F01450D9261550DA22DECF16F0DDDB
:10757B00CF17F03950165E3A50175A16503526175A
:10758B00503622000E3722000E3822294A2A2A337F
:10759B004A342A20EE05F01450D9261550DA22DE93
:1075AB0050335CDE503458D8B012003BD7000E007D
:1075BB0001A36F000EA26F7EC0B4F07FC0B5F08048
:1075CB00C0B6F081C0B7F0B7AF16D0000EA36F01F5
:1075DB000EA26FB4C001F0B5C002F0B6C003F0B795
:1075EB00C004F045EC11F001C0B4F002C0B5F003DB
:1075FB00C0B6F004C0B7F0000E0001BB6F000EBAAE
:10760B006F18C3A7F019C3A8F0A251A311D8A403F4
:10761B00D003011CA514D00001A251A311D8A404BE
:10762B00D0000E8D6F2B0E03D0000E8D6F2D0E8C98
:10763B006F8CC01EF3BA4BBB2BA707D8A0A807B4FF
:10764B00C001F0B5C002F0B6C003F0B7C004F01330
:10765B00EC18F001040210D8A44CD0BF0E0001832B
:10766B006FFF0E846F8251856F866B8351852784E4
:10767B00518623865106E11A0E855DD8B002D001E2
:10768B000E01D0000E8E6F8F6B8E518F11D8B40DF3
:10769B00D01E0EBA25016E030EBB21026EE20E0345
:1076AB006EFF0E046E2DEC13F00CD01E0EBA2501DE
:1076BB006E030EBB21026EEA0E036EFF0E046E2DDF
:1076CB00EC13F00001FD0EA727FF0EA8237CC011C1
:1076DB00F07DC012F01E0E136E030E146EA7C015B4
:1076EB00F0A8C016F067EC15F011C07CF012C07D4D
:1076FB00F01200B4C001F0B5C002F0B6C003F0B791
:10770B00C004F013EC18F001500210D8A435D0BF10
:10771B000E0001836FFF0E846F8251856F866B8322
:10772B0051852784518623865106E11A0E855DD833
:10773B00B002D0010E01D0000E906F916B90519161
:10774B0011D8B40DD01E0EBA25016E030EBB21024B
:10775B006EE60E036EFF0E046E2DEC13F0B2D71E09
:10776B000EBA25016E030EBB21026EEE0E036EFFE9
:10777B000E046E2DEC13F0A5D7000E0001BC6F00AC
:10778B000EBD6F800EBE6F3F0EBF6F000EB96F0048
:10779B000EB86FB4C001F0B5C002F0B6C003F0B7BD
:1077AB00C004F0000E056E000E066E000E076E0094
:1077BB000E086E22EC15F0D8A01ED078D0BCC044B9
:1077CB00F0BDC045F0BEC046F0BFC047F0000E484C
:1077DB006E000E496E200E4A6E410E4B6E2CEC2A3B
:1077EB00F044C0BCF045C0BDF046C0BEF047C0BFC2
:1077FB00F00001B84BB92BB4C068F0B5C069F0B656
:10780B00C06AF0B7C06BF0000E486E000E496E20D8
:10781B000E4A6E410E4B6EBCC044F0BDC045F0BE6F
:10782B00C046F0BFC047F02CEC2AF044C06CF045CA
:10783B00C06DF046C06EF047C06FF0E0EC18F00082
:10784B0001D8A01FD0BBD7BCC01BF0BDC01CF0BE65
:10785B00C01DF0BFC01EF0000E1F6E000E206E206C
:10786B000E216E410E226E05EC26F01BC0BCF01CE7
:10787B00C0BDF01DC0BEF01EC0BFF00001B807D8E0
:10788B00A0B907B4C068F0B5C069F0B6C06AF0B76C
:10789B00C06BF0BCC06CF0BDC06DF0BEC06EF0BF75
:1078AB00C06FF0E0EC18F00001D8A0CDD782C00774
:1078BB00F0086AB8EC12F007500001A96FA9C0A636
:1078CB00F0670EA919D8A41BD003011A511B11D8AC
:1078DB00A404D0000E1B6F010E1A6F1BBF05D01B2B
:1078EB005109E11A05D8B006D0000E0001A56F06AC
:1078FB000EA46F09D01AC3A4F01BC3A5F004D003C8
:10790B00011BAFF8D7F1D7670E0001A919D8A42234
:10791B00D0B9AF06D0FC0EB85DFF0EB959D8A01880
:10792B00D0FF0E836FFF0E846FA4C085F0A5C086B9
:10793B00F08351852784518623B851855D8651800C
:10794B000A876FB951800A8759D8A002D0660E01F9
:10795B00D0650EA66FA4C09CF0A5C09DF0670EA9C4
:10796B0019D8A405D0660EA619D8B4B9AF02D09C0D
:10797B004B9D2B660EA619D8A416D0B9AF0CD00010
:10798B000EBC6F000EBD6F800EBE6F3F0EBF6F0043
:10799B000EB96F000EB86F670EA919D8B404D0B822
:1079AB00519C27B9519D23000EB36F000EB26FB4DB
:1079BB00C0AAF0B5C0ABF0B6C0ACF0B7C0ADF0BC70
:1079CB00C088F0BDC089F0BEC08AF0BFC08BF07B11
:1079DB00D0AAC01BF0ABC01CF0ACC01DF0ADC01EDC
:1079EB00F0BCC01FF0BDC020F0BEC021F0BFC02254
:1079FB00F005EC26F01BC034F01CC035F01DC03672
:107A0B00F01EC037F016EC1FF034C0AEF035C0AF2F
:107A1B00F036C0B0F037C0B1F0AEC074F0AFC07587
:107A2B00F0B0C076F0B1C077F055EC17F074C0A091
:107A3B00F075C0A1F0AAC060F0ABC061F0ACC06241
:107A4B00F0ADC063F0BCC048F0BDC049F0BEC04A49
:107A5B00F0BFC04BF0AEC044F0AFC045F0B0C04675
:107A6B00F0B1C047F02CEC2AF044C064F045C0657F
:107A7B00F046C066F047C067F06FEC12F060C0AA2A
:107A8B00F061C0ABF062C0ACF063C0ADF0BCC01B2A
:107A9B00F0BDC01CF0BEC01DF0BFC01EF0000E1F1D
:107AAB006E000E206E200E216E410E226E05EC260E
:107ABB00F01BC0BCF01CC0BDF01DC0BEF01EC0BF93
:107ACB00F00001B24BB32B9C51B25DB351800A83D2
:107ADB006F9D51800A8359D8A07BD7BCC044F0BDA1
:107AEB00C045F0BEC046F0BFC047F0000E486E0068
:107AFB000E496EA00E4A6E400E4B6E2CEC2AF044D3
:107B0B00C0AEF045C0AFF046C0B0F047C0B1F0AA70
:107B1B00C068F0ABC069F0ACC06AF0ADC06BF0AE42
:107B2B00C06CF0AFC06DF0B0C06EF0B1C06FF0E0E4
:107B3B00EC18F00001D8A017D0AAC001F0ABC0021E
:107B4B00F0ACC003F0ADC004F0AEC005F0AFC006A2
:107B5B00F0B0C007F0B1C008F022EC15F0D8A00BC4
:107B6B00D00001A0B108D0000EAE6F000EAF6F00B9
:107B7B000EB06F000EB16FB4C034F0B5C035F0B6B7
:107B8B00C036F0B7C037F0AEC038F0AFC039F0B088
:107B9B00C03AF0B1C03BF0A6EC28F034C0AAF035E7
:107BAB00C0ABF036C0ACF037C0ADF088C0BCF089CC
:107BBB00C0BDF08AC0BEF08BC0BFF0650E0001A641
:107BCB0019D8B405D0B8C09EF0B9C09FF004D0004E
:107BDB000E9F6F000E9E6F000E9B6F000E9A6F0034
:107BEB000E996F000E986F000EB36F000EB26FC838
:107BFB00D0AAC01BF0ABC01CF0ACC01DF0ADC01EBA
:107C0B00F0BCC01FF0BDC020F0BEC021F0BFC02231
:107C1B00F005EC26F01BC034F01CC035F01DC0364F
:107C2B00F01EC037F016EC1FF034C0AEF035C0AF0D
:107C3B00F036C0B0F037C0B1F0AEC074F0AFC07565
:107C4B00F0B0C076F0B1C077F055EC17F074C0A06F
:107C5B00F075C0A1F003011CB90DD00001A051A11A
:107C6B0011D8A408D0670EA919D8B49FAF03D09828
:107C7B004B992B3AD000019A519B11D8B49FAF224C
:107C8B00D01E0EBA25D96E030EBB21DA6E2E0EDF77
:107C9B006EBA4BBB2BA707D8A0A807000E9B6F0192
:107CAB000E9A6F10D01E0EBA25D96E030EBB21DAB9
:107CBB006E300EDF6EBA4BBB2BA707D8A0A8079868
:107CCB0007D8A0990798519911D8A4ECD71E0EBAD2
:107CDB0025D96E030EBB21DA6EA051300FDF6EBAC1
:107CEB004BBB2BA707D8A0A807AAC060F0ABC061FD
:107CFB00F0ACC062F0ADC063F0BCC048F0BDC04991
:107D0B00F0BEC04AF0BFC04BF0AEC044F0AFC045B0
:107D1B00F0B0C046F0B1C047F02CEC2AF044C06480
:107D2B00F045C065F046C066F047C067F06FEC12D7
:107D3B00F060C0AAF061C0ABF062C0ACF063C0AD44
:107D4B00F0BCC01BF0BDC01CF0BEC01DF0BFC01E00
:107D5B00F0000E1F6E000E206E200E216E410E22C3
:107D6B006E05EC26F01BC0BCF01CC0BDF01DC0BEE8
:107D7B00F01EC0BFF000019E07D8A09F07B24BB307
:107D8B002B9C51B25DB351800A836F9D51800A8346
:107D9B0059D8B008D0BBBF2CD7BB5104E14B0EBA9E
:107DAB005DD8A026D79A519B11D8A40ED003011CE5
:107DBB00A90BD01E0E0001BA25D96E030EBB21DA1A
:107DCB006E2E0EDF6EBA4BBB2B1E0E0001BA25D9E1
:107DDB006E030EBB21DA6E000EDF6E650EA619D890
:107DEB00A475D4000EB36F4F0EB26F1E0EB225D911
:107DFB006E030EB321DA6E000EDF6E000EA36F0062
:107E0B000EA26FB9AF08D0000EA36F010EA26FB810
:107E1B006DB91FD8B0B92B000EA56F020EA46F2B36
:107E2B00D0B207D8A0B3071E0EB225D96E030EB37E
:107E3B0021DA6EB8C001F0B9C002F0000E046E0A70
:107E4B000E036E20EC14F00150300FDF6EB8C00142
:107E5B00F0B9C002F0000E046E0A0E036E58EC145B
:107E6B00F001C0B8F002C0B9F00001A407D8A0A57A
:107E7B0007A707D8A0A807B851B911D8A4D1D7A57F
:107E8B00BF05D0A551CDE1A405D8B0CAD7B207D84C
:107E9B00A0B307A251A311D8A404D0000E936F2B4B
:107EAB000E03D0000E936F2D0E926F1E0EB225D9BE
:107EBB006E030EB321DA6E92C0DFFFA707D8A0A81E
:107ECB0007B207D8A0B307BF0E836FFF0E846F8274
:107EDB0051856F866B835185278451862386510686
:107EEB00E11A0E855DD8B002D0010E01D0000E96BE
:107EFB006F976B96519711D8A404D0000E956F65B0
:107F0B000E03D0000E956F450E946F1E0EB225D941
:107F1B006E030EB321DA6E94C0DFFFA707D8A0A8BB
:107F2B00071E0EBA25016E030EBB21026E1E0EB28A
:107F3B0025036E030EB321046E2DEC13F06CEF3B97
:107F4B00F0000E056E400E046E000E076E120E064C
:107F5B006EFF0E086EB7EC13F0000E026E960E015C
:107F6B006EA5EC11F0000E056E400E046E000E07B0
:107F7B006E120E066E000E086EB7EC13F0000E05B7
:107F8B006E420E046E000E076E130E066EFF0E0889
:107F9B006EB7EC13F0000E026E960E016EA5EC118F
:107FAB00F0000E056E420E046E000E076E130E06E9
:107FBB006E000E086EB7EC13F0000E056E420E0449
:107FCB006E000E076E120E066EFF0E086EB7EC13E8
:107FDB00F0000E026E960E016EA5EC11F0000E0570
:107FEB006E420E046E000E076E120E066E000E0829
:107FFB006EB7EC13F0000E056E440E046E000E0708
:10800B006E130E066EFF0E086EB7EC13F0000E0229
:10801B006E960E016EA5EC11F0000E056E440E046B
:10802B006E000E076E130E066E000E086EB7EC1385
:10803B00F0000E056E440E046E000E076E120E0657
:10804B006EFF0E086EB7EC13F0000E026E960E016B
:10805B006EA5EC11F0000E056E440E046E000E07BB
:10806B006E120E066E000E086EB7EC13F0000E05C6
:10807B006E400E046E000E076E130E066EFF0E089A
:10808B006EB7EC13F0000E026E960E016EA5EC119E
:10809B00F0000E056E400E046E000E076E130E06FA
:1080AB006E000E086EB7EC13F0000E056E400E045A
:1080BB006E000E076E120E066EFF0E086EB7EC13F7
:1080CB00F0000E026E960E016EA5EC11F0000E057F
:1080DB006E400E046E000E076E120E066E000E083A
:1080EB006EB7EC13F0000E056E420E046E000E0719
:1080FB006E130E066EFF0E086EB7EC13F0000E0239
:10810B006E960E016EA5EC11F0000E056E420E047C
:10811B006E000E076E130E066E000E086EB7EC1394
:10812B00F0000E056E420E046E000E076E120E0668
:10813B006EFF0E086EB7EC13F0000E026E960E017A
:10814B006EA5EC11F0000E056E420E046E000E07CC
:10815B006E120E066E000E086EB7EC13F0000E05D5
:10816B006E440E046E000E076E130E066EFF0E08A5
:10817B006EB7EC13F0000E026E960E016EA5EC11AD
:10818B00F0000E056E440E046E000E076E130E0605
:10819B006E000E086EB7EC13F0000E056E440E0465
:1081AB006E000E076E120E066EFF0E086EB7EC1306
:1081BB00F0000E026E960E016EA5EC11F0000E058E
:1081CB006E440E046E000E076E120E066E000E0845
:1081DB006EB7EC13F0000E056E400E046E000E072A
:1081EB006E130E066EFF0E086EB7EC13F0000E0248
:1081FB006E960E016EA5EC11F0000E056E400E048E
:10820B006E000E076E130E066E000E086EB7EC13A3
:10821B00F0AA0E266E000E0D6E000E0C6E000E05F3
:10822B006E400E046E000E076E120E066E26C00810
:10823B00F0B7EC13F0000E056E420E046E000E0745
:10824B006E130E066E26C008F0B7EC13F0000E0589
:10825B006E420E046E000E076E120E066E26C008DE
:10826B00F0B7EC13F0000E056E440E046E000E0713
:10827B006E130E066E26C008F0B7EC13F0000E0559
:10828B006E440E046E000E076E120E066E26C008AC
:10829B00F0B7EC13F0000E056E400E046E000E07E7
:1082AB006E130E066E26C008F0B7EC13F0000E022C
:1082BB006E640E016EA5EC11F0000E056E400E04FF
:1082CB006E000E076E120E066E550E086EB7EC138F
:1082DB00F0000E056E420E046E000E076E130E06B6
:1082EB006E550E086EB7EC13F0000E056E420E04C1
:1082FB006E000E076E120E066E550E086EB7EC135F
:10830B00F0000E056E440E046E000E076E130E0683
:10831B006E550E086EB7EC13F0000E056E440E048E
:10832B006E000E076E120E066E550E086EB7EC132E
:10833B00F0000E056E400E046E000E076E130E0657
:10834B006E550E086EB7EC13F0000E026E640E0144
:10835B006EA5EC11F00C4A0D2A0DBE60D70D500422
:10836B00E10A0E0C5CD8A05AD7000E056E400E0425
:10837B006E000E076E120E066E000E086EB7EC1333
:10838B00F0000E056E420E046E000E076E130E0605
:10839B006E000E086EB7EC13F0000E056E420E0465
:1083AB006E000E076E130E066E000E086EB7EC1302
:1083BB00F0000E056E440E046E000E076E130E06D3
:1083CB006E000E086EB7EC13F0000E056E440E0433
:1083DB006E000E076E120E066E000E086EB7EC13D3
:1083EB00F0000E056E400E046E000E076E130E06A7
:1083FB006E000E086EB7EC13F0000E286E800E2781
:10840B006E000E0F6E000E0E6E000E056E400E040B
:10841B006E000E076E120E066E27C008F0B7EC1337
:10842B00F0283428300A6E2730276E0AC028F00057
:10843B000E026E0A0E016EA5EC11F00E4A0F2A0FFA
:10844B00BEE3D70F5004E1080E0E5CD8A0DDD700B9
:10845B000E056E400E046E000E076E120E066E00B9
:10846B000E086EB7EC13F0000E286E800E276E0010
:10847B000E116E000E106E000E056E420E046E0095
:10848B000E076E130E066E27C008F0B7EC13F0281C
:10849B003428300A6E2730276E0AC028F0000E02EF
:1084AB006E0A0E016EA5EC11F0104A112A11BEE3F3
:1084BB00D7115004E1080E105CD8A0DDD7000E05D3
:1084CB006E420E046E000E076E130E066E000E0843
:1084DB006EB7EC13F0000E286E800E276E000E1395
:1084EB006E000E126E000E056E420E046E000E072D
:1084FB006E120E066E27C008F0B7EC13F028342866
:10850B00300A6E2730276E0AC028F0000E026E0A62
:10851B000E016EA5EC11F0124A132A13BEE3D7130A
:10852B005004E1080E125CD8A0DDD7000E056E4298
:10853B000E046E000E076E120E066E000E086EB75E
:10854B00EC13F0000E286E800E276E000E156E00D9
:10855B000E146E000E056E440E046E000E076E13A5
:10856B000E066E27C008F0B7EC13F0283428300A3B
:10857B006E2730276E0AC028F0000E026E0A0E011D
:10858B006EA5EC11F0144A152A15BEE3D71550044D
:10859B00E1080E145CD8A0DDD7000E056E440E0466
:1085AB006E000E076E130E066E000E086EB7EC1300
:1085BB00F0000E286E800E276E000E176E000E1642
:1085CB006E000E056E440E046E000E076E120E0644
:1085DB006E27C008F0B7EC13F0283428300A6E274A
:1085EB0030276E0AC028F0000E026E0A0E016EA52F
:1085FB00EC11F0164A172A17BEE3D7175004E108FF
:10860B000E165CD8A0DDD7000E056E440E046E006E
:10861B000E076E120E066E000E086EB7EC13F0000E
:10862B000E286E800E276E000E196E000E186E1936
:10863B00BE06D0195020E1080E185CD8B01CD00033
:10864B000E056E400E046E000E076E130E066E279F
:10865B00C008F0B7EC13F0283428300A6E27302707
:10866B006E0AC028F0000E026E0A0E016EA5EC1108
:10867B00F0184A192ADCD7000E056E400E046E0066
:10868B000E076E130E066E000E086EB7EC13F0009D
:10869B000E286E010E276E000E1B6E000E1A6E1B3F
:1086AB00BE06D01B501EE1080E1A5CD8B01AD000C3
:1086BB000E056E400E046E000E076E130E066E272F
:1086CB00C008F0B7EC13F0D8902734276E28342865
:1086DB006E000E026E0A0E016EA5EC11F01A4A1B0B
:1086EB002ADED7000E056E400E046E000E076E13C9
:1086FB000E066E000E086EB7EC13F0000E286E011E
:10870B000E276E000E1D6E000E1C6E1DBE06D01DBC
:10871B00501EE1080E1C5CD8B01AD0000E056E443A
:10872B000E046E000E076E120E066E27C008F0B711
:10873B00EC13F0D8902734276E2834286E000E02E5
:10874B006E0A0E016EA5EC11F01C4A1D2ADED70035
:10875B000E056E440E046E000E076E120E066E00B2
:10876B000E086EB7EC13F0000E286E010E276E008C
:10877B000E1F6E000E1E6E1FBE06D01F501EE10890
:10878B000E1E5CD8B01AD0000E056E440E046E009F
:10879B000E076E130E066E27C008F0B7EC13F0D859
:1087AB00902734276E2834286E000E026E0A0E01B5
:1087BB006EA5EC11F01E4A1F2ADED7000E056E4483
:1087CB000E046E000E076E130E066E000E086EB7CB
:1087DB00EC13F0000E286E010E276E000E216E00BA
:1087EB000E206E21BE06D021501EE1080E205CD853
:1087FB00B01AD0000E056E420E046E000E076E12FC
:10880B000E066E27C008F0B7EC13F0D8902734276C
:10881B006E2834286E000E026E0A0E016EA5EC1146
:10882B00F0204A212ADED7000E056E420E046E00A0
:10883B000E076E120E066E000E086EB7EC13F000EC
:10884B000E286E010E276E000E236E000E226E2375
:10885B00BE06D023501EE1080E225CD8B01AD00001
:10886B000E056E420E046E000E076E130E066E277B
:10887B00C008F0B7EC13F0D8902734276E283428B3
:10888B006E000E026E0A0E016EA5EC11F0224A2349
:10889B002ADED7000E056E420E046E000E076E1315
:1088AB000E066E000E086EB7EC13F0000E286E016C
:1088BB000E276E000E256E000E246E25BE06D025EB
:1088CB00501EE1080E245CD8B01AD0000E056E4085
:1088DB000E046E000E076E120E066E27C008F0B760
:1088EB00EC13F0D8902734276E2834286E000E0234
:1088FB006E0A0E016EA5EC11F0244A252ADED70074
:10890B000E056E400E046E000E076E120E066E0004
:10891B000E086EB7EC13F01200000E01017D6F0014
:10892B000E7C6F79EC18F004C07EF105C07FF17EF0
:10893B00C1D9FF7FC1DAFFDF500101086F08510A6F
:10894B006F096B20EE01F07E51D9267F51DA22DFC1
:10895B00500B6F0B5109112E6F0A512F6F20EE0424
:10896B00F07E51D9267F51DA22DF50086F08510A69
:10897B006F096B20EE05F07E51D9267F51DA22DF8D
:10898B00500B6F0B510911306F0A51316F20EE02F2
:10899B00F07E51D9267F51DA22DF50086F08510A39
:1089AB006F096B20EE03F07E51D9267F51DA22DF5F
:1089BB00500B6F0B510911326F0A51336FD8907CEA
:1089CB0035D96E7D35DA6E3A0ED926010EDA222EA6
:1089DB00C1DEFF2FC1DDFFD8907C35D96E7D35DA36
:1089EB006E480ED926010EDA2230C1DEFF31C1DD11
:1089FB00FFD8907C35D96E7D35DA6E560ED92601AF
:108A0B000EDA2232C1DEFF33C1DDFF7C4B7D2B7DC5
:108A1B00BF88D77D5104E1070E7C5DD8A082D700BB
:108A2B000E886F000E896F000E8A6F000E8B6F0120
:108A3B000E8825846F000E8921856F000E8A218692
:108A4B006F000E8B21876F87518611851160E15B5B
:108A5B00D0D8908835D96E8935DA6E3A0ED9260181
:108A6B000EDA22D8908435E16E8535E26E3A0EE14E
:108A7B0026010EE222DE50E65CE650800A0C6FDE29
:108A8B0050800A0C59D8B035D0D8908835D96E891A
:108A9B0035DA6E3A0ED926010EDA22DECF74F1DD0D
:108AAB00CF75F1000E75BFFF0E766F776FD8908480
:108ABB0035D96E8535DA6E3A0ED926010EDA22D803
:108ACB00908835E16E8935E26E3A0EE126010EE2B1
:108ADB0022DECFE6FFDDCFE5FFD8908435D96E855A
:108AEB0035DA6E3A0ED926010EDA2274C1DEFF7525
:108AFB00C1DDFF010E8427000E8523862387238784
:108B0B00518611851104E1070E845DD8A0A1D70110
:108B1B000E8827000E89238A238B238B518A118978
:108B2B001104E1060E885DD8A082D7000E886F0075
:108B3B000E896F000E8A6F000E8B6F010E882584D5
:108B4B006F000E8921856F000E8A21866F000E8BB8
:108B5B0021876F87518611851160E15BD0D8908892
:108B6B0035D96E8935DA6E480ED926010EDA22D840
:108B7B00908435E16E8535E26E480EE126010EE2FA
:108B8B0022DE50E65CE650800A0C6FDE50800A0C49
:108B9B0059D8B035D0D8908835D96E8935DA6E482A
:108BAB000ED926010EDA22DECF74F1DDCF75F1007E
:108BBB000E75BFFF0E766F776FD8908435D96E85A3
:108BCB0035DA6E480ED926010EDA22D8908835E1B7
:108BDB006E8935E26E480EE126010EE222DECFE60B
:108BEB00FFDDCFE5FFD8908435D96E8535DA6E4839
:108BFB000ED926010EDA2274C1DEFF75C1DDFF012D
:108C0B000E8427000E8523862387238751861185A3
:108C1B001104E1070E845DD8A0A1D7010E882700AF
:108C2B000E89238A238B238B518A11891104E10628
:108C3B000E885DD8A082D7000E886F000E896F005A
:108C4B000E8A6F000E8B6F010E8825846F000E89C4
:108C5B0021856F000E8A21866F000E8B21876F870F
:108C6B00518611851160E15BD0D8908835D96E891A
:108C7B0035DA6E560ED926010EDA22D8908435E1FC
:108C8B006E8535E26E560EE126010EE222DE50E6CF
:108C9B005CE650800A0C6FDE50800A0C59D8B03558
:108CAB00D0D8908835D96E8935DA6E560ED9260113
:108CBB000EDA22DECF74F1DDCF75F1000E75BFFF3A
:108CCB000E766F776FD8908435D96E8535DA6E5600
:108CDB000ED926010EDA22D8908835E16E8935E25D
:108CEB006E560EE126010EE222DECFE6FFDDCFE56A
:108CFB00FFD8908435D96E8535DA6E560ED926019C
:108D0B000EDA2274C1DEFF75C1DDFF010E84270070
:108D1B000E85238623872387518611851104E1074E
:108D2B000E845DD8A0A1D7010E8827000E89238A57
:108D3B00238B238B518A11891104E1060E885DD890
:108D4B00A082D740513E25086F41513F21096F4208
:108D5B00510825016E43510921026E000E046E036A
:108D6B000E036E58EC14F001C034F102C035F10162
:108D7B00014E514C25086F4F514D21096F50510831
:108D8B0025016E51510921026E000E046E030E0374
:108D9B006E58EC14F001C036F102C037F101015CE2
:108DAB00515A25086F5D515B21096F5E51082501F2
:108DBB006E5F510921026E000E046E030E036E5896
:108DCB00EC14F001C038F102C039F101010051344B
:108DDB005D086F01513559096F08C101F009C102D6
:108DEB00F0000E02BEFF0E036E046E010E8BEC1C28
:108DFB00F001C034F002C035F003C036F004C037C8
:108E0B00F004C138F005C139F006C13AF007C13B97
:108E1B00F0A6EC28F034C070F135C071F136C07299
:108E2B00F137C073F101010251365D086F03513701
:108E3B0059096F08C101F009C102F0000E02BEFF13
:108E4B000E036E046E010E8BEC1CF001C034F002AD
:108E5B00C035F003C036F004C037F004C138F0055C
:108E6B00C139F006C13AF007C13BF0A6EC28F0344B
:108E7B00C078F135C079F136C07AF137C07BF13863
:108E8B00C101F039C102F0000E02BEFF0E036E04E9
:108E9B006E010E8BEC1CF001C02AF102C02BF1030A
:108EAB00C02CF104C02DF1330E0101646F330E653C
:108EBB006F650E666F420E676F000E0001686F00E4
:108ECB000E696F000E6A6F000E6B6F78C16CF079D4
:108EDB00C16DF07AC16EF07BC16FF0E0EC18F00061
:108EEB0001D8B052D078C11FF079C120F07AC121DE
:108EFB00F07BC122F070C11BF071C11CF072C11D5F
:108F0B00F073C11EF005EC26F01BC068F11CC069A4
:108F1B00F11DC06AF11EC06BF168C168F069C169CF
:108F2B00F06AC16AF06BC16BF0EDEC32F068C06CAB
:108F3B00F169C06DF16AC06EF16BC06FF1000E008C
:108F4B0001606F000E616FB40E626F420E636F644F
:108F5B00C148F065C149F066C14AF067C14BF06C7E
:108F6B00C144F06DC145F06EC146F06FC147F02CA6
:108F7B00EC2AF044C064F045C065F046C066F0478B
:108F8B00C067F06FEC12F054D001017BAF5AD07870
:108F9B00C11FF079C120F07AC121F07BC122F070A2
:108FAB00C11BF071C11CF072C11DF073C11EF00525
:108FBB00EC26F01BC068F11CC069F11DC06AF11EE4
:108FCB00C06BF168C168F069C169F06AC16AF06B86
:108FDB00C16BF0EDEC32F068C06CF169C06DF16AF9
:108FEB00C06EF16BC06FF1000E0001606F000E617F
:108FFB006F870E626F430E636F64C148F065C149A2
:10900B00F066C14AF067C14BF06CC144F06DC145CD
:10901B00F06EC146F06FC147F02CEC2AF044C064EF
:10902B00F045C065F046C066F047C067F06FEC12C4
:10903B00F060C080F161C081F162C082F163C083D6
:10904B00F128D078C101F079C102F07AC103F07B2D
:10905B00C104F0000E056E000E066E000E076E00CA
:10906B000E086E22EC15F0D8A00BD0010173AF08DF
:10907B00D0000E806F000E816F340E826F430E088E
:10908B00D0000E0101806F000E816F000E826F0009
:10909B000E836F0D0E0001EC6F010EED6FD20EEE15
:1090AB006FFF0EEF6F80C1F0F081C1F1F082C1F262
:1090BB00F083C1F3F004EC13F0000E476E0F0E4675
:1090CB006E000E496E230E486E0D0E4A6E010E4B4E
:1090DB006EB2EC22F0000E476E4B0E466E000E4940
:1090EB006E230E486ECA0E4A6EFF0E4B6EB2EC220A
:1090FB00F0DEEC10F010C364F011C365F012C36620
:10910B00F013C367F080C160F081C161F082C1626E
:10911B00F083C163F06FEC12F060C068F061C0695E
:10912B00F062C06AF063C06BF0000E00016C6F0060
:10913B000E6D6F700E6E6F400E6F6FE0EC18F000DF
:10914B0001D8A0E0D0000E686F000E696F340E6A74
:10915B006F430E6B6F10C364F011C365F012C366DF
:10916B00F013C367F080C160F081C161F082C1620E
:10917B00F083C163F06FEC12F060C06CF061C06DF6
:10918B00F062C06EF063C06FF0E0EC18F00001D835
:10919B00B025D090D010C334F011C335F012C336C4
:1091AB00F013C337F0000E386E000E396EF00E3A26
:1091BB006E400E3B6EA6EC28F034C010F335C01198
:1091CB00F336C012F337C013F310C374F011C37529
:1091DB00F012C376F013C377F090EC4AF010C3642F
:1091EB00F011C365F012C366F013C367F080C16062
:1091FB00F081C161F082C162F083C163F06FEC1248
:10920B00F060C068F061C069F062C06AF063C06B67
:10921B00F0000E00016C6F000E6D6F700E6E6F40E4
:10922B000E6F6FE0EC18F00001D8A06CD0B3D71024
:10923B00C360F011C361F012C362F013C363F0009B
:10924B000E646F000E656FF00E666F400E676F6FEA
:10925B00EC12F060C010F361C011F362C012F36343
:10926B00C013F3000E0001686F000E696F000E6AE9
:10927B006F000E6B6F10C36CF011C36DF012C36EE9
:10928B00F013C36FF0E0EC18F00001D8A009D00088
:10929B000E0301106F000E116FB40E126F430E13FD
:1092AB006F10C374F011C375F012C376F013C3774C
:1092BB00F090EC4AF010C364F011C365F012C36672
:1092CB00F013C367F080C160F081C161F082C162AD
:1092DB00F083C163F06FEC12F060C068F061C0699D
:1092EB00F062C06AF063C06BF0000E00016C6F009F
:1092FB000E6D6F700E6E6F400E6F6FE0EC18F0001E
:10930B0001D8B095D7000E686F000E696F700E6AAA
:10931B006F400E6B6F80C164F081C165F082C166D6
:10932B00F083C167F010C360F011C361F012C36228
:10933B00F013C363F06FEC12F060C06CF061C06DA2
:10934B00F062C06EF063C06FF0E0EC18F00001D873
:10935B00B01200000E686F000E696F340E6A6F4317
:10936B000E6B6F80C164F081C165F082C166F083C2
:10937B00C167F010C360F011C361F012C362F01348
:10938B00C363F06FEC12F060C06CF061C06DF06203
:10939B00C06EF063C06FF0E0EC18F00001D8B025A0
:1093AB00D090D010C360F011C361F012C362F01300
:1093BB00C363F0000E646F000E656FF00E666F40B6
:1093CB000E676F6FEC12F060C010F361C011F362A7
:1093DB00C012F363C013F310C374F011C375F01212
:1093EB00C376F013C377F090EC4AF080C164F08140
:1093FB00C165F082C166F083C167F010C360F011E4
:10940B00C361F012C362F013C363F06FEC12F06030
:10941B00C068F061C069F062C06AF063C06BF000B5
:10942B000E00016C6F000E6D6F700E6E6F400E6F45
:10943B006FE0EC18F00001D8A01200B3D710C334C2
:10944B00F011C335F012C336F013C337F0000E38EA
:10945B006E000E396EF00E3A6E400E3B6EA6EC2887
:10946B00F034C010F335C011F336C012F337C0130C
:10947B00F310C368F011C369F012C36AF013C36B26
:10948B00F0000E00016C6F000E6D6FB40E6E6F432B
:10949B000E6F6FE0EC18F00001D8A009D0000E039E
:1094AB0001106F000E116F000E126F000E136F1074
:1094BB00C374F011C375F012C376F013C377F09039
:1094CB00EC4AF080C164F081C165F082C166F08323
:1094DB00C167F010C360F011C361F012C362F013E7
:1094EB00C363F06FEC12F060C068F061C069F062AA
:1094FB00C06AF063C06BF0000E00016C6F000E6D64
:10950B006F700E6E6F400E6F6FE0EC18F00001D8AD
:10951B00A0120094D774C068F075C069F076C06A69
:10952B00F077C06BF0000E00016C6F200E6D6FB208
:10953B000E6E6F430E6F6FE0EC18F00001D8B01594
:10954B00D074C068F075C069F076C06AF077C06BF4
:10955B00F0000E6C6F000E6D6F610E6E6F420E6F32
:10956B006FE0EC18F00001D8B0C2D174C068F07590
:10957B00C069F076C06AF077C06BF0000E6C6F209C
:10958B000E6D6FB20E6E6F430E6F6FE0EC18F00046
:10959B0001D8B015D074C068F075C069F076C06A98
:1095AB00F077C06BF0000E6C6F000E6D6F700E6E6F
:1095BB006F400E6F6FE0EC18F00001D8B00ED000CA
:1095CB000E0B6E400E0A6E000E0D6E120E0C6E80A0
:1095DB000E0E6ED5EC2BF000EF56F074C068F075E4
:1095EB00C069F076C06AF077C06BF0000E6C6F004C
:1095FB000E6D6F700E6E6F400E6F6FE0EC18F0001B
:10960B0001D8A023D074C068F075C069F076C06A29
:10961B00F077C06BF0000E6C6F000E6D6F340E6E3A
:10962B006F410E6F6FE0EC18F00001D8B00ED00058
:10963B000E0B6E400E0A6E000E0D6E120E0C6E406F
:10964B000E0E6ED5EC2BF000EF56F074C068F07573
:10965B00C069F076C06AF077C06BF0000E6C6F00DB
:10966B000E6D6F340E6E6F410E6F6FE0EC18F000E5
:10967B0001D8A023D074C068F075C069F076C06AB9
:10968B00F077C06BF0000E6C6F000E6D6F960E6E68
:10969B006F410E6F6FE0EC18F00001D8B00ED000E8
:1096AB000E0B6E400E0A6E000E0D6E120E0C6E201F
:1096BB000E0E6ED5EC2BF000EF56F074C068F07503
:1096CB00C069F076C06AF077C06BF0000E6C6F006B
:1096DB000E6D6F960E6E6F410E6F6FE0EC18F00013
:1096EB0001D8A023D074C068F075C069F076C06A49
:1096FB00F077C06BF0000E6C6F000E6D6FD20E6EBC
:10970B006F410E6F6FE0EC18F00001D8B00ED00077
:10971B000E0B6E400E0A6E000E0D6E120E0C6E10BE
:10972B000E0E6ED5EC2BF000EF56F074C068F07592
:10973B00C069F076C06AF077C06BF0000E6C6F00FA
:10974B000E6D6FD20E6E6F410E6F6FE0EC18F00066
:10975B0001D8A023D074C068F075C069F076C06AD8
:10976B00F077C06BF0000E6C6F000E6D6F070E6E16
:10977B006F420E6F6FE0EC18F00001D8B00ED00006
:10978B000E0B6E400E0A6E000E0D6E120E0C6E0856
:10979B000E0E6ED5EC2BF000EF56F074C068F07522
:1097AB00C069F076C06AF077C06BF0000E6C6F008A
:1097BB000E6D6F070E6E6F420E6F6FE0EC18F000C0
:1097CB0001D8A023D074C068F075C069F076C06A68
:1097DB00F077C06BF0000E6C6F000E6D6F250E6E88
:1097EB006F420E6F6FE0EC18F00001D8B00ED00096
:1097FB000E0B6E400E0A6E000E0D6E120E0C6E04EA
:10980B000E0E6ED5EC2BF000EF56F074C068F075B1
:10981B00C069F076C06AF077C06BF0000E6C6F0019
:10982B000E6D6F250E6E6F420E6F6FE0EC18F00031
:10983B0001D8A023D074C068F075C069F076C06AF7
:10984B00F077C06BF0000E6C6F000E6D6F430E6EF9
:10985B006F420E6F6FE0EC18F00001D8B00ED00025
:10986B000E0B6E400E0A6E000E0D6E120E0C6E027B
:10987B000E0E6ED5EC2BF000EF56F074C068F07541
:10988B00C069F076C06AF077C06BF0000E6C6F00A9
:10989B000E6D6F430E6E6F420E6F6FE0EC18F000A3
:1098AB0001D8A000EF56F074C068F075C069F0766F
:1098BB00C06AF077C06BF0000E6C6F000E6D6F61BD
:1098CB000E6E6F420E6F6FE0EC18F00001D8B00017
:1098DB00EF56F0000E0B6E400E0A6E000E0D6E1260
:1098EB000E0C6E010E0E6ED5EC2BF000EF56F074D5
:1098FB00C068F075C069F076C06AF077C06BF00095
:10990B000E6C6F000E6D6F610E6E6F420E6F6FE01F
:10991B00EC18F00001D8A0D7D174C068F075C069FD
:10992B00F076C06AF077C06BF0000E6C6F800E6D36
:10993B006FE80E6E6F420E6F6FE0EC18F00001D8FF
:10994B00B0C2D174C068F075C069F076C06AF077A8
:10995B00C06BF0000E6C6F000E6D6F610E6E6F4280
:10996B000E6F6FE0EC18F00001D8A023D074C06824
:10997B00F075C069F076C06AF077C06BF0000E6CC2
:10998B006F000E6D6F7F0E6E6F420E6F6FE0EC18F7
:10999B00F00001D8B00ED0000E0B6E420E0A6E0016
:1099AB000E0D6E130E0C6E800E0E6ED5EC2BF000A2
:1099BB00EF56F074C068F075C069F076C06AF07746
:1099CB00C06BF0000E6C6F000E6D6F7F0E6E6F42F2
:1099DB000E6F6FE0EC18F00001D8A023D074C068B4
:1099EB00F075C069F076C06AF077C06BF0000E6C52
:1099FB006F800E6D6F8E0E6E6F420E6F6FE0EC18F8
:109A0B00F00001D8B00ED0000E0B6E420E0A6E00A5
:109A1B000E0D6E130E0C6E400E0E6ED5EC2BF00071
:109A2B00EF56F074C068F075C069F076C06AF077D5
:109A3B00C06BF0000E6C6F800E6D6F8E0E6E6F42F2
:109A4B000E6F6FE0EC18F00001D8A023D074C06843
:109A5B00F075C069F076C06AF077C06BF0000E6CE1
:109A6B006F800E6D6F9D0E6E6F420E6F6FE0EC1878
:109A7B00F00001D8B00ED0000E0B6E420E0A6E0035
:109A8B000E0D6E130E0C6E200E0E6ED5EC2BF00021
:109A9B00EF56F074C068F075C069F076C06AF07765
:109AAB00C06BF0000E6C6F800E6D6F9D0E6E6F4273
:109ABB000E6F6FE0EC18F00001D8A023D074C068D3
:109ACB00F075C069F076C06AF077C06BF0000E6C71
:109ADB006F800E6D6FAC0E6E6F420E6F6FE0EC18F9
:109AEB00F00001D8B00ED0000E0B6E420E0A6E00C5
:109AFB000E0D6E130E0C6E100E0E6ED5EC2BF000C1
:109B0B00EF56F074C068F075C069F076C06AF077F4
:109B1B00C06BF0000E6C6F800E6D6FAC0E6E6F42F3
:109B2B000E6F6FE0EC18F00001D8A023D074C06862
:109B3B00F075C069F076C06AF077C06BF0000E6C00
:109B4B006F800E6D6FBB0E6E6F420E6F6FE0EC1879
:109B5B00F00001D8B00ED0000E0B6E420E0A6E0054
:109B6B000E0D6E130E0C6E080E0E6ED5EC2BF00058
:109B7B00EF56F074C068F075C069F076C06AF07784
:109B8B00C06BF0000E6C6F800E6D6FBB0E6E6F4274
:109B9B000E6F6FE0EC18F00001D8A023D074C068F2
:109BAB00F075C069F076C06AF077C06BF0000E6C90
:109BBB006F800E6D6FCA0E6E6F420E6F6FE0EC18FA
:109BCB00F00001D8B00ED0000E0B6E420E0A6E00E4
:109BDB000E0D6E130E0C6E040E0E6ED5EC2BF000EC
:109BEB00EF56F074C068F075C069F076C06AF07714
:109BFB00C06BF0000E6C6F800E6D6FCA0E6E6F42F5
:109C0B000E6F6FE0EC18F00001D8A023D074C06881
:109C1B00F075C069F076C06AF077C06BF0000E6C1F
:109C2B006F800E6D6FD90E6E6F420E6F6FE0EC187A
:109C3B00F00001D8B00ED0000E0B6E420E0A6E0073
:109C4B000E0D6E130E0C6E020E0E6ED5EC2BF0007D
:109C5B00EF56F074C068F075C069F076C06AF077A3
:109C6B00C06BF0000E6C6F800E6D6FD90E6E6F4275
:109C7B000E6F6FE0EC18F00001D8A000EF56F074F7
:109C8B00C068F075C069F076C06AF077C06BF00001
:109C9B000E6C6F800E6D6FE80E6E6F420E6F6FE085
:109CAB00EC18F00001D8B000EF56F0000E0B6E422E
:109CBB000E0A6E000E0D6E130E0C6E010E0E6ED58F
:109CCB00EC2BF000EF56F074C068F075C069F076BD
:109CDB00C06AF077C06BF0000E6C6F800E6D6FE892
:109CEB000E6E6F420E6F6FE0EC18F00001D8A0D72C
:109CFB00D174C068F075C069F076C06AF077C06B3C
:109D0B00F0000E6C6F400E6D6F300E6E6F430E6F6A
:109D1B006FE0EC18F00001D8B0C2D174C068F075D8
:109D2B00C069F076C06AF077C06BF0000E6C6F8084
:109D3B000E6D6FE80E6E6F420E6F6FE0EC18F00059
:109D4B0001D8A023D074C068F075C069F076C06AE2
:109D5B00F077C06BF0000E6C6F800E6D6FF70E6EB0
:109D6B006F420E6F6FE0EC18F00001D8B00ED00010
:109D7B000E0B6E420E0A6E000E0D6E120E0C6E80E6
:109D8B000E0E6ED5EC2BF000EF56F074C068F0752C
:109D9B00C069F076C06AF077C06BF0000E6C6F8014
:109DAB000E6D6FF70E6E6F420E6F6FE0EC18F000DA
:109DBB0001D8A023D074C068F075C069F076C06A72
:109DCB00F077C06BF0000E6C6F400E6D6F030E6E74
:109DDB006F430E6F6FE0EC18F00001D8B00ED0009F
:109DEB000E0B6E420E0A6E000E0D6E120E0C6E40B6
:109DFB000E0E6ED5EC2BF000EF56F074C068F075BC
:109E0B00C069F076C06AF077C06BF0000E6C6F40E3
:109E1B000E6D6F030E6E6F430E6F6FE0EC18F0005C
:109E2B0001D8A023D074C068F075C069F076C06A01
:109E3B00F077C06BF0000E6C6FC00E6D6F0A0E6E7C
:109E4B006F430E6F6FE0EC18F00001D8B00ED0002E
:109E5B000E0B6E420E0A6E000E0D6E120E0C6E2065
:109E6B000E0E6ED5EC2BF000EF56F074C068F0754B
:109E7B00C069F076C06AF077C06BF0000E6C6FC0F3
:109E8B000E6D6F0A0E6E6F430E6F6FE0EC18F000E5
:109E9B0001D8A023D074C068F075C069F076C06A91
:109EAB00F077C06BF0000E6C6F400E6D6F120E6E84
:109EBB006F430E6F6FE0EC18F00001D8B00ED000BE
:109ECB000E0B6E420E0A6E000E0D6E120E0C6E1005
:109EDB000E0E6ED5EC2BF000EF56F074C068F075DB
:109EEB00C069F076C06AF077C06BF0000E6C6F4003
:109EFB000E6D6F120E6E6F430E6F6FE0EC18F0006D
:109F0B0001D8A023D074C068F075C069F076C06A20
:109F1B00F077C06BF0000E6C6FC00E6D6F190E6E8C
:109F2B006F430E6F6FE0EC18F00001D8B00ED0004D
:109F3B000E0B6E420E0A6E000E0D6E120E0C6E089C
:109F4B000E0E6ED5EC2BF000EF56F074C068F0756A
:109F5B00C069F076C06AF077C06BF0000E6C6FC012
:109F6B000E6D6F190E6E6F430E6F6FE0EC18F000F5
:109F7B0001D8A023D074C068F075C069F076C06AB0
:109F8B00F077C06BF0000E6C6F400E6D6F210E6E94
:109F9B006F430E6F6FE0EC18F00001D8B00ED000DD
:109FAB000E0B6E420E0A6E000E0D6E120E0C6E0430
:109FBB000E0E6ED5EC2BF000EF56F074C068F075FA
:109FCB00C069F076C06AF077C06BF0000E6C6F4022
:109FDB000E6D6F210E6E6F430E6F6FE0EC18F0007D
:109FEB0001D8A023D074C068F075C069F076C06A40
:109FFB00F077C06BF0000E6C6FC00E6D6F280E6E9D
:10A00B006F430E6F6FE0EC18F00001D8B00ED0006C
:10A01B000E0B6E420E0A6E000E0D6E120E0C6E02C1
:10A02B000E0E6ED5EC2BF000EF56F074C068F07589
:10A03B00C069F076C06AF077C06BF0000E6C6FC031
:10A04B000E6D6F280E6E6F430E6F6FE0EC18F00005
:10A05B0001D8A000EF56F074C068F075C069F076B7
:10A06B00C06AF077C06BF0000E6C6F400E6D6F30F6
:10A07B000E6E6F430E6F6FE0EC18F00001D8B0005E
:10A08B00EF56F0000E0B6E420E0A6E000E0D6E12A6
:10A09B000E0C6E010E0E6ED5EC2BF000EF56F0741D
:10A0AB00C068F075C069F076C06AF077C06BF000DD
:10A0BB000E6C6F400E6D6F300E6E6F430E6F6FE058
:10A0CB00EC18F00001D8A0D3D174C068F075C0694A
:10A0DB00F076C06AF077C06BF0000E6C6F400E6DBF
:10A0EB006F6C0E6E6F430E6F6FE0EC18F00001D8C3
:10A0FB00B0BED174C068F075C069F076C06AF077F5
:10A10B00C06BF0000E6C6F400E6D6F300E6E6F43B8
:10A11B000E6F6FE0EC18F00001D8A023D074C0686C
:10A12B00F075C069F076C06AF077C06BF0000E6C0A
:10A13B006FC00E6D6F370E6E6F430E6F6FE0EC18C6
:10A14B00F00001D8B00ED0000E0B6E440E0A6E005C
:10A15B000E0D6E130E0C6E800E0E6ED5EC2BF000EA
:10A16B00EF56F074C068F075C069F076C06AF0778E
:10A17B00C06BF0000E6C6FC00E6D6F370E6E6F43C1
:10A18B000E6F6FE0EC18F00001D8A023D074C068FC
:10A19B00F075C069F076C06AF077C06BF0000E6C9A
:10A1AB006F400E6D6F3F0E6E6F430E6F6FE0EC18CE
:10A1BB00F00001D8B00ED0000E0B6E440E0A6E00EC
:10A1CB000E0D6E130E0C6E400E0E6ED5EC2BF000BA
:10A1DB00EF56F074C068F075C069F076C06AF0771E
:10A1EB00C06BF0000E6C6F400E6D6F3F0E6E6F43C9
:10A1FB000E6F6FE0EC18F00001D8A023D074C0688C
:10A20B00F075C069F076C06AF077C06BF0000E6C29
:10A21B006FC00E6D6F460E6E6F430E6F6FE0EC18D6
:10A22B00F00001D8B00ED0000E0B6E440E0A6E007B
:10A23B000E0D6E130E0C6E200E0E6ED5EC2BF00069
:10A24B00EF56F074C068F075C069F076C06AF077AD
:10A25B00C06BF0000E6C6FC00E6D6F460E6E6F43D1
:10A26B000E6F6FE0EC18F00001D8A023D074C0681B
:10A27B00F075C069F076C06AF077C06BF0000E6CB9
:10A28B006F400E6D6F4E0E6E6F430E6F6FE0EC18DE
:10A29B00F00001D8B00ED0000E0B6E440E0A6E000B
:10A2AB000E0D6E130E0C6E100E0E6ED5EC2BF00009
:10A2BB00EF56F074C068F075C069F076C06AF0773D
:10A2CB00C06BF0000E6C6F400E6D6F4E0E6E6F43D9
:10A2DB000E6F6FE0EC18F00001D8A023D074C068AB
:10A2EB00F075C069F076C06AF077C06BF0000E6C49
:10A2FB006FC00E6D6F550E6E6F430E6F6FE0EC18E7
:10A30B00F00001D8B00ED0000E0B6E440E0A6E009A
:10A31B000E0D6E130E0C6E080E0E6ED5EC2BF000A0
:10A32B00EF56F074C068F075C069F076C06AF077CC
:10A33B00C06BF0000E6C6FC00E6D6F550E6E6F43E1
:10A34B000E6F6FE0EC18F00001D8A023D074C0683A
:10A35B00F075C069F076C06AF077C06BF0000E6CD8
:10A36B006F400E6D6F5D0E6E6F430E6F6FE0EC18EE
:10A37B00F00001D8B00ED0000E0B6E440E0A6E002A
:10A38B000E0D6E130E0C6E040E0E6ED5EC2BF00034
:10A39B00EF56F074C068F075C069F076C06AF0775C
:10A3AB00C06BF0000E6C6F400E6D6F5D0E6E6F43E9
:10A3BB000E6F6FE0EC18F00001D8A022D074C068CB
:10A3CB00F075C069F076C06AF077C06BF0000E6C68
:10A3DB006FC00E6D6F640E6E6F430E6F6FE0EC18F7
:10A3EB00F00001D8B00DD0000E0B6E440E0A6E00BB
:10A3FB000E0D6E130E0C6E020E0E6ED5EC2BF0FACC
:10A40B00D374C068F075C069F076C06AF077C06B22
:10A41B00F0000E6C6FC00E6D6F640E6E6F430E6F9F
:10A42B006FE0EC18F00001D8A0E5D374C068F075AC
:10A43B00C069F076C06AF077C06BF0000E6C6F40AD
:10A44B000E6D6F6C0E6E6F430E6F6FE0EC18F000BD
:10A45B0001D8B0D0D3000E0B6E440E0A6E000E0D59
:10A46B006E130E0C6E010E0E6ED5EC2BF0C3D37467
:10A47B00C068F075C069F076C06AF077C06BF00009
:10A48B000E6C6F400E6D6F6C0E6E6F430E6F6FE048
:10A49B00EC18F00001D8A0CDD174C068F075C0697C
:10A4AB00F076C06AF077C06BF0000E6C6F200E6D0B
:10A4BB006F940E6E6F430E6F6FE0EC18F00001D8C7
:10A4CB00B0B8D174C068F075C069F076C06AF07727
:10A4DB00C06BF0000E6C6F400E6D6F6C0E6E6F43A9
:10A4EB000E6F6FE0EC18F00001D8A022D074C0689A
:10A4FB00F075C069F076C06AF077C06BF0000E6C37
:10A50B006FC00E6D6F730E6E6F430E6F6FE0EC18B6
:10A51B00F00001D8B00DD0000E0B6E440E0A6E0089
:10A52B000E0D6E120E0C6E800E0E6ED5EC2BF062B5
:10A53B00D374C068F075C069F076C06AF077C06BF1
:10A54B00F0000E6C6FC00E6D6F730E6E6F430E6F5F
:10A55B006FE0EC18F00001D8A022D074C068F07541
:10A56B00C069F076C06AF077C06BF0000E6C6F407C
:10A57B000E6D6F7B0E6E6F430E6F6FE0EC18F0007D
:10A58B0001D8B00DD0000E0B6E440E0A6E000E0DEE
:10A59B006E120E0C6E400E0E6ED5EC2BF02BD37490
:10A5AB00C068F075C069F076C06AF077C06BF000D8
:10A5BB000E6C6F400E6D6F7B0E6E6F430E6F6FE008
:10A5CB00EC18F00001D8A022D074C068F075C069F7
:10A5DB00F076C06AF077C06BF0000E6C6F600E6D9A
:10A5EB006F810E6E6F430E6F6FE0EC18F00001D8A9
:10A5FB00B00DD0000E0B6E440E0A6E000E0D6E12D7
:10A60B000E0C6E200E0E6ED5EC2BF0F4D274C068CF
:10A61B00F075C069F076C06AF077C06BF0000E6C15
:10A62B006F600E6D6F810E6E6F430E6F6FE0EC18E7
:10A63B00F00001D8A022D074C068F075C069F07624
:10A64B00C06AF077C06BF0000E6C6F200E6D6F85DB
:10A65B000E6E6F430E6F6FE0EC18F00001D8B00D6B
:10A66B00D0000E0B6E440E0A6E000E0D6E120E0C09
:10A67B006E100E0E6ED5EC2BF0BDD274C068F0755B
:10A68B00C069F076C06AF077C06BF0000E6C6F207B
:10A69B000E6D6F850E6E6F430E6F6FE0EC18F00052
:10A6AB0001D8A022D074C068F075C069F076C06A7A
:10A6BB00F077C06BF0000E6C6FE00E6D6F880E6E56
:10A6CB006F430E6F6FE0EC18F00001D8B00DD000A7
:10A6DB000E0B6E440E0A6E000E0D6E120E0C6E08F3
:10A6EB000E0E6ED5EC2BF086D274C068F075C06977
:10A6FB00F076C06AF077C06BF0000E6C6FE00E6DF9
:10A70B006F880E6E6F430E6F6FE0EC18F00001D880
:10A71B00A022D074C068F075C069F076C06AF0777B
:10A72B00C06BF0000E6C6FA00E6D6F8C0E6E6F43D6
:10A73B000E6F6FE0EC18F00001D8B00DD0000E0BCF
:10A74B006E440E0A6E000E0D6E120E0C6E040E0E83
:10A75B006ED5EC2BF04FD274C068F075C069F076F3
:10A76B00C06AF077C06BF0000E6C6FA00E6D6F8C33
:10A77B000E6E6F430E6F6FE0EC18F00001D8A02245
:10A78B00D074C068F075C069F076C06AF077C06BA2
:10A79B00F0000E6C6F600E6D6F900E6E6F430E6F50
:10A7AB006FE0EC18F00001D8B00DD0000E0B6E442A
:10A7BB000E0A6E000E0D6E120E0C6E020E0E6ED584
:10A7CB00EC2BF018D274C068F075C069F076C06AD3
:10A7DB00F077C06BF0000E6C6F600E6D6F900E6EAD
:10A7EB006F430E6F6FE0EC18F00001D8A003D2742A
:10A7FB00C068F075C069F076C06AF077C06BF00086
:10A80B000E6C6F200E6D6F940E6E6F430E6F6FE0BC
:10A81B00EC18F00001D8B0EED1000E0B6E440E0A0E
:10A82B006E000E0D6E120E0C6E010E0E6ED5EC2B15
:10A83B00F0E1D174C068F075C069F076C06AF0774A
:10A84B00C06BF0000E6C6F200E6D6F940E6E6F432D
:10A85B000E6F6FE0EC18F00001D8A0CCD174C0687B
:10A86B00F075C069F076C06AF077C06BF0000E6CC3
:10A87B006F200E6D6FB20E6E6F430E6F6FE0EC18A4
:10A88B00F00001D8B0B7D174C068F075C069F0762C
:10A89B00C06AF077C06BF0000E6C6F200E6D6F947A
:10A8AB000E6E6F430E6F6FE0EC18F00001D8A02214
:10A8BB00D074C068F075C069F076C06AF077C06B71
:10A8CB00F0000E6C6FE00E6D6F970E6E6F430E6F98
:10A8DB006FE0EC18F00001D8B00DD0000E0B6E40FD
:10A8EB000E0A6E000E0D6E130E0C6E800E0E6ED5D4
:10A8FB00EC2BF080D174C068F075C069F076C06A3B
:10A90B00F077C06BF0000E6C6FE00E6D6F970E6EF4
:10A91B006F430E6F6FE0EC18F00001D8A022D074DB
:10A92B00C068F075C069F076C06AF077C06BF00054
:10A93B000E6C6FA00E6D6F9B0E6E6F430E6F6FE004
:10A94B00EC18F00001D8B00DD0000E0B6E400E0AC3
:10A95B006E000E0D6E130E0C6E400E0E6ED5EC2BA4
:10A96B00F049D174C068F075C069F076C06AF077B1
:10A97B00C06BF0000E6C6FA00E6D6F9B0E6E6F4375
:10A98B000E6F6FE0EC18F00001D8A022D074C068F5
:10A99B00F075C069F076C06AF077C06BF0000E6C92
:10A9AB006F600E6D6F9F0E6E6F430E6F6FE0EC1846
:10A9BB00F00001D8B00DD0000E0B6E400E0A6E00E9
:10A9CB000E0D6E130E0C6E200E0E6ED5EC2BF012C0
:10A9DB00D174C068F075C069F076C06AF077C06B4F
:10A9EB00F0000E6C6F600E6D6F9F0E6E6F430E6FEF
:10A9FB006FE0EC18F00001D8A022D074C068F0759D
:10AA0B00C069F076C06AF077C06BF0000E6C6F20F7
:10AA1B000E6D6FA30E6E6F430E6F6FE0EC18F000B0
:10AA2B0001D8B00DD0000E0B6E400E0A6E000E0D4D
:10AA3B006E130E0C6E100E0E6ED5EC2BF0DBD0746D
:10AA4B00C068F075C069F076C06AF077C06BF00033
:10AA5B000E6C6F200E6D6FA30E6E6F430E6F6FE05B
:10AA6B00EC18F00001D8A022D074C068F075C06952
:10AA7B00F076C06AF077C06BF0000E6C6FE00E6D75
:10AA8B006FA60E6E6F430E6F6FE0EC18F00001D8DF
:10AA9B00B00DD0000E0B6E400E0A6E000E0D6E1335
:10AAAB000E0C6E080E0E6ED5EC2BF0A4D074C06895
:10AABB00F075C069F076C06AF077C06BF0000E6C71
:10AACB006FE00E6D6FA60E6E6F430E6F6FE0EC189E
:10AADB00F00001D8A022D074C068F075C069F07680
:10AAEB00C06AF077C06BF0000E6C6FA00E6D6FAA92
:10AAFB000E6E6F430E6F6FE0EC18F00001D8B00DC7
:10AB0B00D0000E0B6E400E0A6E000E0D6E130E0C67
:10AB1B006E040E0E6ED5EC2BF06DD074C068F07514
:10AB2B00C069F076C06AF077C06BF0000E6C6FA056
:10AB3B000E6D6FAA0E6E6F430E6F6FE0EC18F00088
:10AB4B0001D8A022D074C068F075C069F076C06AD5
:10AB5B00F077C06BF0000E6C6F600E6D6FAE0E6E0B
:10AB6B006F430E6F6FE0EC18F00001D8B00DD00002
:10AB7B000E0B6E400E0A6E000E0D6E130E0C6E0257
:10AB8B000E0E6ED5EC2BF036D074C068F075C06924
:10AB9B00F076C06AF077C06BF0000E6C6F600E6DD4
:10ABAB006FAE0E6E6F430E6F6FE0EC18F00001D8B6
:10ABBB00A021D074C068F075C069F076C06AF077D8
:10ABCB00C06BF0000E6C6F200E6D6FB20E6E6F438C
:10ABDB000E6F6FE0EC18F00001D8B00CD0000E0B2C
:10ABEB006E400E0A6E000E0D6E130E0C6E010E0EE5
:10ABFB006ED5EC2BF0000E026E0A0E016EA5EC1159
:10AC0B00F012009B8C700ED312000E0F01386F00E8
:10AC1B000E396F000E3A6F010E936E180E946EF193
:10AC2B009E938C400E616EF19EC650F00B0809C6C8
:10AC3B006EC68A270EC86EC59A000E026E640E0190
:10AC4B006EA5EC11F0B4EC15F06E0E016E030E0256
:10AC5B006EF20E036E2D0E046E000E066E800E0548
:10AC6B006E000E086E400E076E49EC27F06E0E015B
:10AC7B006E030E026ED9EC10F0000E1D6E000E1C52
:10AC8B006E57EC13F0880E016EFF0E026E1FEC1167
:10AC9B00F0000E476E070E466E000E496E190E48F9
:10ACAB006EBA0E4A6EFF0E4B6EB2EC22F0DEEC105B
:10ACBB00F0000E026E0A0E016EA5EC11F0F1EC1B0A
:10ACCB00F0000E026E0A0E016EA5EC11F053EC169D
:10ACDB00F0000E026E0A0E016EA5EC11F093EC1251
:10ACEB00F0000E026E0A0E016EA5EC11F0000E05BF
:10ACFB006E400E046E9AEC14F0000E056E420E04BC
:10AD0B006E9AEC14F0000E056E440E046E9AEC1461
:10AD1B00F0A20EC0EC19F006C0FDF107C0FEF1D099
:10AD2B000E0101BC6FC90EE82EFED7BC2FFCD7005D
:10AD3B00D0A40EC0EC19F006C056F207C057F2D0E3
:10AD4B000E0101BC6FC90EE82EFED7BC2FFCD7003D
:10AD5B00D0A60EC0EC19F006C058F207C059F2D0BD
:10AD6B000E0101BC6FC90EE82EFED7BC2FFCD7001D
:10AD7B00D0A80EC0EC19F006C05AF207C05BF2D097
:10AD8B000E0101BC6FC90EE82EFED7BC2FFCD700FD
:10AD9B00D0AA0EC0EC19F006C05CF207C05DF2D071
:10ADAB000E0101BC6FC90EE82EFED7BC2FFCD700DD
:10ADBB00D0AC0EC0EC19F006C05EF207C05FF2001B
:10ADCB000E0201FD6F000EFC6F000EFB6F000EFA02
:10ADDB006F000E5F6E000E0101FF6F000E026E0022
:10ADEB000E016EE5EC10F00101BC6FBC510201FCD1
:10ADFB00250101BD6F000E0201FD210101BE6FBDDA
:10AE0B00C1BEF1BD6BBDC1FCF2BEC1FDF2000E02B5
:10AE1B006E0A0E016EA5EC11F0000E026E010E0112
:10AE2B006EE5EC10F00101BC6FBC510201FC25FC7E
:10AE3B006F000EFD21FD6F000E026E0A0E016EA556
:10AE4B00EC11F0000E026E100E016EE5EC10F0012D
:10AE5B0001BC6FBC510201FA250101BD6F000E024E
:10AE6B0001FB210101BE6FBDC1BEF1BD6BBDC1FABE
:10AE7B00F2BEC1FBF2000E026E0A0E016EA5EC11C2
:10AE8B00F0000E026E110E016EE5EC10F00101BC2C
:10AE9B006FBC510201FA25FA6F000EFB21FB6F000C
:10AEAB000E026E0A0E016EA5EC11F0000E026E2062
:10AEBB000E016EE5EC10F05F6E000E026E0A0E01D5
:10AECB006EA5EC11F0000E026E210E016EE5EC107A
:10AEDB00F00101FF6F000E026E0A0E016EA5EC1160
:10AEEB00F00201FC290BE1FD29D8A408D0000EFDCE
:10AEFB006F000EFC6F000EFB6F000EFA6F000E1F43
:10AF0B006E000E206E700E216E420E226E0101FF3E
:10AF1B0051016E026A036A046A010E8BEC1CF0018C
:10AF2B00C01BF002C01CF003C01DF004C01EF005D6
:10AF3B00EC26F01BC038F01CC039F01DC03AF01ED7
:10AF4B00C03BF05F50016E000E01BEFF0E026E03A0
:10AF5B006E046E010E8BEC1CF001C034F002C03598
:10AF6B00F003C036F004C037F0A6EC28F034C0B0C4
:10AF7B00F235C0B1F236C0B2F237C0B3F2000E1FD9
:10AF8B006E000E206E340E216E430E226EB0C21B6D
:10AF9B00F0B1C21CF0B2C21DF0B3C21EF005EC261C
:10AFAB00F01BC044F01CC045F01DC046F01EC0474E
:10AFBB00F0DB0E486E0F0E496E490E4A6E400E4B7B
:10AFCB006E2CEC2AF044C0D8F245C0D9F246C0DA58
:10AFDB00F247C0DBF2A6EC3FF0FFEC10F0DEEC101A
:10AFEB00F0780E0201A86F320EA96F000E6A6F5037
:10AFFB000E6B6F7D0E6C6F440E6D6F23EEC4F007FE
:10B00B000EDE6AE806FDE222EEB8F0070EDE6AE815
:10B01B0006FDE222EEC0F0070EDE6AE806FDE22234
:10B02B00EEDCF0070EDE6AE806FDE2780EA819D812
:10B03B00A467EF5EF0FCC28CF1FDC28DF1FAC28EFB
:10B04B00F1FBC28FF1D8C290F1D9C291F1DAC29261
:10B05B00F1DBC293F1F1EC1FF001018C51ED6F8D1F
:10B06B0051EE6F8E51EF6F8F51F06FF16BF26BF3FF
:10B07B006BF46B02015C510101BC6F02015D51016C
:10B08B0001BD6FBE6BBF6BBEC1BFF1BDC1BEF1BC1D
:10B09B00C1BDF1BC6BBC51C06FBD51C16FBE51C2C4
:10B0AB006FBF51C36FC46BC56BC66BC76BC051ED24
:10B0BB005D0201F26F0101C151EE590201F36F0103
:10B0CB0001C251EF590201F46F0101C351F0590252
:10B0DB0001F56F0101C451F1590201F66F0101C570
:10B0EB0051F2590201F76F0101C651F3590201F8F0
:10B0FB006F0101C751F4590201F96F170E0101BC21
:10B10B006F5EC201F05FC202F0036A046A056A0651
:10B11B006A076A086AF2C209F0F3C20AF0F4C20BBA
:10B12B00F0F5C20CF0F6C20DF0F7C20EF0F8C20F3C
:10B13B00F0F9C210F0DDEC14F001C0BDF102C0BE9D
:10B14B00F103C0BFF104C0C0F105C0C1F106C0C21C
:10B15B00F107C0C3F108C0C4F10101BC6701D00BFA
:10B16B00D0C435C433C333C233C133C033BF33BE92
:10B17B0033BD33BC2FF1D7D00E0101BD250301C464
:10B18B006F070E0101BE210301C56F000E0101BF48
:10B19B00210301C66F000E0101C0210301C76F001F
:10B1AB000E0101C1210301C86F000E0101C2210371
:10B1BB0001C96F000E0101C3210301CA6F000E010B
:10B1CB0001C4210301CB6F070E0101BC6F5AC201F1
:10B1DB00F05BC202F0036A046A056A066A076A0832
:10B1EB006AF2C209F0F3C20AF0F4C20BF0F5C20C1A
:10B1FB00F0F6C20DF0F7C20EF0F8C20FF0F9C21064
:10B20B00F0DDEC14F001C0BDF102C0BEF103C0BF14
:10B21B00F104C0C0F105C0C1F106C0C2F107C0C343
:10B22B00F108C0C4F10101BC6701D00BD0C435C417
:10B23B0033C333C233C133C033BF33BE33BD33BC6F
:10B24B002FF1D7020156510101C56F020157510170
:10B25B0001C66FC76BC86BC6C1C8F1C5C1C7F1C604
:10B26B006BC56BC551C96FC651CA6FC751CB6FC880
:10B27B0051CC6FCD6BCE6BCF6BD06BBD51C9250253
:10B28B0001C06F0101BE51CA210201C16F0101BF93
:10B29B0051CB210201C26F0101C051CC210201C36C
:10B2AB006F0101C151CD210201C46F0101C251CE09
:10B2BB00210201C56F0101C351CF210201C66F01EC
:10B2CB0001C451D0210201C76F58C201F059C2020B
:10B2DB00F0036A046A056A066A076A086AF2C20919
:10B2EB00F0F3C20AF0F4C20BF0F5C20CF0F6C20D8B
:10B2FB00F0F7C20EF0F8C20FF0F9C210F0DDEC144B
:10B30B00F001C0BCF102C0BDF103C0BEF104C0BF6F
:10B31B00F105C0C0F106C0C1F107C0C2F108C0C33E
:10B32B00F1BDC1BCF1BEC1BDF1BFC1BEF1C0C1BF5A
:10B33B00F1C1C1C0F1C2C1C1F1C3C1C2F10101C3AD
:10B34B006BC2BFC369FD51C46FFE51C56FC66BC7DE
:10B35B006B0F0ED890C437C537C637C737E82EF9F1
:10B36B00D7C451C86FC551C96FC651CA6FC751CB2E
:10B37B006FCC6BCD6BCE6BCF6BBC51C8250201B8BC
:10B38B006F0101BD51C9210201B96F0101BE51CA43
:10B39B00210201BA6F0101BF51CB210201BB6F0129
:10B3AB0001C051CC210201BC6F0101C151CD210261
:10B3BB0001BD6F0101C251CE210201BE6F0101C35C
:10B3CB0051CF210201BF6F22EE62F0070EDE6AE859
:10B3DB0006FDE222EEC8F0070EDE6AE806FDE22269
:10B3EB00EED0F0070EDE6AE806FDE20301CBBF0DDF
:10B3FB00D0CB51CA11C911C811C711C61105E1D063
:10B40B000EC45D070EC559D8B088D1F2C209F0F34E
:10B41B00C20AF0F4C20BF0F5C20CF0F6C20DF0F755
:10B42B00C20EF0F8C20FF0F9C210F0F2C201F0F345
:10B43B00C202F0F4C203F0F5C204F0F6C205F0F755
:10B44B00C206F0F8C207F0F9C208F0DDEC14F00107
:10B45B00C019F002C01AF003C01BF004C01CF005A9
:10B46B00C01DF006C01EF007C01FF008C020F00082
:10B47B000E216E000E226E000E236E800E246E00C7
:10B48B000E256E000E266E000E276E000E286ECD5A
:10B49B00EC1DF019C062F21AC063F21BC064F21CFF
:10B4AB00C065F21DC066F21EC067F21FC068F220B5
:10B4BB00C069F223EEC4F0300EDE24096EF80EDE06
:10B4CB00200A6EFF0EDE200B6EFF0EDE200C6EFFD1
:10B4DB000EDE200D6EFF0EDE200E6EFF0EDE200F39
:10B4EB006EFF0EDE20106E23EEC4F0300EDE240154
:10B4FB006EF80EDE20026EFF0EDE20036EFF0EDEF8
:10B50B0020046EFF0EDE20056EFF0EDE20066EFFA2
:10B51B000EDE20076EFF0EDE20086EDDEC14F00150
:10B52B00C0EAF202C0EBF203C0ECF204C0EDF2058C
:10B53B00C0EEF206C0EFF207C0F0F208C0F1F20560
:10B54B000E096E000E0A6E000E0B6E000E0C6E00D6
:10B55B000E0D6E000E0E6E000E0F6E000E106EEACC
:10B56B00C201F0EBC202F0ECC203F0EDC204F0EE4C
:10B57B00C205F0EFC206F0F0C207F0F1C208F0DD31
:10B58B00EC14F001C019F002C01AF003C01BF00458
:10B59B00C01CF005C01DF006C01EF007C01FF00850
:10B5AB00C020F0020E216E000E226E000E236E00E4
:10B5BB000E246E000E256E000E266E000E276E00FA
:10B5CB000E286ECDEC1DF019C0C8F21AC0C9F21BC3
:10B5DB00C0CAF21CC0CBF21DC0CCF21EC0CDF21FF4
:10B5EB00C0CEF220C0CFF223EEC4F0300EDE240921
:10B5FB006EF80EDE200A6EFF0EDE200B6EFF0EDEE7
:10B60B00200C6EFF0EDE200D6EFF0EDE200E6EFF89
:10B61B000EDE200F6EFF0EDE20106E23EEC4F03018
:10B62B000EDE24016EF80EDE20026EFF0EDE20030E
:10B63B006EFF0EDE20046EFF0EDE20056EFF0EDEAB
:10B64B0020066EFF0EDE20076EFF0EDE20086EDD7D
:10B65B00EC14F001C0EAF202C0EBF203C0ECF2040E
:10B66B00C0EDF205C0EEF206C0EFF207C0F0F20833
:10B67B00C0F1F2050E096E000E0A6E000E0B6E0085
:10B68B000E0C6E000E0D6E000E0E6E000E0F6E0089
:10B69B000E106EEAC201F0EBC202F0ECC203F0ED49
:10B6AB00C204F0EEC205F0EFC206F0F0C207F0F1F3
:10B6BB00C208F0DDEC14F001C019F002C01AF0035F
:10B6CB00C01BF004C01CF005C01DF006C01EF00727
:10B6DB00C01FF008C020F0040E216E000E226E0079
:10B6EB000E236E000E246E000E256E000E266E00CD
:10B6FB000E276E000E286ECDEC1DF019C0D0F21A7D
:10B70B00C0D1F21BC0D2F21CC0D3F21DC0D4F21EAA
:10B71B00C0D5F21FC0D6F220C0D7F20301CBAF7653
:10B72B00D1240EC45DFA0EC559FF0EC659FF0EC7C4
:10B73B0059FF0EC859FF0EC959FF0ECA59FF0ECB40
:10B74B0059D8B064D123EEC4F0DC0EDE24096E05AB
:10B75B000EDE200A6E000EDE200B6E000EDE200CBD
:10B76B006E000EDE200D6E000EDE200E6E000EDE65
:10B77B00200F6E000EDE20106E23EEC4F0DC0EDE0A
:10B78B0024016E050EDE20026E000EDE20036E001D
:10B79B000EDE20046E000EDE20056E000EDE20068F
:10B7AB006E000EDE20076E000EDE20086EDDEC1440
:10B7BB00F001C0EAF202C0EBF203C0ECF204C0ED00
:10B7CB00F205C0EEF206C0EFF207C0F0F208C0F1CE
:10B7DB00F2EAC201F0EBC202F0ECC203F0EDC204DC
:10B7EB00F0EEC205F0EFC206F0F0C207F0F1C208AE
:10B7FB00F0070E096E000E0A6E000E0B6E000E0C9B
:10B80B006E000E0D6E000E0E6E000E0F6E000E1003
:10B81B006EDDEC14F001C0BCF102C0BDF103C0BE83
:10B82B00F104C0BFF105C0C0F106C0C1F107C0C231
:10B83B00F108C0C3F10201C8510101BC250201C8C6
:10B84B006FC9510101BD210201C96FCA510101BE6E
:10B85B00210201CA6FCB510101BF210201CB6FCC79
:10B86B00510101C0210201CC6FCD510101C1210257
:10B87B0001CD6FCE510101C2210201CE6FCF51011B
:10B88B0001C3210201CF6F23EEC4F0DC0EDE2409CD
:10B89B006E050EDE200A6E000EDE200B6E000EDE35
:10B8AB00200C6E000EDE200D6E000EDE200E6E00E4
:10B8BB000EDE200F6E000EDE20106E23EEC4F0DCC9
:10B8CB000EDE24016E050EDE20026E000EDE20035E
:10B8DB006E000EDE20046E000EDE20056E000EDE06
:10B8EB0020066E000EDE20076E000EDE20086EDDD9
:10B8FB00EC14F001C0EAF202C0EBF203C0ECF2046C
:10B90B00C0EDF205C0EEF206C0EFF207C0F0F20890
:10B91B00C0F1F20B0E096E000E0A6E000E0B6E00DC
:10B92B000E0C6E000E0D6E000E0E6E000E0F6E00E6
:10B93B000E106EEAC201F0EBC202F0ECC203F0EDA6
:10B94B00C204F0EEC205F0EFC206F0F0C207F0F150
:10B95B00C208F0DDEC14F001C019F002C01AF003BC
:10B96B00C01BF004C01CF005C01DF006C01EF00784
:10B97B00C01FF008C020F0020E216E000E226E00D8
:10B98B000E236E000E246E000E256E000E266E002A
:10B99B000E276E000E286ECDEC1DF019C0BCF11AEF
:10B9AB00C0BDF11BC0BEF11CC0BFF11DC0C0F11E5C
:10B9BB00C0C1F11FC0C2F120C0C3F10201D05101BF
:10B9CB0001BC250201D06FD1510101BD210201D172
:10B9DB006FD2510101BE210201D26FD3510101BFC0
:10B9EB00210201D36FD4510101C0210201D46FD5C3
:10B9FB00510101C1210201D56FD6510101C22102B2
:10BA0B0001D66FD7510101C3210201D76F02016229
:10BA1B00510301C45DC46F020163510301C559C5D4
:10BA2B006F020164510301C659C66F0201655103D0
:10BA3B0001C759C76F020166510301C859C86F028C
:10BA4B000167510301C959C96F020168510301CA4A
:10BA5B0059CA6F020169510301CB59CB6F0201C85F
:10BA6B0051C05DC06FC951C159C16FCA51C259C2D2
:10BA7B006FCB51C359C36FCC51C459C46FCD51C592
:10BA8B0059C56FCE51C659C66FCF51C759C76FD065
:10BA9B0051B85DB86FD151B959B96FD251BA59BAC2
:10BAAB006FD351BB59BB6FD451BC59BC6FD551BD72
:10BABB0059BD6FD651BE59BE6FD751BF59BF6F819C
:10BACB00AC77D0C4C301F0C5C302F0C6C303F0C743
:10BADB00C304F0C8C305F0C9C306F0CAC307F0CB53
:10BAEB00C308F0010EC6EC23F001C01BF002C01C12
:10BAFB00F003C01DF004C01EF0000E1F6E000E20E0
:10BB0B006EC80E216E420E226E05EC26F01BC0B4E1
:10BB1B00F21CC0B5F21DC0B6F21EC0B7F2190E0072
:10BB2B0001EC6F020EED6FD80EEE6FFF0EEF6FB4E0
:10BB3B00C2F0F0B5C2F1F0B6C2F2F0B7C2F3F00446
:10BB4B00EC13F0000E476E0F0E466E000E496E059D
:10BB5B000E486E190E4A6E020E4B6EB2EC22F07B43
:10BB6B000E016EFF0E026E1FEC11F0000E476E4BB6
:10BB7B000E466E000E496E040E486EFD0E4A6EFFA9
:10BB8B000E4B6EB2EC22F0880E016EFF0E026E1F92
:10BB9B00EC11F0000E476E510E466E000E496E050D
:10BBAB000E486EFB0E4A6EFF0E4B6EB2EC22F08609
:10BBBB00D0660E486E660E496EE60E4A6E3F0E4B11
:10BBCB006E000E1F6E000E206EC80E216E420E22EE
:10BBDB006EC4C301F0C5C302F0C6C303F0C7C304F0
:10BBEB00F0C8C305F0C9C306F0CAC307F0CBC3083E
:10BBFB00F0010EC6EC23F001C01BF002C01CF003D9
:10BC0B00C01DF004C01EF005EC26F01BC044F01C58
:10BC1B00C045F01DC046F01EC047F02CEC2AF04486
:10BC2B00C034F045C035F046C036F047C037F000A1
:10BC3B000E386E000E396E000E3A6E420E3B6EA63B
:10BC4B00EC28F034C042F235C043F236C044F23730
:10BC5B00C045F2190E0001EC6F020EED6FD80EEE1F
:10BC6B006FFF0EEF6F42C2F0F043C2F1F044C2F22D
:10BC7B00F045C2F3F004EC13F0000E476E0F0E46C6
:10BC8B006E000E496E050E486E190E4A6E020E4B73
:10BC9B006EB2EC22F0880E016EFF0E026E1FEC11DD
:10BCAB00F0000E476E4B0E466E000E496E040E48AA
:10BCBB006EE40E4A6EFF0E4B6EB2EC22F0000E02DB
:10BCCB0001A86F320EA919D8A403EF63F0000EE59B
:10BCDB006F000EE46FE5BF06D0E5514AE1070EE4B5
:10BCEB005DD8B046D0FCC28CF1FDC28DF1FAC28E8C
:10BCFB00F1FBC28FF1D8C290F1D9C291F1DAC292A5
:10BD0B00F1DBC293F1D5EC20F001018C51F56F8D75
:10BD1B0051F66F8E51F76F8F51F86FF96BFA6BFB12
:10BD2B006BFC6BE4C2BCF1E5C2BDF1D890BC37BD76
:10BD3B0037D890BC37BD37D890BC37BD37700EBCE9
:10BD4B0025D96E020EBD21DA6EF5C1DEFFF6C1DE1E
:10BD5B00FFF7C1DEFFF8C1DEFFF9C1DEFFFAC1DE7E
:10BD6B00FFFBC1DEFFFCC1DEFF0201E44BE52BB2A2
:10BD7B00D723EEBCF0070EDE6AE806FDE20301C333
:10BD8B0051C211C111C011BF11BE11BD1101E12171
:10BD9B00D124D1010EBC25B46F000EBD21B56F00AF
:10BDAB000EBE21B66F000EBF21B76F000EC021B8BB
:10BDBB006F000EC121B96F000EC221BA6F000EC306
:10BDCB0021BB6FBB51BA11B911B811B711B611B56F
:10BDDB001101E1E9D0ECD0BCC3BCF1BDC3BDF10195
:10BDEB0001D890BC37BD37D890BC37BD37D890BC85
:10BDFB0037BD37700EBC25D96E020EBD21DA6EB47D
:10BE0B00C3C6F1B5C3C7F1D890C637C737D890C6EC
:10BE1B0037C737D890C637C737700EC625E16E02C5
:10BE2B000EC721E26EDE50E65CDE50E658DE50E6D1
:10BE3B0058DE50E658DE50E658DE50E658DE50E647
:10BE4B0058DE50E658D8B09CD0BCC3BCF1BDC3BDC6
:10BE5B00F1D890BC37BD37D890BC37BD37D890BC24
:10BE6B0037BD37700EBC25D96E020EBD21DA6EDEE2
:10BE7B00CFBEF1DECFBFF1DECFC0F1DECFC1F1DE41
:10BE8B00CFC2F1DECFC3F1DECFC4F1DECFC5F1BE41
:10BE9B00C132F2BFC133F2C0C134F2C1C135F2C2FB
:10BEAB00C136F2C3C137F2C4C138F2C5C139F2B4DD
:10BEBB00C3BCF1B5C3BDF1D890BC37BD37D890BC6E
:10BECB0037BD37D890BC37BD37700EBC25D96E0245
:10BEDB000EBD21DA6EDECFBEF1DECFBFF1DECFC0FD
:10BEEB00F1DECFC1F1DECFC2F1DECFC3F1DECFC4C5
:10BEFB00F1DECFC5F1BCC3C6F1BDC3C7F1D890C647
:10BF0B0037C737D890C637C737D890C637C73770BB
:10BF1B000EC625D96E020EC721DA6EBEC1DEFFBF7B
:10BF2B00C1DEFFC0C1DEFFC1C1DEFFC2C1DEFFC388
:10BF3B00C1DEFFC4C1DEFFC5C1DEFFB4C3BCF1B5BA
:10BF4B00C3BDF1D890BC37BD37D890BC37BD37D8FF
:10BF5B0090BC37BD37700EBC25D96E020EBD21DAF1
:10BF6B006E32C2DEFF33C2DEFF34C2DEFF35C2DE0D
:10BF7B00FF36C2DEFF37C2DEFF38C2DEFF39C2DE5C
:10BF8B00FF010E0301B427000EB523B623B723B868
:10BF9B0023B923BA23BB23BB51BA11B911B811B7BB
:10BFAB0011B611B51104E1070EB45DD8A014D70179
:10BFBB000EBC27000EBD23BE23BF23C023C123C24B
:10BFCB0023C323C351C211C111C011BF11BE11BD77
:10BFDB001104E1060EBC5DD8A0DCD6D8900201801E
:10BFEB00350101BC6F020181350101BD6F02018278
:10BFFB00350101BE6F020183350101BF6F02018460
:10C00B00350101C06F020185350101C16F02018647
:10C01B00350101C26F020187350101C36F02019027
:10C02B00510101BC25C46F020191510101BD21C514
:10C03B006F020192510101BE21C66F0201935101A2
:10C04B0001BF21C76F020194510101C021C86F02CA
:10C05B000195510101C121C96F020196510101C224
:10C06B0021CA6F020197510101C321CB6F020198C5
:10C07B00510101C425CC6F020199510101C521CD9C
:10C08B006F02019A510101C621CE6F02019B510132
:10C09B0001C721CF6F02019C510101C821D06F0252
:10C0AB00019D510101C921D16F02019E510101CAAC
:10C0BB0021D26F02019F510101CB21D36F030E09D6
:10C0CB00D0D890D333D233D133D033CF33CE33CD4B
:10C0DB0033CC33E82EF5D7CCC13AF2CDC13BF2CEFF
:10C0EB00C13CF2CFC13DF2D0C13EF2D1C13FF2D241
:10C0FB00C140F2D3C141F2B8C201F0B9C202F0BAE9
:10C10B00C203F0BBC204F0BCC205F0BDC206F0BE58
:10C11B00C207F0BFC208F03AC209F03BC20AF03CBA
:10C12B00C20BF03DC20CF03EC20DF03FC20EF04010
:10C13B00C20FF041C210F0DDEC14F001C0BCF102F3
:10C14B00C0BDF103C0BEF104C0BFF105C0C0F10614
:10C15B00C0C1F107C0C2F108C0C3F1160E0AD0016D
:10C16B0001D890C333C233C133C033BF33BE33BDE9
:10C17B0033BC33E82EF4D70201C0510101BC5DC4BE
:10C18B006F0201C1510101BD59C56F0201C25101BD
:10C19B0001BE59C66F0201C3510101BF59C76F02DE
:10C1AB0001C4510101C059C86F0201C5510101C140
:10C1BB0059C96F0201C6510101C259CA6F0201C7A9
:10C1CB00510101C359CB6F100E09D0D890CB33CA94
:10C1DB0033C933C833C733C633C533C433E82EF53D
:10C1EB00D7C4C1DCF2C5C1DDF2C6C1DEF2C7C1DF07
:10C1FB00F2C8C1E0F2C9C1E1F2CAC1E2F2CBC1E3BC
:10C20B00F2DCC201F0DDC202F0DEC203F0DFC204D9
:10C21B00F0E0C205F0E1C206F0E2C207F0E3C208AB
:10C22B00F0010EC6EC23F001C01BF002C01CF003A2
:10C23B00C01DF004C01EF0000E1F6E000E206EC855
:10C24B000E216E420E226E05EC26F01BC0B4F21CC2
:10C25B00C0B5F21DC0B6F21EC0B7F2D40E0001EC91
:10C26B006F010EED6FD80EEE6FFF0EEF6FB4C2F0D5
:10C27B00F0B5C2F1F0B6C2F2F0B7C2F3F004EC13B2
:10C28B00F0000E476E0F0E466E000E496E140E48F0
:10C29B006ED40E4A6E010E4B6EB2EC22F0DEEC1039
:10C2AB00F0000E476E4B0E466E000E496E140E4894
:10C2BB006EDD0E4A6EFF0E4B6EB2EC22F0DEEC1012
:10C2CB00F0000E1F6E000E206EC80E216E420E2265
:10C2DB006EDCC201F0DDC202F0DEC203F0DFC2048D
:10C2EB00F0E0C205F0E1C206F0E2C207F0E3C208DB
:10C2FB00F0010EC6EC23F001C01BF002C01CF003D2
:10C30B00C01DF004C01EF005EC26F01BC0B0F21CE3
:10C31B00C0B1F21DC0B2F21EC0B3F2B0C21FF0B179
:10C32B00C220F0B2C221F0B3C222F06AC21BF06B82
:10C33B00C21CF06CC21DF06DC21EF005EC26F01B8A
:10C34B00C04AF21CC04BF21DC04CF21EC04DF2B4E1
:10C35B000E0001A96FC90EAA6F420EAB6F3E0EAC59
:10C36B006F4AC2A5F04BC2A6F04CC2A7F04DC2A8B3
:10C37B00F051EC63F0A5C04EF2A6C04FF2A7C0502F
:10C38B00F2A8C051F2330E386E930E396E880E3A06
:10C39B006E430E3B6E000E1F6E000E206EC80E21FC
:10C3AB006E420E226EC4C301F0C5C302F0C6C303B6
:10C3BB00F0C7C304F0C8C305F0C9C306F0CAC3076E
:10C3CB00F0CBC308F0010EC6EC23F001C01BF0024A
:10C3DB00C01CF003C01DF004C01EF005EC26F01BC2
:10C3EB00C034F01CC035F01DC036F01EC037F0A6AF
:10C3FB00EC28F034C048F035C049F036C04AF0376D
:10C40B00C04BF0000E386E000E396E800E3A6EBFC8
:10C41B000E3B6E4EC234F04FC235F050C236F05167
:10C42B00C237F0A6EC28F034C044F035C045F036E6
:10C43B00C046F037C047F02CEC2AF044C052F2450E
:10C44B00C053F246C054F247C055F252C21BF053D0
:10C45B00C21CF054C21DF055C21EF0F40E1F6EFD2F
:10C46B000E206ED40E216E3B0E226E05EC26F01BB9
:10C47B00C0E6F21CC0E7F21DC0E8F21EC0E9F202F2
:10C48B0001E9BF04D0B90E6E6FFF0E03D0F90E6E2B
:10C49B006FFF0E6F6FE9BF09D0E6C2ACF2E7C2AD1A
:10C4AB00F2E8C2AEF2E9C2AFF212D0E6C201F0E797
:10C4BB00C202F0E8C203F0E9C204F045EC11F0014E
:10C4CB00C0ACF202C0ADF203C0AEF204C0AFF2AC2E
:10C4DB00C274F0ADC275F0AEC276F0AFC277F05554
:10C4EB00EC17F074C0AAF275C0ABF2ACC260F0AD41
:10C4FB00C261F0AEC262F0AFC263F0AAC201F0AB90
:10C50B00C202F0000E02BEFF0E036E046E010E8B14
:10C51B00EC1CF001C064F002C065F003C066F004CF
:10C52B00C067F06FEC12F060C046F261C047F26278
:10C53B00C048F263C049F2000E486E000E496EC847
:10C54B000E4A6E420E4B6E46C244F047C245F0484F
:10C55B00C246F049C247F02CEC2AF044C060F045CB
:10C56B00C061F046C062F047C063F038EC1AF0606F
:10C57B00C074F061C075F062C076F063C077F0559F
:10C58B00EC17F074C060F275C061F2000E0001ECA4
:10C59B006F020EED6FA90EEE6FFF0EEF6F6EC2F016
:10C5AB00F06FC2F1F0AAC2F2F0ABC2F3F060C2F4CA
:10C5BB00F061C2F5F004EC13F0000E476E0F0E465F
:10C5CB006E000E496E320E486E000E4A6E020E4B16
:10C5DB006EB2EC22F0000E476E4B0E466E000E490B
:10C5EB006E320E486EF20E4A6EFF0E4B6EB2EC229E
:10C5FB00F0DEEC10F0000E0201A96F81B035D00017
:10C60B000E026E140E016EA5EC11F081B02DD0DC74
:10C61B00C201F0DDC202F0DEC203F0DFC204F0E0C3
:10C62B00C205F0E1C206F0E2C207F0E3C208F00176
:10C63B000EC6EC23F001C01BF002C01CF003C01DA2
:10C64B00F004C01EF0000E1F6E000E206EC80E21EF
:10C65B006E420E226E05EC26F01BC06AF21CC06BFC
:10C66B00F21DC06CF21EC06DF2FCC200F1FDC201E6
:10C67B00F1FAC202F1FBC203F1D8C204F1D9C2052F
:10C68B00F1DAC206F1DBC207F192EC44F00201A829
:10C69B002BA92B1BEF58F0A5C0B8F1A6C0B9F1A779
:10C6AB00C0BAF1A8C0BBF1B8C160F1B9C161F1BAB0
:10C6BB00C162F1BBC163F1A9C0B8F1AAC0B9F1ABBA
:10C6CB00C0BAF1ACC0BBF1B8C184F1B9C185F1BA44
:10C6DB00C186F1BBC187F1FF0E01016015A86FFF89
:10C6EB000E6115A96FFF0E6215AA6F7F0E6315AB56
:10C6FB006FFF0E8415986FFF0E8515996FFF0E86D1
:10C70B00159A6F7F0E87159B6F985199119A119BF4
:10C71B0011D8A40AD0000E0001A56F000EA66F80E1
:10C72B000EA76F3F0EA86F1200800E621910E13F2B
:10C73B000E631960116111D8A40AD0000E0001A577
:10C74B006F000EA66F800EA76F3F0EA86F1200AB87
:10C75B00BF09D0A805000EA959800EAA597F0EABB0
:10C76B0059D8B00BD09BBF24D09805000E99598097
:10C77B000E9A597F0E9B59D8A01BD0A5C034F0A69A
:10C78B00C035F0A7C036F0A8C037F0A9C038F0AA62
:10C79B00C039F0ABC03AF0ACC03BF0A6EC28F0349B
:10C7AB00C0A5F035C0A6F036C0A7F037C0A8F01270
:10C7BB0000000E506F000E516F000E526F000E53A3
:10C7CB006F63AFB1D09BBF0ED0800E9A5D4B0E9BAB
:10C7DB0059D8A008D0020E506F000E516F000E52A8
:10C7EB006F000EA0D09BBF9FD0800E9A5D3F0E9B1B
:10C7FB0059D8A099D0170E0001AD6F98C1AEF09922
:10C80B00C1AFF09AC1B0F09BC1B1F0AD6701D007D9
:10C81B00D0B135B133B033AF33AE33AD2FF6D781A3
:10C82B000E0001AE250101A06FFF0E0001AF21012B
:10C83B0001A16FFF0E0001B0210101A26FFF0E00DD
:10C84B0001B1210101A36FA05117080001AD6F9831
:10C85B00C1AEF099C1AFF09AC1B0F09BC1B1F0ADD0
:10C86B006701D007D0B135B133B033AF33AE33AD91
:10C87B002FF6D7AEC0ACF1AFC0ADF1B0C0AEF1B1D9
:10C88B00C0AFF10101A05117080001AD6FACC1AEF3
:10C89B00F0ADC1AFF0AEC1B0F0AFC1B1F0AD2B0593
:10C8AB00D0D890AE37AF37B037B137AD2FF9D701FE
:10C8BB000198510001AE1937E1010199510001AF07
:10C8CB001932E101019A510001B0192DE101019BCF
:10C8DB00510001B119D8A427D0010E0101AC1500EC
:10C8EB0001AD6F000E0101AD150001AE6F000E0121
:10C8FB0001AE150001AF6F000E0101AF150001B0C5
:10C90B006FAD5102080101506F000E0001AE5501D1
:10C91B0001516F000E0001AF550101526F000E0067
:10C92B0001B0550101536F800E01019A1958E17F37
:10C93B000E9B1998119911D8A452D0800EAA1910D8
:10C94B00E13F0EAB19A811A911D8A40AD0000E0013
:10C95B0001A56F000EA66F800EA76F3F0EA86F127A
:10C96B0000ABBF1ED0A805000EA959800EAA593FD7
:10C97B000EAB59D8A015D087AF0AD0000E0001A579
:10C98B006F000EA66F000EA76F000EA86F1200A906
:10C99B00C0A5F0AAC0A6F0ABC0A7F0ACC0A8F0121F
:10C9AB000087AF13D0A9C001F0AAC002F0ABC0033F
:10C9BB00F0ACC004F045EC11F001C0A5F002C0A62C
:10C9CB00F003C0A7F004C0A8F01200000E0001A5F0
:10C9DB006F000EA66F000EA76F000EA86F120080DF
:10C9EB000E9A192CE13F0E9B1998119911D8A42678
:10C9FB00D087AF1BD0000E1B6E000E1C6E800E1D61
:10CA0B006E3F0E1E6EA5C01FF0A6C020F0A7C02162
:10CA1B00F0A8C022F005EC26F01BC0A5F01CC0A6A8
:10CA2B00F01DC0A7F01EC0A8F01200A5C0A5F0A66F
:10CA3B00C0A6F0A7C0A7F0A8C0A8F01200400E87B0
:10CA4B0019841185118611D8A41BD0A5C044F0A65A
:10CA5B00C045F0A7C046F0A8C047F0A5C048F0A657
:10CA6B00C049F0A7C04AF0A8C04BF02CEC2AF04408
:10CA7B00C0A5F045C0A6F046C0A7F047C0A8F0126D
:10CA8B00003F0E8719841185118611D8B463BF132B
:10CA9B00D0A5C074F0A6C075F0A7C076F0A8C0777B
:10CAAB00F0A7EC2DF074C0A5F075C0A6F076C0A76A
:10CABB00F077C0A8F01200A5C001F0A6C002F0A745
:10CACB00C003F0A8C004F0BFEC11F001C070F1027C
:10CADB00C071F103C072F104C073F1800E0101AAA1
:10CAEB001906E17F0EAB19A811A911D8B40FD0A864
:10CAFB0051A911AA11AB11D8B409D0800EAA1905EE
:10CB0B00E13F0EAB19A811A911D8A4B5D070C1B4CF
:10CB1B00F171C1B5F172C1B6F173C1B7F187AF1A3B
:10CB2B00D0000E1B6E000E1C6E800E1D6E3F0E1E77
:10CB3B006EB4C11FF0B5C120F0B6C121F0B7C12250
:10CB4B00F005EC26F01BC0B4F11CC0B5F11DC0B64E
:10CB5B00F11EC0B7F1010163AF85D0000EA825000F
:10CB6B0001AD6F000E0101A9210001AE6F800E0116
:10CB7B0001AA210001AF6FC00E0101AB210001B072
:10CB8B006F010150510001AD11B16F010151510005
:10CB9B0001AE11B26F010152510001AF11B36F0120
:10CBAB000153510001B011B46FB151B211B311B4B3
:10CBBB0011D8A43FD0B4C164F0B5C165F0B6C1665D
:10CBCB00F0B7C167F0B4C160F0B5C161F0B6C16236
:10CBDB00F0B7C163F06FEC12F060C01BF061C01CCA
:10CBEB00F062C01DF063C01EF0B4C164F0B5C16546
:10CBFB00F0B6C166F0B7C167F0B4C160F0B5C16102
:10CC0B00F0B6C162F0B7C163F06FEC12F060C01FF9
:10CC1B00F061C020F062C021F063C022F005EC2669
:10CC2B00F01BC0B4F11CC0B5F11DC0B6F11EC0B7EE
:10CC3B00F119D001015005511152115311D8A41201
:10CC4B00D0B4C101F0B5C102F0B6C103F0B7C10455
:10CC5B00F045EC11F001C0B4F102C0B5F103C0B660
:10CC6B00F104C0B7F1B4C1A5F0B5C1A6F0B6C1A728
:10CC7B00F0B7C1A8F01200000E886F000E896F800C
:10CC8B000E8A6F3F0E8B6F63AF53D05051511152C1
:10CC9B00115311D8A43FD0A5C064F0A6C065F0A76E
:10CCAB00C066F0A8C067F0A5C060F0A6C061F0A791
:10CCBB00C062F0A8C063F06FEC12F060C01BF061B3
:10CCCB00C01CF062C01DF063C01EF0A5C064F0A6CE
:10CCDB00C065F0A7C066F0A8C067F0A5C060F0A65D
:10CCEB00C061F0A7C062F0A8C063F06FEC12F060F7
:10CCFB00C01FF061C020F062C021F063C022F005BC
:10CD0B00EC26F01BC0A5F01CC0A6F01DC0A7F01EA2
:10CD1B00C0A8F012005005511152115311D8A4089C
:10CD2B00D0000E886F000E896F800E8A6FBF0E8B3E
:10CD3B006F9BBF6DD29805000E9959000E9A594DF5
:10CD4B000E9B59D8A064D2ABBF0AD0F80EA85DFFDA
:10CD5B000EA9597F0EAA593F0EAB59D8B06CD0878C
:10CD6B00BF35D0600E486E420E496EA20E4A6E0D54
:10CD7B000E4B6E88C144F089C145F08AC146F08BD9
:10CD8B00C147F02CEC2AF044C0A4F145C0A5F146F4
:10CD9B00C0A6F147C0A7F1A4C144F0A5C145F0A6B8
:10CDAB00C146F0A7C147F0600E486E420E496EA215
:10CDBB000E4A6E0D0E4B6E2CEC2AF044C0A5F045BE
:10CDCB00C0A6F046C0A7F047C0A8F01200CA0E4894
:10CDDB006EF20E496E490E4A6E710E4B6E88C1444F
:10CDEB00F089C145F08AC146F08BC147F02CEC2A83
:10CDFB00F044C0A4F145C0A5F146C0A6F147C0A7B9
:10CE0B00F1A4C144F0A5C145F0A6C146F0A7C147A6
:10CE1B00F0CA0E486EF20E496E490E4A6E710E4BF9
:10CE2B006E2CEC2AF044C0A5F045C0A6F046C0A776
:10CE3B00F047C0A8F01200ABBF7DD0080EA85D0074
:10CE4B000EA959800EAA593F0EAB59D8A073D087A3
:10CE5B00BF07D087518611851138E18405D8B035CD
:10CE6B00D0600E486E420E496EA20E4A6E0D0E4BEE
:10CE7B006E88C144F089C145F08AC146F08BC14729
:10CE8B00F02CEC2AF044C0A4F145C0A5F146C0A695
:10CE9B00F147C0A7F1A4C144F0A5C145F0A6C14616
:10CEAB00F0A7C147F0600E486E420E496EA20E4AC3
:10CEBB006E0D0E4B6E2CEC2AF044C0A5F045C0A6AF
:10CECB00F046C0A7F047C0A8F01200CA0E486EF299
:10CEDB000E496E490E4A6E710E4B6E88C144F08935
:10CEEB00C145F08AC146F08BC147F02CEC2AF044C7
:10CEFB00C0A4F145C0A5F146C0A6F147C0A7F1A457
:10CF0B00C144F0A5C145F0A6C146F0A7C147F0CA80
:10CF1B000E486EF20E496E490E4A6E710E4B6E2C18
:10CF2B00EC2AF044C0A5F045C0A6F046C0A7F047D8
:10CF3B00C0A8F0120070C134F071C135F072C13667
:10CF4B00F073C137F0000E386E000E396E800E3A5A
:10CF5B006EBF0E3B6EA6EC28F034C0B0F135C0B1FD
:10CF6B00F136C0B2F137C0B3F1000E486E000E4976
:10CF7B006E800E4A6E3E0E4B6EB0C144F0B1C14591
:10CF8B00F0B2C146F0B3C147F02CEC2AF044C064B8
:10CF9B00F045C065F046C066F047C067F0AB0E00C9
:10CFAB0001606FAA0E616FAA0E626F3E0E636F6F08
:10CFBB00EC12F060C0A4F161C0A5F162C0A6F163F0
:10CFCB00C0A7F1B0C148F0B1C149F0B2C14AF0B34A
:10CFDB00C14BF0B0C144F0B1C145F0B2C146F0B3A2
:10CFEB00C147F02CEC2AF044C054F145C055F14632
:10CFFB00C056F147C057F1B0C148F0B1C149F0B2CA
:10D00B00C14AF0B3C14BF0A4C144F0A5C145F0A691
:10D01B00C146F0A7C147F02CEC2AF044C064F045A0
:10D02B00C065F046C066F047C067F0000E000160B7
:10D03B006F000E616F000E626F3F0E636F6FEC122D
:10D04B00F060C048F161C049F162C04AF163C04B66
:10D05B00F154C144F055C145F056C146F057C14794
:10D06B00F048C148F049C149F04AC14AF04BC14BA5
:10D07B00F02CEC2AF044C044F145C045F146C046C3
:10D08B00F147C047F1B0C144F0B1C145F0B2C14660
:10D09B00F0B3C147F0000E486EAA0E496EB80E4AA7
:10D0AB006E3F0E4B6E2CEC2AF044C074F145C075EC
:10D0BB00F146C076F147C077F1700E486EA50E4968
:10D0CB006EEC0E4A6E360E4B6EB0C144F0B1C145DC
:10D0DB00F0B2C146F0B3C147F02CEC2AF044C0606B
:10D0EB00F045C061F046C062F047C063F03B0E48AC
:10D0FB006EAA0E496EB80E4A6E3F0E4B6E44C1447B
:10D10B00F045C145F046C146F047C147F02CEC2A2B
:10D11B00F044C064F045C065F046C066F047C06798
:10D12B00F06FEC12F060C078F161C079F162C07AF7
:10D13B00F163C07BF174C134F075C135F076C13643
:10D14B00F077C137F078C138F079C139F07AC13A4C
:10D15B00F07BC13BF0A6EC28F034C080F135C081E8
:10D16B00F136C082F137C083F180C1B8F181C1B90A
:10D17B00F182C1BAF183C1BBF1B8C190F1B9C191D0
:10D18B00F1BAC192F1BBC193F1000E01019015B838
:10D19B006FF00E9115B96FFF0E9215BA6FFF0E93CC
:10D1AB0015BB6FB8C180F1B9C181F1BAC182F1BBB6
:10D1BB00C183F174C164F075C165F076C166F07717
:10D1CB00C167F080C160F081C161F082C162F08300
:10D1DB00C163F06FEC12F060C094F161C095F16225
:10D1EB00C096F163C097F178C160F079C161F07AB4
:10D1FB00C162F07BC163F094C164F095C165F09698
:10D20B00C166F097C167F06FEC12F066EF70F0003B
:10D21B000E7C6F000E7D6F000E7E6F000E7F6FAB6E
:10D22B00BF06D0AB5137E1800EAA5DD8B033D070BA
:10D23B00C144F071C145F072C146F073C147F000B3
:10D24B000E486E000E496E800E4A6E4B0E4B6E2CC6
:10D25B00EC2AF044C070F145C071F146C072F14741
:10D26B00C073F1E80E01017C27FF0E7D23FF0E7EBC
:10D27B0023FF0E7F2370C1B8F171C1B9F172C1BA2E
:10D28B00F173C1BBF1B8C1A8F1B9C1A9F1BAC1AA77
:10D29B00F1BBC1ABF1170E0001AD6FA8C1AEF0A988
:10D2AB00C1AFF0AAC1B0F0ABC1B1F0AD6701D0070F
:10D2BB00D0B135B133B033AF33AE33AD2FF6D781F9
:10D2CB000E0001AE25B26FFF0EAF21B36FFF0EB094
:10D2DB0021B46FFF0EB121B56FB25101017C270054
:10D2EB0001B35101017D230001B45101017E2300E3
:10D2FB0001B55101017F23FF0EA815AC6FFF0EA9DD
:10D30B0015AD6F7F0EAA15AE6F000EAB15AF6F008C
:10D31B000EAC11A86F000EAD11A96F800EAE11AA45
:10D32B006F3F0EAF11AB6FAFBF0AD0AF510AE172B7
:10D33B000EAC5DC40EAD591C0EAE59D8B002D00068
:10D34B000E0DD0AFBF0AD0AF5111E1D70EAC5DB30C
:10D35B000EAD595D0EAE59D8B009D0010EA06F00BD
:10D36B000EA16F000EA26F000EA36F16D0000EA0C1
:10D37B006F000EA16F000EA26F000EA36F010E7C4B
:10D38B0027000E7D237E237F23000EA827000EA9E6
:10D39B0023800EAA23FF0EAB23A8C1B8F1A9C1B9F4
:10D3AB00F1AAC1BAF1ABC1BBF1B8C170F1B9C1718E
:10D3BB00F1BAC172F1BBC173F170C160F071C1619F
:10D3CB00F072C162F073C163F0A0C1ADF0A1C1AE48
:10D3DB00F00001D890AD37AE37D890AD37AE37955A
:10D3EB000EAD25F66EFF0EAE21F76EF86A000EF845
:10D3FB00220900F5CF64F00900F5CF65F00900F5BF
:10D40B00CF66F00A00F5CF67F06FEC12F060C074D6
:10D41B00F161C075F162C076F163C077F1000E1B4C
:10D42B006E000E1C6E800E1D6E3F0E1E6E70C13890
:10D43B00F071C139F072C13AF073C13BF0A0C1ADCC
:10D44B00F0A1C1AEF00001D890AD37AE37D890AD9A
:10D45B0037AE37950EAD25F66EFF0EAE21F76EF893
:10D46B006A000EF8220900F5CF34F00900F5CF352C
:10D47B00F00900F5CF36F00A00F5CF37F0A6EC280F
:10D48B00F034C01FF035C020F036C021F037C02279
:10D49B00F005EC26F01BC078F11CC079F11DC07AA9
:10D4AB00F11EC07BF174C144F075C145F076C146E5
:10D4BB00F077C147F078C148F079C149F07AC14A99
:10D4CB00F07BC14BF02CEC2AF044C05CF145C05D05
:10D4DB00F146C05EF147C05FF15CC16CF15DC16D9F
:10D4EB00F15EC16EF15FC16FF16CC1B8F16DC1B985
:10D4FB00F16EC1BAF16FC1BBF1B8C190F1B9C19175
:10D50B00F1BAC192F1BBC193F1000E01019015B8B4
:10D51B006FF00E9115B96FFF0E9215BA6FFF0E9348
:10D52B0015BB6FB8C16CF1B9C16DF1BAC16EF1BB6E
:10D53B00C16FF1A8C1ADF0A9C1AEF0AAC1AFF0ABFC
:10D54B00C1B0F00001B035B033AF33AE33AD330003
:10D55B000EAD15B16FF00EAE15B26FFF0EAF15B36A
:10D56B006FFF0EB015B46F000EB1110101906F007B
:10D57B000E0001B2110101916F000E0001B31101F8
:10D58B0001926F200E0001B4110101936FA0C1AD88
:10D59B00F0A1C1AEF0A2C1AFF0A3C1B0F0150ED88F
:10D5AB00900001AD37AE37AF37B037E82EF8D70163
:10D5BB000190510001AD25B16F010191510001AEF8
:10D5CB0021B26F010192510001AF21B36F010193A1
:10D5DB00510001B021B46F000EB1250101B86F00ED
:10D5EB000E0001B2210101B96F400E0001B3210100
:10D5FB0001BA6F000E0001B4210101BB6FB8C16805
:10D60B00F1B9C169F1BAC16AF1BBC16BF1A0C1AD8E
:10D61B00F0A1C1AEF00001D890AD37AE37D890ADC8
:10D62B0037AE37950EAD25F66EFF0EAE21F76EF8C1
:10D63B006A000EF8220900F5CF64F00900F5CF65FA
:10D64B00F00900F5CF66F00A00F5CF67F068C1600E
:10D65B00F069C161F06AC162F06BC163F06FEC12EB
:10D66B00F060C094F161C095F162C096F163C09710
:10D67B00F170C160F071C161F072C162F073C1638E
:10D68B00F094C164F095C165F096C166F097C167DF
:10D69B00F06FEC12F060C034F161C035F162C0364E
:10D6AB00F163C037F168C148F069C149F06AC14AFA
:10D6BB00F06BC14BF06CC144F06DC145F06EC146CF
:10D6CB00F06FC147F02CEC2AF044C064F045C06504
:10D6DB00F046C066F047C067F074C160F075C16179
:10D6EB00F076C162F077C163F06FEC12F060C0941A
:10D6FB00F161C095F162C096F163C097F134C148F6
:10D70B00F035C149F036C14AF037C14BF06CC1441A
:10D71B00F06DC145F06EC146F06FC147F02CEC2A9D
:10D72B00F044C064F045C065F046C066F047C06782
:10D73B00F094C160F095C161F096C162F097C1633E
:10D74B00F06FEC12F060C054F161C055F162C0563D
:10D75B00F163C057F154C144F055C145F056C14671
:10D76B00F057C147F078C148F079C149F07AC14A06
:10D77B00F07BC14BF02CEC2AF044C030F145C031AA
:10D78B00F146C032F147C033F15CC144F05DC14595
:10D79B00F05EC146F05FC147F05CC148F05DC14926
:10D7AB00F05EC14AF05FC14BF02CEC2AF044C08C08
:10D7BB00F145C08DF146C08EF147C08FF1550E3843
:10D7CB006E320E396E6C0E3A6E3E0E3B6E420E484A
:10D7DB006EF10E496E530E4A6E3E0E4B6E8CC1446B
:10D7EB00F08DC145F08EC146F08FC147F02CEC2A6D
:10D7FB00F044C034F045C035F046C036F047C03772
:10D80B00F0A6EC28F034C0A4F135C0A5F136C0A6C3
:10D81B00F137C0A7F1050E386EA30E396E8B0E3A99
:10D82B006E3E0E3B6E8CC148F08DC149F08EC14AE5
:10D83B00F08FC14BF0A4C144F0A5C145F0A6C14681
:10D84B00F0A7C147F02CEC2AF044C034F045C035AA
:10D85B00F046C036F047C037F0A6EC28F034C05481
:10D86B00F135C055F136C056F137C057F1AB0E3814
:10D87B006EAA0E396EAA0E3A6E3E0E3B6E8CC148E6
:10D88B00F08DC149F08EC14AF08FC14BF054C144A9
:10D89B00F055C145F056C146F057C147F02CEC2A64
:10D8AB00F044C034F045C035F046C036F047C037C1
:10D8BB00F0A6EC28F034C048F135C049F136C04A27
:10D8CB00F137C04BF1B70E386E6D0E396EDB0E3A79
:10D8DB006E3E0E3B6E8CC148F08DC149F08EC14A35
:10D8EB00F08FC14BF048C144F049C145F04AC146E5
:10D8FB00F04BC147F02CEC2AF044C034F045C03556
:10D90B00F046C036F047C037F0A6EC28F034C038EC
:10D91B00F135C039F136C03AF137C03BF19A0E38C8
:10D92B006E990E396E190E3A6E3F0E3B6E8CC148D6
:10D93B00F08DC149F08EC14AF08FC14BF038C14414
:10D94B00F039C145F03AC146F03BC147F02CEC2A07
:10D95B00F044C034F045C035F046C036F047C03710
:10D96B00F0A6EC28F034C000F135C001F136C0024E
:10D97B00F137C003F18CC148F08DC149F08EC14A1B
:10D98B00F08FC14BF08CC144F08DC145F08EC14678
:10D99B00F08FC147F02CEC2AF044C004F145C005D0
:10D9AB00F146C006F147C007F100C144F001C14583
:10D9BB00F002C146F003C147F004C148F005C1496C
:10D9CB00F006C14AF007C14BF02CEC2AF044C04CD6
:10D9DB00F145C04DF146C04EF147C04FF130C14843
:10D9EB00F031C149F032C14AF033C14BF05CC13860
:10D9FB00F05DC139F05EC13AF05FC13BF06CC134F0
:10DA0B00F06DC135F06EC136F06FC137F0A6EC2862
:10DA1B00F034C044F035C045F036C046F037C0474F
:10DA2B00F02CEC2AF044C058F145C059F146C05ACD
:10DA3B00F147C05BF14CC134F04DC135F04EC136EE
:10DA4B00F04FC137F058C138F059C139F05AC13ACB
:10DA5B00F05BC13BF0A6EC28F034C04CF135C04D67
:10DA6B00F136C04EF137C04FF16CC144F06DC1457A
:10DA7B00F06EC146F06FC147F06CC148F06DC14903
:10DA8B00F06EC14AF06FC14BF02CEC2AF044C08C05
:10DA9B00F145C08DF146C08EF147C08FF1000E38B5
:10DAAB006E000E396E400E3A6E400E3B6E8CC134DA
:10DABB00F08DC135F08EC136F08FC137F0A6EC2852
:10DACB00F034C058F135C059F136C05AF137C05B4C
:10DADB00F158C134F059C135F05AC136F05BC1373A
:10DAEB00F04CC138F04DC139F04EC13AF04FC13B4B
:10DAFB00F0A6EC28F034C068F135C069F136C06A85
:10DB0B00F137C06BF168C1B8F169C1B9F16AC1BA3B
:10DB1B00F16BC1BBF1B8C190F1B9C191F1BAC1922E
:10DB2B00F1BBC193F1000E01019015B86FF00E918E
:10DB3B0015B96FFF0E9215BA6FFF0E9315BB6FB829
:10DB4B00C168F1B9C169F1BAC16AF1BBC16BF1002E
:10DB5B000E386E000E396E400E3A6EC00E3B6E687C
:10DB6B00C134F069C135F06AC136F06BC137F0A62C
:10DB7B00EC28F034C03CF135C03DF136C03EF137F6
:10DB8B00C03FF18CC164F08DC165F08EC166F08F22
:10DB9B00C167F03CC160F03DC161F03EC162F03F36
:10DBAB00C163F06FEC12F060C040F161C041F162F3
:10DBBB00C042F163C043F14CC160F04DC161F04E06
:10DBCB00C162F04FC163F040C164F041C165F042E6
:10DBDB00C166F043C167F06FEC12F060C034F161C5
:10DBEB00C035F162C036F163C037F16CC144F06DE2
:10DBFB00C145F06EC146F06FC147F068C148F0698E
:10DC0B00C149F06AC14AF06BC14BF02CEC2AF044CD
:10DC1B00C074F145C075F146C076F147C077F16825
:10DC2B00C148F069C149F06AC14AF06BC14BF03091
:10DC3B00C144F031C145F032C146F033C147F02C3D
:10DC4B00EC2AF044C034F045C035F046C036F047FE
:10DC5B00C037F05CC148F05DC149F05EC14AF05F6E
:10DC6B00C14BF034C144F035C145F036C146F037F5
:10DC7B00C147F02CEC2AF044C038F045C039F046CF
:10DC8B00C03AF047C03BF0A6EC28F034C078F13531
:10DC9B00C079F136C07AF137C07BF174C134F075BD
:10DCAB00C135F076C136F077C137F078C138F079ED
:10DCBB00C139F07AC13AF07BC13BF0A6EC28F034C5
:10DCCB00C09CF135C09DF136C09EF137C09FF19CD1
:10DCDB00C1B8F19DC1B9F19EC1BAF19FC1BBF1B8F9
:10DCEB00C190F1B9C191F1BAC192F1BBC193F100ED
:10DCFB000E01019015B86FF00E9115B96FFF0E92D2
:10DD0B0015BA6FFF0E9315BB6FB8C19CF1B9C19DCE
:10DD1B00F1BAC19EF1BBC19FF174C164F075C165CD
:10DD2B00F076C166F077C167F09CC160F09DC16170
:10DD3B00F09EC162F09FC163F06FEC12F060C09473
:10DD4B00F161C095F162C096F163C097F178C16043
:10DD5B00F079C161F07AC162F07BC163F094C16468
:10DD6B00F095C165F096C166F097C167F06FEC1244
:10DD7B00F060C064F161C065F162C066F163C067B9
:10DD8B00F19CC144F09DC145F09EC146F09FC14737
:10DD9B00F0000E486E400E496E760E4A6E3F0E4BEB
:10DDAB006E2CEC2AF044C020F145C021F146C02274
:10DDBB00F147C023F14F0E486E380E496E760E4A6E
:10DDCB006E3F0E4B6E64C144F065C145F066C146B3
:10DDDB00F067C147F02CEC2AF044C038F045C0394D
:10DDEB00F046C03AF047C03BF0C60E486E230E49D2
:10DDFB006EF60E4A6EB80E4B6E9CC144F09DC1453B
:10DE0B00F09EC146F09FC147F02CEC2AF044C03481
:10DE1B00F045C035F046C036F047C037F0A6EC28C9
:10DE2B00F034C058F135C059F136C05AF137C05BE8
:10DE3B00F158C134F059C135F05AC136F05BC137D6
:10DE4B00F0A0C1ADF0A1C1AEF00001D890AD37AEDE
:10DE5B0037D890AD37AE379B0EAD25F66EEE0EAEC6
:10DE6B0021F76EF86A000EF8220900F5CF38F00999
:10DE7B0000F5CF39F00900F5CF3AF00A00F5CF3BAA
:10DE8B00F0A6EC28F034C024F135C025F136C026BD
:10DE9B00F137C027F17CC101F07DC102F07EC103D7
:10DEAB00F07FC104F0010E8BEC1CF001C0B0F1024D
:10DEBB00C0B1F103C0B2F104C0B3F124C138F025F5
:10DECB00C139F026C13AF027C13BF020C134F02113
:10DEDB00C135F022C136F023C137F0A6EC28F0345F
:10DEEB00C058F135C059F136C05AF137C05BF1A0BB
:10DEFB00C1ADF0A1C1AEF00001D890AD37AE37D8AF
:10DF0B0090AD37AE37A30EAD25F66EEE0EAE21F704
:10DF1B006EF86A000EF8220900F5CF38F00900F50B
:10DF2B00CF39F00900F5CF3AF00A00F5CF3BF058A6
:10DF3B00C134F059C135F05AC136F05BC137F0A688
:10DF4B00EC28F034C008F135C009F136C00AF137BE
:10DF5B00C00BF108C134F009C135F00AC136F00B22
:10DF6B00C137F0B0C138F0B1C139F0B2C13AF0B33A
:10DF7B00C13BF0A6EC28F034C080F135C081F136FE
:10DF8B00C082F137C083F180C1B8F181C1B9F18290
:10DF9B00C1BAF183C1BBF1B8C190F1B9C191F1BA6A
:10DFAB00C192F1BBC193F1000E01019015B86FF056
:10DFBB000E9115B96FFF0E9215BA6FFF0E9315BB2D
:10DFCB006FB8C180F1B9C181F1BAC182F1BBC18314
:10DFDB00F1B0C164F0B1C165F0B2C166F0B3C16715
:10DFEB00F080C160F081C161F082C162F083C163D6
:10DFFB00F06FEC12F060C094F161C095F162C096C5
:10E00B00F163C097F1A0C1ADF0A1C1AEF00001D892
:10E01B0090AD37AE37D890AD37AE37A30EAD25F6F2
:10E02B006EEE0EAE21F76EF86A000EF8220900F5BF
:10E03B00CF64F00900F5CF65F00900F5CF66F00A63
:10E04B0000F5CF67F094C160F095C161F096C162A5
:10E05B00F097C163F06FEC12F060C040F161C0410A
:10E06B00F162C042F163C043F120C164F021C1658C
:10E07B00F022C166F023C167F040C160F041C1617D
:10E08B00F042C162F043C163F06FEC12F060C00C60
:10E09B00F161C00DF162C00EF163C00FF124C160DC
:10E0AB00F025C161F026C162F027C163F00CC16499
:10E0BB00F00DC165F00EC166F00FC167F06FEC1289
:10E0CB00F060C01CF161C01DF162C01EF163C01F86
:10E0DB00F1A9C0B8F1AAC0B9F1ABC0BAF1ACC0BBE1
:10E0EB00F1B8C190F1B9C191F1BAC192F1BBC19331
:10E0FB00F1000E01019015B86FF00E9115B96FFF7D
:10E10B000E9215BA6FFF0E9315BB6FB8C128F1B9FC
:10E11B00C129F1BAC12AF1BBC12BF180C148F081F1
:10E12B00C149F082C14AF083C14BF028C164F02988
:10E13B00C165F02AC166F02BC167F0A9C060F0AAD7
:10E14B00C061F0ABC062F0ACC063F06FEC12F0607A
:10E15B00C044F061C045F062C046F063C047F02C8C
:10E16B00EC2AF044C010F145C011F146C012F14742
:10E17B00C013F110C134F011C135F012C136F013D8
:10E18B00C137F01CC148F01DC149F01EC14AF01F38
:10E19B00C14BF0A9C044F0AAC045F0ABC046F0ACEF
:10E1AB00C047F02CEC2AF044C038F045C039F0469B
:10E1BB00C03AF047C03BF0A6EC28F034C064F13510
:10E1CB00C065F136C066F137C067F128C144F0294C
:10E1DB00C145F02AC146F02BC147F080C148F08100
:10E1EB00C149F082C14AF083C14BF02CEC2AF044B8
:10E1FB00C09CF145C09DF146C09EF147C09FF164A4
:10E20B00C134F065C135F066C136F067C137F09C9B
:10E21B00C138F09DC139F09EC13AF09FC13BF0A6C9
:10E22B00EC28F034C0B4F135C0B5F136C0B6F137D7
:10E23B00C0B7F1B4C1B8F1B5C1B9F1B6C1BAF1B754
:10E24B00C1BBF1B8C1ACF1B9C1ADF1BAC1AEF1BB53
:10E25B00C1AFF10101AFBF3ED0AC05000EAD59000F
:10E26B000EAE59430EAF59D8A035D0CA0E486EF238
:10E27B000E496E490E4A6E710E4B6E88C144F08981
:10E28B00C145F08AC146F08BC147F02CEC2AF04413
:10E29B00C0A4F145C0A5F146C0A6F147C0A7F1A4A3
:10E2AB00C144F0A5C145F0A6C146F0A7C147F0CACD
:10E2BB000E486EF20E496E490E4A6E710E4B6E2C65
:10E2CB00EC2AF044C0A5F045C0A6F046C0A7F04725
:10E2DB00C0A8F01200430EAF19AC11AD11AE11D89E
:10E2EB00A46ED09CC164F09DC165F09EC166F09F89
:10E2FB00C167F0B4C160F0B5C161F0B6C162F0B7EF
:10E30B00C163F06FEC12F060C068F061C069F0623D
:10E31B00C06AF063C06BF03C0E386EAA0E396E38D3
:10E32B000E3A6E330E3B6E64C134F065C135F06648
:10E33B00C136F067C137F0A6EC28F034C06CF0356D
:10E34B00C06DF036C06EF037C06FF0E0EC18F00027
:10E35B0001D8B0EED0CA0E486EF20E496E490E4A85
:10E36B006E710E4B6E88C144F089C145F08AC1466F
:10E37B00F08BC147F02CEC2AF044C0A4F145C0A5AA
:10E38B00F146C0A6F147C0A7F1A4C144F0A5C14511
:10E39B00F0A6C146F0A7C147F0CA0E486EF20E496F
:10E3AB006E490E4A6E710E4B6E2CEC2AF044C0A5D2
:10E3BB00F045C0A6F046C0A7F047C0A8F01200FF7A
:10E3CB000EAC150001AD6FFF0E0101AD150001AED6
:10E3DB006FFF0E0101AE150001AF6F7F0E0101AF94
:10E3EB00150001B06FB0BF3ED0AD05000EAE591693
:10E3FB000EAF59430EB059D8A035D0600E486E42BF
:10E40B000E496EA20E4A6E0D0E4B6E88C144F089FA
:10E41B00C145F08AC146F08BC147F02CEC2AF04481
:10E42B00C0A4F145C0A5F146C0A6F147C0A7F1A411
:10E43B00C144F0A5C145F0A6C146F0A7C147F060A5
:10E44B000E486E420E496EA20E4A6E0D0E4B6E2C8E
:10E45B00EC2AF044C0A5F045C0A6F046C0A7F04793
:10E46B00C0A8F01200160E0101AE1962E1C30EAF87
:10E47B0019AC11AD11D8A45CD09CC164F09DC165E1
:10E48B00F09EC166F09FC167F0B4C160F0B5C16189
:10E49B00F0B6C162F0B7C163F06FEC12F060C06808
:10E4AB00F061C069F062C06AF063C06BF064C16C6C
:10E4BB00F065C16DF066C16EF067C16FF0E0EC18EE
:10E4CB00F00001D8A035D0600E486E420E496EA206
:10E4DB000E4A6E0D0E4B6E88C144F089C145F08A11
:10E4EB00C146F08BC147F02CEC2AF044C0A4F14597
:10E4FB00C0A5F146C0A6F147C0A7F1A4C144F0A541
:10E50B00C145F0A6C146F0A7C147F0600E486E4268
:10E51B000E496EA20E4A6E0D0E4B6E2CEC2AF04479
:10E52B00C0A5F045C0A6F046C0A7F047C0A8F012A2
:10E53B0000FF0E0101AC152C6FFF0EAD152D6FFFFB
:10E54B000EAE152E6F7F0EAF152F6F170E0001AD90
:10E55B006F2CC1AEF02DC1AFF02EC1B0F02FC1B1F9
:10E56B00F0AD6701D007D0B135B133B033AF33AEB7
:10E57B0033AD2FF6D7810E0001AE250101A06FFF41
:10E58B000E0001AF210101A16FFF0E0001B02101AF
:10E59B0001A26FFF0E0001B1210101A36F000E7CE0
:10E5AB006F000E7D6F000E7E6F000E7F6F2FBFFC16
:10E5BB00D02C05000E2D59000E2E593F0E2F59D879
:10E5CB00A0F3D0A0C1ADF0010E0001AD27000EAE3F
:10E5DB006F000EAF6F800EB06F000EB16FAD6701A5
:10E5EB00D007D0B135B133B033AF33AE33AD2FF637
:10E5FB00D70101AC510001AE2501017C6FAD51007B
:10E60B0001AF2101017D6FAE510001B02101017EEF
:10E61B006FAF510001B12101017F6F810E0001AD80
:10E62B006FFF0EAE6FFF0EAF6FFF0EB06F170EB119
:10E63B006F7CC1B2F07DC1B3F07EC1B4F07FC1B5C8
:10E64B00F0B16701D007D0B535B533B433B333B2BE
:10E65B0033B12FF6D70001B251AD250101A06F00E8
:10E66B000E0001AE210101A16F000E0001AF2101CF
:10E67B0001A26F000E0001B0210101A36FA0C1AD7B
:10E68B00F0FF0E0001AE6FFF0EAF6F7F0EB06F008D
:10E69B000EB16FAD6701D007D0B135B133B033AF29
:10E6AB0033AE33AD2FF6D70001AE1DB26FAF1DB336
:10E6BB006FB01DB46FB11DB56F01017C510001B27C
:10E6CB00150101B86F7D510001B3150101B96F7EC2
:10E6DB00510001B4150101BA6F7F510001B515014D
:10E6EB0001BB6FB8C1B0F1B9C1B1F1BAC1B2F1BBE5
:10E6FB00C1B3F1A05117080001AD6FFF0E01017CF2
:10E70B00150001AE6FFF0E01017D150001AF6F7F8C
:10E71B000E01017E150001B06F000E01017F150087
:10E72B0001B16F000EAE11B26F000EAF11B36F805F
:10E73B000EB011B46F000EB111B56FAD6701D007FC
:10E74B00D0B535B533B433B333B233AD2FF6D7B20F
:10E75B00C07CF1B3C07DF1B4C07EF1B5C07FF101D7
:10E76B0001AFAF08D07F1F7E1F7D1F7C6D000E7D1C
:10E77B00237E237F239CC160F09DC161F09EC1620B
:10E78B00F09FC163F0B0C164F0B1C165F0B2C16676
:10E79B00F0B3C167F06FEC12F060C09CF161C09DEB
:10E7AB00F162C09EF163C09FF164C134F065C13565
:10E7BB00F066C136F067C137F09CC138F09DC139A6
:10E7CB00F09EC13AF09FC13BF0A6EC28F034C0B0EC
:10E7DB00F135C0B1F136C0B2F137C0B3F1B0C1B849
:10E7EB00F1B1C1B9F1B2C1BAF1B3C1BBF1B8C190CA
:10E7FB00F1B9C191F1BAC192F1BBC193F1000E0114
:10E80B00019015B86F800E9115B96FFF0E9215BA66
:10E81B006FFF0E9315BB6FB8C1B0F1B9C1B1F1BAAF
:10E82B00C1B2F1BBC1B3F1B0C144F0B1C145F0B25B
:10E83B00C146F0B3C147F0000E486E720E496E31FF
:10E84B000E4A6E3F0E4B6E2CEC2AF044C074F14511
:10E85B00C075F146C076F147C077F19CC164F09D5D
:10E86B00C165F09EC166F09FC167F0B0C160F0B1A9
:10E87B00C161F0B2C162F0B3C163F06FEC12F06032
:10E88B00C094F161C095F162C096F163C097F11825
:10E89B000E486E720E496E310E4A6E3F0E4B6E94E1
:10E8AB00C164F095C165F096C166F097C167F064DD
:10E8BB00C160F065C161F066C162F067C163F06F62
:10E8CB00EC12F060C044F061C045F062C046F063EA
:10E8DB00C047F02CEC2AF044C014F145C015F146AA
:10E8EB00C016F147C017F114C134F015C135F0163D
:10E8FB00C136F017C137F08C0E486EBE0E496EBF95
:10E90B000E4A6E350E4B6EB0C144F0B1C145F0B23C
:10E91B00C146F0B3C147F02CEC2AF044C038F045A7
:10E92B00C039F046C03AF047C03BF0A6EC28F034B3
:10E93B00C078F135C079F136C07AF137C07BF1740C
:10E94B00C134F075C135F076C136F077C137F07848
:10E95B00C138F079C139F07AC13AF07BC13BF0A6EE
:10E96B00EC28F034C0B4F135C0B5F136C0B6F13790
:10E97B00C0B7F174C164F075C165F076C166F0770C
:10E98B00C167F0B4C160F0B5C161F0B6C162F0B758
:10E99B00C163F06FEC12F060C094F161C095F1624D
:10E9AB00C096F163C097F178C160F079C161F07ADC
:10E9BB00C162F07BC163F094C164F095C165F096C0
:10E9CB00C166F097C167F06FEC12F060C044F16163
:10E9DB00C045F162C046F163C047F1B4C144F0B524
:10E9EB00C145F0B6C146F0B7C147F0B4C148F0B568
:10E9FB00C149F0B6C14AF0B7C14BF02CEC2AF04438
:10EA0B00C0B0F145C0B1F146C0B2F147C0B3F10E91
:10EA1B000E386EEA0E396EDD0E3A6EB50E3B6E4C4D
:10EA2B000E486EBB0E496E310E4A6E330E4B6EB0F6
:10EA3B00C144F0B1C145F0B2C146F0B3C147F02CAF
:10EA4B00EC2AF044C034F045C035F046C036F047F0
:10EA5B00C037F0A6EC28F034C0A4F135C0A5F136D0
:10EA6B00C0A6F137C0A7F1550E386EB30E396E8ABA
:10EA7B000E3A6E380E3B6EB0C148F0B1C149F0B2E0
:10EA8B00C14AF0B3C14BF0A4C144F0A5C145F0A6F7
:10EA9B00C146F0A7C147F02CEC2AF044C034F04536
:10EAAB00C035F046C036F047C037F0A6EC28F0343E
:10EABB00C054F135C055F136C056F137C057F1612E
:10EACB000E386E0B0E396E360E3A6EBB0E3B6EB0B9
:10EADB00C148F0B1C149F0B2C14AF0B3C14BF054D7
:10EAEB00C144F055C145F056C146F057C147F02C13
:10EAFB00EC2AF044C034F045C035F046C036F04740
:10EB0B00C037F0A6EC28F034C048F135C049F136D7
:10EB1B00C04AF137C04BF1AB0E386EAA0E396E2AD4
:10EB2B000E3A6E3E0E3B6EB0C148F0B1C149F0B229
:10EB3B00C14AF0B3C14BF048C144F049C145F04A5A
:10EB4B00C146F04BC147F02CEC2AF044C034F045E1
:10EB5B00C035F046C036F047C037F0A6EC28F0348D
:10EB6B00C038F135C039F136C03AF137C03BF1B49A
:10EB7B00C160F0B5C161F0B6C162F0B7C163F0B06E
:10EB8B00C148F0B1C149F0B2C14AF0B3C14BF03842
:10EB9B00C144F039C145F03AC146F03BC147F02CB6
:10EBAB00EC2AF044C064F045C065F046C066F047FF
:10EBBB00C067F06FEC12F060C080F161C081F16250
:10EBCB00C082F163C083F1000E386E000E396E0007
:10EBDB000E3A6EC00E3B6E80C134F081C135F082AF
:10EBEB00C136F083C137F0A6EC28F034C01FF035E6
:10EBFB00C020F036C021F037C022F080C148F08130
:10EC0B00C149F082C14AF083C14BF0B4C144F0B5A5
:10EC1B00C145F0B6C146F0B7C147F02CEC2AF04421
:10EC2B00C01BF045C01CF046C01DF047C01EF005D0
:10EC3B00EC26F01BC03CF11CC03DF11DC03EF11E8B
:10EC4B00C03FF144C138F045C139F046C13AF047F5
:10EC5B00C13BF044C148F045C149F046C14AF047B9
:10EC6B00C14BF0B4C144F0B5C145F0B6C146F0B7E5
:10EC7B00C147F02CEC2AF044C034F045C035F046C7
:10EC8B00C036F047C037F0A6EC28F034C018F13589
:10EC9B00C019F136C01AF137C01BF13CC160F03D11
:10ECAB00C161F03EC162F03FC163F018C164F0195D
:10ECBB00C165F01AC166F01BC167F06FEC12F06012
:10ECCB00C04CF161C04DF162C04EF163C04FF1B465
:10ECDB00C164F0B5C165F0B6C166F0B7C167F04C61
:10ECEB00C160F04DC161F04EC162F04FC163F06F76
:10ECFB00EC12F060C094F161C095F162C096F163C3
:10ED0B00C097F1000E0001606F000E616F800E6204
:10ED1B006F3F0E636F94C164F095C165F096C16649
:10ED2B00F097C167F06FEC12F060C0B4F161C0B541
:10ED3B00F162C0B6F163C0B7F1B4C1B8F1B5C1B9F6
:10ED4B00F1B6C1BAF1B7C1BBF1B8C1ACF1B9C1AD44
:10ED5B00F1BAC1AEF1BBC1AFF17CC1ADF07DC1AEBB
:10ED6B00F07EC1AFF07FC1B0F0170ED8900001ADAF
:10ED7B0037AE37AF37B037E82EF8D7AD510101AC0E
:10ED8B00270001AE510101AD230001AF510101AECE
:10ED9B00230001B0510101AF23170E0001AD6FAC81
:10EDAB00C1AEF0ADC1AFF0AEC1B0F0AFC1B1F0AD1F
:10EDBB006701D007D0B135B133B033AF33AE33AD1C
:10EDCB002FF6D70001B1BF07D0B151B011AF111A57
:10EDDB00E1AE05D8B017D0B4C160F0B5C161F0B6E3
:10EDEB00C162F0B7C163F07CC164F07DC165F0BA5C
:10EDFB00EC21F060C0B4F161C0B5F162C0B6F16353
:10EE0B00C0B7F110D0ACC1B8F1ADC1B9F1AEC1BA58
:10EE1B00F1AFC1BBF1B8C1B4F1B9C1B5F1BAC1B66B
:10EE2B00F1BBC1B7F188C144F089C145F08AC14635
:10EE3B00F08BC147F0B4C148F0B5C149F0B6C14A37
:10EE4B00F0B7C14BF02CEC2AF044C0A5F045C0A69E
:10EE5B00F046C0A7F047C0A8F0120000A9AAAA3E2E
:10EE6B0098CA4CBE0DF5113E4712DABD25AC7C3D60
:10EE7B006937AC3168212233B40F14336821A233C4
:10EE8B003863ED3EDA0F493F5E987B3FDA0FC93F9F
:10EE9B0000000000DCCFD1350000000000C0153FA2
:10EEAB006042A20D70A5EC363BAAB83F4F38763FB7
:10EEBB003CAA38338CBEBF350072313F1872313FDC
:10EECB004CBB31330EEADDB555B38A38610B36BB1B
:10EEDB00ABAA2A3E42F1533E55326C3E05A38B3E04
:10EEEB00ABAAAA3EB76DDB3E9A99193F6042A20DC1
:10EEFB00CAF249710000804B0000000000000000C6
:10EF0B0000000000001E232D3F1E00000000001E0D
:10EF1B00373F331E000000333F3F3F1E1E0C0000E7
:10EF2B0000080C1E3F1E0C080000000C0C3F3F3F5E
:10EF3B000404000000081C1E3F3F040400000000F6
:10EF4B0000000000000000000000000000000000B6
:10EF5B0000000000000000000000000000000000A6
:10EF6B000000000000000018300E1111110E0000FF
:10EF7B00000E1111110E0E04000000000000000025
:10EF8B000000000000203C24243C3C070300000050
:10EF9B00081E33121E0800000000010F3F0F07016F
:10EFAB0000000000203C3F3C3820000000081C08FB
:10EFBB000808081C0800000A0A0A0A0A000A0000CE
:10EFCB00001F1716141414141400001C020C121634
:10EFDB0008100E000000003F3F0000000000081C5E
:10EFEB00080808081C08001C00081C08080808086A
:10EFFB000800000808080808081C0800000000109A
:10F00B003F1000000000000000023F020000000063
:10F01B00000000010101013F0000000000123F123F
:10F02B0000000000000008081C1E1E3F000000002E
:10F03B003F1E1E1C0808000000000000000000001E
:10F04B000000000404040404000400000A0A0A007F
:10F05B000000000000000014143E0A1F050500000C
:10F06B00041E05070C14140F04000022150A0C14BF
:10F07B002A11000000040A0E262D191E000004049C
:10F08B00040000000000000030080404040404081D
:10F09B0030000304080808080804030000041B06DA
:10F0AB000A000000000000000004041F040400001C
:10F0BB000000000000000C0C0804000000001E0003
:10F0CB00000000000000000000000C0C00002010ED
:10F0DB0010080C0402020100000E11111111110E87
:10F0EB000000000605040404041F0000000E1010AD
:10F0FB000804021E0000001E10100C10100E000061
:10F10B0000080C0A091F08080000001E02020E105E
:10F11B00100E0000001C02010D13110E0000001E4A
:10F12B001008040402020000000E11090E11110E4A
:10F13B000000000E11111E10080700000000000C4B
:10F14B000C000C0C00000000000C0C000C0C080454
:10F15B00000000100C030C100000000000003F002A
:10F16B003F00000000000001061806010000001E11
:10F17B001210080400040000001E111D153D011E95
:10F18B000000000C0C0A121E12210000000F1111BE
:10F19B000F11110F0000001C02010101021C0000E5
:10F1AB00000F11111111110F0000001E02020E02AF
:10F1BB00021E0000001E02020E0202020000001CD2
:10F1CB0002011911121C0000001111111F11111154
:10F1DB000000001F04040404041F0000000E0808B4
:10F1EB0008080806000000110905030509110000B5
:10F1FB00000202020202021E000000111B1B171567
:10F20B001511000000111317151919110000000E2C
:10F21B0011111111110E0000000F11110F0101013D
:10F22B000000000E11111111110E30000007090919
:10F23B00070509110000001C02020C10100E000043
:10F24B00001F040404040404000000111111111127
:10F25B00110E000000211112120A0C040000001103
:10F26B001515150F0A0A00000021120C080C1221AB
:10F27B00000000110A0A040404040000001F100817
:10F28B000402011F00001C040404040404041C00F9
:10F29B00010202040408101020000E0808080808D8
:10F2AB0008080E000004040A0A0A110000000000FE
:10F2BB000000000000003F000408000000000000F8
:10F2CB0000000000000E101C123E00000101010D99
:10F2DB001311110F00000000001E0101011E0000A0
:10F2EB001010101E1111191600000000000E111F36
:10F2FB00011E00001804041E040404040000000096
:10F30B00001E11111916100E0101011D13111111FF
:10F31B0000000800000E0808080800000800000E96
:10F32B00080808080807020202120A060A1200005F
:10F33B00070404040404040400000000001F151556
:10F34B00151500000000001D131111110000000025
:10F35B00000E1111110E00000000000D1311110F02
:10F36B0001010000001E1111191610100000001AE7
:10F37B001602020200000000001C020C100E00001E
:10F38B000004041E040404180000000000111111F5
:10F39B0019170000000000110A0A0A0400000000FF
:10F3AB0000252D2D12120000000000110A040A1175
:10F3BB0000000000002112120C0C04030000001FBF
:10F3CB000804021F00001C040404020404041C00B3
:10F3DB00040404040404040404000E0808081008C0
:10F3EB0008080E0000000000273900000000000094
:10F3FB00040A1111111F0000001C02010101021C63
:10F40B00080C000A00111111191700001008000E4A
:10F41B00111F011E0000040A000E101C123E0000FA
:10F42B00000A000E101C123E00000204000E101CFD
:10F43B00123E00000008140E101C123E00000000CB
:10F44B00001E0101011E080C040A000E111F011EF3
:10F45B000000000A000E111F011E00000204000E26
:10F46B00111F011E0000000A000E0808080800000A
:10F47B00040A000E0808080800000204000E080821
:10F48B00080800000A0C0C0A121E122100001C08AE
:10F49B000C14121E22210000101E02020E02021E6C
:10F4AB0000000000001B243E053B000000380C0C44
:10F4BB001A0A0E390000040A000E1111110E000079
:10F4CB00000A000E1111110E00000204000E1111A2
:10F4DB00110E0000040A001111111917000002048B
:10F4EB000011111119170000000A002112120C0C47
:10F4FB0004030A0E11111111110E00000A11111142
:10F50B001111110E00000000001E1915130F000041
:10F51B00001804040E04041E0000001E1915151318
:10F52B00130F0000000000110A040A1100001C0454
:10F53B00040E0404040404071008000E101C123EF1
:10F54B0000000804000E0808080800000804000E5C
:10F55B001111110E000008040011111119170000F0
:10F56B000A0E001D1311111100000A15131715199E
:10F57B0019110000000E0E0A1E0000000000000C06
:10F58B0012120C000000000000000008000804022A
:10F59B00121E000E1117110E0000000000000000DB
:10F5AB001F101000000000130A0A3C221A39000039
:10F5BB0000130A0A1C163E11000000000004000490
:10F5CB0004040404000000140A050A1400000000DF
:10F5DB0000050A140A05000015001500150015009A
:10F5EB0015002A152A152A152A152A153F153F1518
:10F5FB003F153F153F1508080808080808080808B4
:10F60B00080808080F0808080808080C0C0A121E3E
:10F61B0012210000040E0C0A121E12210000020C13
:10F62B000C0A121E12210000001E212D252D211E59
:10F63B0000001414141710171414141414141414A5
:10F64B001414141414140000001F101714141414A1
:10F65B0014141417101F0000000000081C0A0A0ADB
:10F66B001C0800000021120C0E040E040000000008
:10F67B0000000F08080808080808080838000000F0
:10F68B000000080808083F00000000000000000010
:10F69B003F08080808080808080838080808080878
:10F6AB00000000003F0000000000080808083F08A9
:10F6BB00080808080A0E000E101C123E00000A0D66
:10F6CB000C0A121E1221000014141434043C000006
:10F6DB0000000000003C04341414141414141437E8
:10F6EB00003F000000000000003F0037141414140A
:10F6FB00141414340434141414140000003F003F89
:10F70B0000000000141414370037141414140021D3
:10F71B001E12121E210000000B06091E1111110EE4
:10F72B000000000F11111311110F0000041E020233
:10F73B000E02021E00000A1E02020E02021E000032
:10F74B00041E02020E02021E00000000000E08083A
:10F75B0008080000081F04040404041F0000041F11
:10F76B0004040404041F00000A1F04040404041FFF
:10F77B000000080808080F0000000000000000004F
:10F78B003808080808083F3F3F3F3F3F3F3F3F3F98
:10F79B0000000000003F3F3F3F3F04040400000017
:10F7AB0004040400041F04040404041F00003F3F6E
:10F7BB003F3F3F0000000000080E11111111110E08
:10F7CB0000000E0909050509111D0000040E111199
:10F7DB001111110E0000040E11111111110E000068
:10F7EB000A0E000E1111110E00000A0F111111114A
:10F7FB00110E000000000011111119170101010178
:10F80B00010D1311110F010100010F1111110F0146
:10F81B000000081511111111110E0000041B11111C
:10F82B001111110E0000041911111111110E00000C
:10F83B001008002112120C0C040310190A0A0404FC
:10F84B00040400003F00000000000000000008045A
:10F85B000000000000000000000000001E0000007F
:10F86B000000000004041F04041F0000000000003F
:10F87B00000000003F000027130F1C143E11000076
:10F88B00001F1716141414141400001C020C12166B
:10F89B0008100E0000000004001F00040000000010
:10F8AB00000000000000080C00040A040000000027
:10F8BB0000000A0000000000000000000000000033
:10F8CB00000C0C000000000C0808000000000000F9
:10F8DB00001C081C000000000000000E040E0000BD
:10F8EB00000000000000003F3F3F3F3F00000000D2
:10F8FB000000000000000000000000000000040AEF
:10F90B000E0A0400040E0A0E0400000A0E0E040078
:10F91B0000040E0E0400040E0E040E0004040E046C
:10F92B000E000000000000000000000000000000BE
:10F93B0000000000000000000000000C080606009C
:10F94B00040A040E0400000000000000040C0A0866
:10F95B000400040E0A0E040002060E060200080C38
:10F96B000E0C0800040E040E04000A0A0A000A001A
:10F97B000008040404040404040402000000000052
:10F98B000E00040E040E040E040E04040400040402
:10F99B00040E040000040F04000000020F0200001C
:10F9AB000000020E0000000A0E0A000000040E0EFA
:10F9BB000000000E0E040000000000000000040414
:10F9CB00040004000A0A000000000A0E0A0E0A00D6
:10F9DB00040C060C0604020804020800040A0C0AB4
:10F9EB000E000602000000000402020204000204E2
:10F9FB00040402000A040E040A0000040E040000B2
:10FA0B0000000000060200000E00000000000000D5
:10FA1B0004000808040202000C0A0A0A0600040685
:10FA2B0004040E00060804020E0006080408060073
:10FA3B00080A0E0808000E02060806000402060A51
:10FA4B0004000E080C040400040A040A0400040A4F
:10FA5B000C0804000000040004000000040006026F
:10FA6B0008040204080000000E000E000204080443
:10FA7B0002000608040004000E0A0A020E00040A23
:10FA8B000E0A0A00060A060A06000C0202020C0005
:10FA9B00060A0A0A06000E0206020E000E020602F3
:10FAAB0002000C020A0A0C000A0A0E0A0A000E04D3
:10FABB0004040E000808080A04000A0A060A0A00D1
:10FACB00020202020E000A0E0E0A0A000A0E0A0AAF
:10FADB000A00040A0A0A0400060A06020200040AC3
:10FAEB000A0E0C00060A060A0A000C020E08060093
:10FAFB000E04040404000A0A0A0A0E000A0A0A0A7F
:10FB0B0004000A0A0E0E0A000A0A040A0A000A0A6C
:10FB1B00040404000E0804020E0006020202060092
:10FB2B00020204080800060404040600040A00008C
:10FB3B00000000000000000F0604000000000000A1
:10FB4B000C0A0E000202060A060000000C020C0052
:10FB5B0008080C0A0C0000000E060C0008040E042A
:10FB6B00040000000E0A080E0202060A0A00040036
:10FB7B000404040004000404040602020A060A003A
:10FB8B0004040404040000000E0E0A000000060A20
:10FB9B000A000000040A04000000060A0602000026
:10FBAB000C0A0C0800000602020000000C04060000
:10FBBB0000040E040C0000000A0A0E0000000A0AE2
:10FBCB00040000000A0E0E0000000A040A000000E8
:10FBDB000A0A0402000006040C000C0406040C00C4
:10FBEB0004040404040006040C0406000A050000C7
:10FBFB00000000040A0E00000C02020E04020A00B0
:10FC0B000A0A0C0008040E060C00040A0C0A0E006B
:10FC1B000A000C0A0E0002040C0A0E0004000C0A67
:10FC2B000E00000E020E0406040A0E060C000A005B
:10FC3B000E060C0002040E060C000A00040404005D
:10FC4B00040A000404000204000404000A040A0E5F
:10FC5B000A0004040A0E0A0008040E060E00000037
:10FC6B000C0E06000C060E060E00040A040A040015
:10FC7B000A00040A04000204040A0400040A000A2D
:10FC8B000E0002040A0A0E000A000A0A04020A0401
:10FC9B000A0A04000A000A0A0E00040E020E0400EF
:10FCAB0008040E040E000A0E040E04000006060AD9
:10FCBB000A000C040C04060008040C0A0E000804CD
:10FCCB000004040008040E0A0E000804000A0E00CB
:10FCDB000E000E0A0A000E000A0E0A000C0A0E0095
:10FCEB000E00040A04000E00040004020C00000EB7
:10FCFB0002020000000704040000020A040A0C00C0
:10FD0B00020A040E0800040004040400000A050A99
:10FD1B00000000050A0500000208020802080A0597
:10FD2B000A050A050D070D070D0704040404040456
:10FD3B000404070404040407040704040A0A0B0A56
:10FD4B000A0A00000F0A0A0A0007040704040A0B38
:10FD5B00080B0A0A0A0A0A0A0A0A000F080B0A0AFF
:10FD6B000A0B080F00000A0A0F0000000407040723
:10FD7B00000000000704040404040C000000040449
:10FD8B000F00000000000F04040404040C0404041E
:10FD9B0000000F00000004040F040404040C040C06
:10FDAB0004040A0A0A0A0A0A0A0A020E0000000ED2
:10FDBB00020A0A0A0A0B000F0000000F000B0A0AC6
:10FDCB000A0A020A0A0A000F000F00000A0B000BB6
:10FDDB000A0A040F000F00000A0A0F000000000FB0
:10FDEB00000F040400000F0A0A0A0A0A0E000000A2
:10FDFB00040C040C0000000C040C040400000E0A9C
:10FE0B000A0A0A0A0B0A0A0A040F000F0404040464
:10FE1B000700000000000C0404040F0F0F0F0F0F5E
:10FE2B000000000F0F0F0303030303030C0C0C0C58
:10FE3B000C0C0F0F0F00000000000E060E00040A42
:10FE4B00060A06020E0A020202000E0A0A0A0A003B
:10FE5B000E0204020E0000000C0A040000000A0A45
:10FE6B000E020008060404000E040A040E00040A25
:10FE7B000E0A040000040A0A0A000C02040A040019
:10FE8B0000000E0A0E00040E0A0E04000C020E02F5
:10FE9B000C00040A0A0A0A000E000E000E00040EE3
:10FEAB0004000E00060806000E000C020C000E00EB
:10FEBB0000080404040404040404020004000E00FB
:10FECB000400000A050A0500040A040000000004EF
:10FEDB000E0400000000040000000C0404060400E3
:10FEEB000E0A0A00000006040206000000000606C7
:10FEFB0000000000000000002C632C632C632C63BB
:10FF0B00FFFFFFFF4D6B4D6B1CE71CE7139D139D14
:10FF1B002C632C632C632C63139D139D139D139DDA
:10FF2B007DEF7DEF7DEF7DEF2C632C632C632C63DA
:10FF3B00FFFFFFFF4D6B4D6B1CE71CE7139D139DE4
:10FF4B002C632C632C632C63139D139D139D139DAA
:10FF5B007DEF7DEF7DEF7DEF2C632C632C632C63AA
:10FF6B00FFFFFFFF4D6B4D6B1CE71CE7139D139DB4
:10FF7B0003F900040006000000FF00000003EF007F
:10FF8B0006000A000000FF0000000000803F000098
:10FF9B00C03F00AAB83FC623F6B80040763F257392
:10FFAB0025642E253032642020202020202000497B
:10FFBB006E69742073656E736F72732E2E2E0068CC
:10FFCB00656164696E670025332E306600252E321D
:10FFDB0066006D62617200494E46004E414E0069EB
:10FFEB006E66006E616E00616C74006C66002D00B5
:05FFFB0043004F00006F
:020000040020DA
:08000000FFFFFFFFFFFFFFFF00
:020000040030CA
:0E000000FF28183CFF3F81FF0FC00FE00F40AC
:00000001FF
